S01900006D63755F616E64726F69645F626F6172642E737265631F
S3150802000000000A203DF00208D9D80208E1D8020801
S31508020010E9D80208F1D80208F9D802088DF00208D0
S3150802002000000000000000000000000001D90208DC
S315080200300FD90208000000001DD902082BD90208B0
S315080200408DF002088DF002088DF002088DF0020884
S315080200508DF002088DF002088DF002088DF0020874
S315080200608DF002088DF002088DF002088DF0020864
S315080200708DF002088DF002088DF002088DF0020854
S315080200808DF002088DF002088DF002088DF0020844
S315080200908DF002088DF002088DF002088DF0020834
S315080200A08DF002088DF002088DF0020839D902088F
S315080200B08DF002088DF002088DF002088DF0020814
S315080200C08DF002088DF002088DF002088DF0020804
S315080200D0000000008DF002088DF002084DD90208D2
S315080200E08DF002088DF002088DF002088DF00208E4
S315080200F08DF0020861D9020875D9020889D9020861
S315080201008DF002088DF002088DF002088DF00208C3
S315080201108DF002088DF002088DF002088DF00208B3
S315080201208DF002088DF002089DD902088DF00208AA
S31508020130B1D90208C5D90208D9D902088DF0020830
S315080201408DF002088DF002088DF002088DF0020883
S315080201508DF002088DF002088DF002088DF0020873
S315080201608DF002088DF002088DF002088DF0020863
S315080201708DF002088DF002088DF002088DF0020853
S315080201808DF002088DF002088DF002088DF0020843
S315080201908DF002088DF002088DF002088DF0020833
S315080201A08DF002088DF002088DF002088DF0020823
S315080201B08DF002088DF002088DF002088DF0020813
S315080201C08DF002088DF002088DF002088DF0020803
S315080201D08DF002088DF002088DF002088DF00208F3
S315080201E08DF002088DF002088DF002088DF00208E3
S315080201F08DF002088DF002088DF002088DF00208D3
S315080202008DF002088DF002088DF002080000000049
S31508020210000000008DF00208000000008DF00208C0
S315080202208DF002088DF002088DF002088DF00208A2
S315080202308DF002088DF002088DF002088DF0020892
S315080202408DF002088DF002088DF002080000000009
S3150802025010B5054C237833B9044B13B10448AFF3F0
S3150802026000800123237010BD080200200000000050
S31508020270140C040808B5034B1BB103490348AFF332
S31508020280008008BD000000000C020020140C0408BF
S31508020290034613F8012B002AFBD1181A01387047B6
S315080202A081F0004102E000BF83F0004330B54FEA17
S315080202B041044FEA430594EA050F08BF90EA020F84
S315080202C01FBF54EA000C55EA020C7FEA645C7FEA17
S315080202D0655C00F0E2804FEA5454D4EB5555B8BF3A
S315080202E06D420CDD2C4480EA020281EA030382EAAB
S315080202F0000083EA010180EA020281EA0303362D3D
S3150802030088BF30BD11F0004F4FEA01314FF4801C0F
S315080203104CEA113102D0404261EB410113F0004F21
S315080203204FEA03334CEA133302D0524263EB4303D8
S3150802033094EA050F00F0A780A4F10104D5F1200E76
S315080203400DDB02FA0EFC22FA05F2801841F10001D1
S3150802035003FA0EF2801843FA05F359410EE0A5F1A5
S3150802036020050EF1200E012A03FA0EFC28BF4CF0D6
S31508020370020C43FA05F3C01851EBE37101F000458C
S3150802038007D54FF0000EDCF1000C7EEB00006EEB99
S315080203900101B1F5801F1BD3B1F5001F0CD3490823
S315080203A05FEA30004FEA3C0C04F101044FEA44527A
S315080203B012F5800F80F09A80BCF1004F08BF5FEA01
S315080203C0500C50F1000041EB045141EA050130BDE1
S315080203D05FEA4C0C404141EB0101013C28BFB1F5F3
S315080203E0801FE9D291F0000F04BF01460020B1FA3E
S315080203F081F308BF2033A3F10B03B3F120020CDA11
S315080204000C3208DD02F1140CC2F10C0201FA0CF0EE
S3150802041021FA02F10CE002F11402D8BFC2F1200C53
S3150802042001FA02F120FA0CFCDCBF41EA0C01904009
S31508020430E41AA2BF01EB0451294330BD6FEA040452
S315080204401F3C1CDA0C340EDC04F11404C4F120023D
S3150802045020FA04F001FA02F340EA030021FA04F34F
S3150802046045EA030130BDC4F10C04C4F1200220FAA6
S3150802047002F001FA04F340EA0300294630BD21FAE4
S3150802048004F0294630BD94F0000F83F4801306BFAA
S3150802049081F480110134013D4EE77FEA645C18BF9E
S315080204A07FEA655C29D094EA050F08BF90EA020F35
S315080204B005D054EA000C04BF1946104630BD91EA2D
S315080204C0030F1EBF0021002030BD5FEA545C05D130
S315080204D04000494128BF41F0004130BD14F580046F
S315080204E03CBF01F5801130BD01F0004545F0FE41E3
S315080204F041F470014FF0000030BD7FEA645C1ABF18
S31508020500194610467FEA655C1CBF0B46024650EA4E
S31508020510013406BF52EA033591EA030F41F400217A
S3150802052030BD00BF90F0000F04BF0021704730B500
S315080205304FF4806404F132044FF000054FF00001D5
S3150802054050E700BF90F0000F04BF0021704730B596
S315080205504FF4806404F1320410F0004548BF40426B
S315080205604FF000013EE700BF42004FEAE2014FEAC0
S3150802057031014FEA02701FBF12F07F4393F07F4F9B
S3150802058081F06051704732F07F4208BF704793F09E
S315080205907F4F04BF41F40021704730B54FF46074B1
S315080205A001F0004521F000411CE700BF50EA0102B4
S315080205B008BF704730B54FF000050AE050EA01025D
S315080205C008BF704730B511F0004502D5404261EBCD
S315080205D041014FF4806404F132045FEA915C3FF40E
S315080205E0D8AE4FF003025FEADC0C18BF03325FEAAB
S315080205F0DC0C18BF033202EBDC02C2F1200300FA5C
S3150802060003FC20FA02F001FA03FE40EA0E0021FA80
S3150802061002F11444BDE600BF70B54FF0FF0C4CF46E
S31508020620E06C1CEA11541DBF1CEA135594EA0C0F20
S3150802063095EA0C0F00F0DEF82C4481EA030621EA5B
S315080206404C5123EA4C5350EA013518BF52EA033596
S3150802065041F4801143F4801338D0A0FB02CE4FF048
S315080206600005E1FB02E506F00042E0FB03E54FF078
S315080206700006E1FB03569CF0000F18BF4EF0010E70
S31508020680A4F1FF04B6F5007F64F5407404D25FEA6C
S315080206904E0E6D4146EB060642EAC62141EA55511F
S315080206A04FEAC52040EA5E504FEACE2EB4F1FD0C61
S315080206B088BFBCF5E06F1ED8BEF1004F08BF5FEADF
S315080206C0500E50F1000041EB045170BD06F0004691
S315080206D046EA010140EA020081EA0301B4EB5C043E
S315080206E0C2BFD4EB0C0541EA045170BD41F4801136
S315080206F04FF0000E013C00F3AB8014F1360FDEBF5B
S31508020700002001F0004170BDC4F10004203C35DA36
S315080207100C341BDC04F11404C4F1200500FA05F3B9
S3150802072020FA04F001FA05F240EA020001F000425A
S3150802073021F0004110EBD37021FA04F642EB0601D0
S315080207405EEA430E08BF20EAD37070BDC4F10C04FA
S31508020750C4F1200500FA04F320FA05F001FA04F2BE
S3150802076040EA020001F0004110EBD37041F10001AA
S315080207705EEA430E08BF20EAD37070BDC4F12005B5
S3150802078000FA05F24EEA020E20FA04F301FA05F21D
S3150802079043EA020321FA04F001F0004121FA04F2C5
S315080207A020EA020000EBD3705EEA430E08BF20EA95
S315080207B0D37070BD94F0000F0FD101F000464000CF
S315080207C041EB010111F4801F08BF013CF7D041EA51
S315080207D0060195F0000F18BF704703F00046520055
S315080207E043EB030313F4801F08BF013DF7D043EA26
S315080207F00603704794EA0C0F0CEA135518BF95EADC
S315080208000C0F0CD050EA410618BF52EA4306D1D162
S3150802081081EA030101F000414FF0000070BD50EA81
S31508020820410606BF1046194652EA430619D094EA0B
S315080208300C0F02D150EA013613D195EA0C0F05D1F5
S3150802084052EA03361CBF104619460AD181EA030149
S3150802085001F0004141F0FE4141F470014FF0000001
S3150802086070BD41F0FE4141F4780170BD70B54FF09C
S31508020870FF0C4CF4E06C1CEA11541DBF1CEA13551C
S3150802088094EA0C0F95EA0C0F00F0A7F8A4EB0504FE
S3150802089081EA030E52EA03354FEA013100F08880F5
S315080208A04FEA03334FF0805545EA131343EA1263BE
S315080208B04FEA022245EA111545EA10654FEA002673
S315080208C00EF000419D4208BF964244F1FD0404F52C
S315080208D0407402D25B084FEA3202B61A65EB030588
S315080208E05B084FEA32024FF480104FF4002CB6EB45
S315080208F0020E75EB030E22BFB61A754640EA0C00C5
S315080209005B084FEA3202B6EB020E75EB030E22BF04
S31508020910B61A754640EA5C005B084FEA3202B6EB45
S31508020920020E75EB030E22BFB61A754640EA9C0004
S315080209305B084FEA3202B6EB020E75EB030E22BFD4
S31508020940B61A754640EADC0055EA060E18D04FEA92
S31508020950051545EA16754FEA06164FEAC30343EA32
S3150802096052734FEAC2025FEA1C1CC0D111F4801FFF
S315080209700BD141EA00014FF000004FF0004CB6E7F8
S3150802098011F4801F04BF01430020B4F1FD0C88BF97
S31508020990BCF5E06F3FF6AFAEB5EB030C04BFB6EBA2
S315080209A0020C5FEA500C50F1000041EB045170BD95
S315080209B00EF0004E4EEA113114EB5C04C2BFD4EBC2
S315080209C00C0541EA045170BD41F480114FF0000E46
S315080209D0013C90E645EA060E8DE60CEA135594EAC2
S315080209E00C0F08BF95EA0C0F3FF43BAF94EA0C0FC5
S315080209F00AD150EA01347FF434AF95EA0C0F7FF43A
S31508020A0025AF104619462CE795EA0C0F06D152EA8D
S31508020A1003353FF4FDAE1046194622E750EA410671
S31508020A2018BF52EA43067FF4C5AE50EA41047FF482
S31508020A300DAF52EA43057FF4EBAE12E74FF0FF3CE7
S31508020A4006E000BF4FF0010C02E000BF4FF0010CB8
S31508020A504DF804CD4FEA410C7FEA6C5C4FEA430C31
S31508020A6018BF7FEA6C5C1BD001B050EA410C0CBF80
S31508020A7052EA430C91EA030F02BF90EA020F0020E2
S31508020A80704710F1000F91EA030F58BF994208BF49
S31508020A9090422CBFD8176FEAE37040F00100704706
S31508020AA04FEA410C7FEA6C5C02D150EA013C07D15D
S31508020AB04FEA430C7FEA6C5CD6D152EA033CD3D0A8
S31508020AC05DF8040B704700BF8446104662468C46A2
S31508020AD01946634600E000BF01B5FFF7B7FF0028D5
S31508020AE048BF10F1000F01BD4DF808EDFFF7F4FFFE
S31508020AF00CBF012000205DF808FB00BF4DF808ED89
S31508020B00FFF7EAFF34BF012000205DF808FB00BFAB
S31508020B104DF808EDFFF7E0FF94BF012000205DF8CD
S31508020B2008FB00BF4DF808EDFFF7CEFF94BF012082
S31508020B3000205DF808FB00BF4DF808EDFFF7C4FF7B
S31508020B4034BF012000205DF808FB00BF4FEA410CC4
S31508020B507FEA6C5C02D150EA013C0AD14FEA430CA7
S31508020B607FEA6C5C02D152EA033C02D14FF00000E4
S31508020B7070474FF0010070474FEA410212F5001222
S31508020B8015D211D56FF47873B3EB625212D94FEAC4
S31508020B90C12343F0004343EA505311F0004F23FAAE
S31508020BA002F018BF404270474FF00000704750EA03
S31508020BB0013005D111F0004008BF6FF000407047C0
S31508020BC04FF00000704700BF4A0011D212F500121A
S31508020BD011D20DD56FF47873B3EB62520ED44FEA85
S31508020BE0C12343F0004343EA505323FA02F0704705
S31508020BF04FF00000704750EA013002D14FF0FF3043
S31508020C0070474FF0000070474FEA4102B2F1E043E5
S31508020C1024BFB3F5001CDCF1FE5C0DD901F0004CD3
S31508020C204FEAC0024CEA5070B2F1004F40EB830023
S31508020C3008BF20F00100704711F0804F21D113F14F
S31508020C403872BCBF01F00040704741F480114FEA88
S31508020C505252C2F11802C2F1200C10FA0CF320FA11
S31508020C6002F018BF40F001004FEAC1234FEAD3232E
S31508020C7003FA0CFC40EA0C0023FA02F34FEA430398
S31508020C80CCE77FEA625307D150EA01331EBF4FF021
S31508020C90FE4040F44000704701F0004040F0FE403C
S31508020CA040F40000704700BF53B94AB9002908BF8B
S31508020CB000281CBF4FF0FF314FF0FF3000F0B4B9E7
S31508020CC0ADF1080C6DE904CE00F03CF8DDF804E05D
S31508020CD0DDE9022304B0704738B500220023044632
S31508020CE00D46FFF70BFF28B920462946BDE83840CE
S31508020CF000F00AB8204605F1004100F005F8404226
S31508020D0061EB410138BD00BFD0B500220B4B064648
S31508020D100F46FFF781FCFFF757FF0446FFF702FC71
S31508020D200022074BFFF778FC02460B463046394647
S31508020D30FFF7BAFAFFF748FF2146D0BD0000F03D9B
S31508020D400000F0412DE9F04F099D0C46002B4DD1CC
S31508020D508A420F4684469646B2FA82F360D94BB166
S31508020D6002FA03FEC3F120029F4000FA03FC20FAAE
S31508020D7002F217434FEA1E461FFA8EF44FEA1C4246
S31508020D80B7FBF6F106FB117701FB04F042EA0742CC
S31508020D90904208D91EEB020201F1FF3702D29042B5
S31508020DA000F22D813946121A1FFA8CFCB2FBF6F0B4
S31508020DB006FB102200FB04F44CEA024C644508D9EF
S31508020DC01EEB0C0C00F1FF3202D2644500F21A81C6
S31508020DD0104640EA0140ACEB040C002125B12CFA7E
S31508020DE003F30022C5E90032BDE8F08F8B4205D92C
S31508020DF00DB1C5E9000100210846F5E7B3FA83F10A
S31508020E0000294DD1A342C0F0F280904280F0EF80D3
S31508020E10064623460846002DE6D0C5E90063E3E701
S31508020E20002B40F0A2808A1A4FEA1E471FFA8EF656
S31508020E300121B2FBF7F407FB14204FEA1C4242EAEF
S31508020E40004206FB04F090420FD91EEB020204F19F
S31508020E50FF382CBF4FF001094FF00009904203D921
S31508020E60B9F1000F00F0C8804446121A1FFA8CFC2A
S31508020E70B2FBF7F007FB102200FB06F64CEA024C1F
S31508020E80664508D91EEB0C0C00F1FF3202D2664504
S31508020E9000F2BB801046ACEB060C40EA04409DE724
S31508020EA0C1F120068B4004FA01FE22FA06F720FA5F
S31508020EB006FCF4408A401F434EEA0C0300FA01FE80
S31508020EC04FEA17484FEA13491FFA87FCB4FBF8F0B2
S31508020ED008FB104449EA044400FB0CF9A1450ED963
S31508020EE03C1900F1FF3A2CBF4FF0010B4FF0000BF3
S31508020EF0A14503D9BBF1000F00F093805046A4EB3D
S31508020F0009041FFA83F9B4FBF8F308FB134403FB3D
S31508020F100CFC49EA0444A44506D93C1903F1FF38F6
S31508020F2001D2A4457AD8434643EA0040A4EB0C040E
S31508020F30A0FB02984445CC46434602D306D1CE4589
S31508020F4004D20138B9EB020C68EB07035DB1BEEBBC
S31508020F500C0264EB030404FA06F622FA01F3CC4007
S31508020F601E43C5E9006400213EE702FA03FEC3F107
S31508020F70200104FA03F200FA03FCCC404FEA1E47AA
S31508020F8020FA01F11FFA8EF6B4FBF7F00A4307FBC3
S31508020F901044110C41EA044100FB06F48C420ED9B6
S31508020FA01EEB010100F1FF382CBF4FF001094FF08B
S31508020FB000098C4202D9B9F1000F2CD04046091B10
S31508020FC092B2B1FBF7F407FB141142EA014204FBA1
S31508020FD006F1914207D91EEB020204F1FF3801D24B
S31508020FE0914215D84446521A44EA004121E7861A24
S31508020FF064EB030301200EE7023C724435E702392B
S315080210007244D0E6F4440238E3E6F444023842E78E
S31508021010023C7244E7E702387144D0E7023B3C449B
S3150802102082E702383C446AE7704700BF80B400AFE3
S31508021030024B1846BD465DF8047B70474002002005
S3150802104080B582B000AF78600B467B807B881A46F3
S3150802105079684FF4804008F0D1F800BF0837BD46DA
S3150802106080BD000090B589B002AFF860B96013463A
S31508021070FB8006200AF0C4F903460133DBB23B754E
S31508021080CE237B75D623BB753B7D1946BB681B7879
S315080210901A460B480DF08CFA0CF03EFE04460CF08C
S315080210A031FE014607F11402FB880093BB6820460D
S315080210B01AF0CDFD00BF00BF1C37BD4690BD00BF6C
S315080210C0300C040880B500AF4FF480720249034819
S315080210D00AF0DEFC00BF80BD8C0B00202402002033
S315080210E080B500AFFFF7EEFF034B044A04490548F3
S315080210F01AF0F9F900BF80BD41100208651002080E
S31508021100400200203402002080B400AF034B1B6863
S315080211101846BD465DF8047B704700BF8C0C00205C
S3150802112090B595B000AF78603960ACE08E4B8F4AC7
S31508021130402178680FF02EFF0346002B40F0A3806B
S315080211408A4B1B68B3F5807F04D16821874805F06E
S3150802115091FB98E0854B1B6840F20112934204D139
S315080211606821824805F082FA8DE0804B1B68B3F548
S31508021170817F04D168217D4805F08AFA83E07B4B9A
S315080211801B6840F20312934204D16821774805F09E
S3150802119091FA78E0754B1B68B3F5827F04D1682112
S315080211A0724805F099FA6EE0704B1B6840F2051218
S315080211B0934204D168216D4805F0A0FA63E06B4BAF
S315080211C01B68B3F5837F04D16821684805F0A8FA3D
S315080211D059E0664B1B6840F20712934204D1682114
S315080211E0624805F0AFFA4EE0604B1B68B3F5847FA0
S315080211F00BD15E4BDB68032B02D15D480DF0D8F9A3
S3150802120068215A4805F0B0FA3DE0584B1B6840F28F
S315080212100912934204D16821544805F0B7FA32E01C
S31508021220524B1B68B3F5857F04D168214F4805F0F8
S31508021230C7FA28E04D4B1B6840F20B12934204D1C1
S3150802124068214A4805F0CEFA1DE0484B1B68B3F5FB
S31508021250867F04D16821454805F0D6FA13E0434B48
S315080212601B6840F20D12934204D168213F4805F0EB
S31508021270DDFA08E03D4B1B68B3F5877F03D1682189
S315080212803A4805F0E5FA402178680FF0F1FF03467F
S31508021290002B7FF44BAF786805F02AFF03461A46FF
S315080212A0344B9A60786805F0EDFE0346314A1360BE
S315080212B0786805F0FFFE03462E4A53602D4B9B685D
S315080212C0002B0CD02B4B1B682A4A526819462A480F
S315080212D00DF06EF9274B9B68184605F051FF0C2254
S315080212E0244926481CF0CAF90346002B33D0214B61
S315080212F01B68DAB207F14C03114618461AF084FF46
S315080213001C4B5B68DAB207F14C03114618461AF011
S3150802131096FF184B9B68DAB207F14C03114618463A
S315080213201AF0A8FF07F1080207F14C0311461846FE
S315080213301BF01CF807F1080318461AF0C5FF044605
S3150802134007F1080318461AF0CBFF03461A46214648
S315080213504A2002F043F9094B064A07CA83E80700FE
S3150802136000BF5437BD4690BD408400201884002033
S31508021370580C0408C8A00120680C0408D4A001204F
S3150802138080B500AF4FF4FD62AD49AE480AF080FB66
S315080213904FF4FD62AC49AD480AF07AFB4FF4FD62A0
S315080213A0AB49AC480AF074FB4FF4FD62AA49AB4854
S315080213B00AF06EFB4FF4FD62A949AA480AF068FBD7
S315080213C04FF4FD62A849A9480AF062FB4FF4FD6290
S315080213D0A749A8480AF05CFB4FF4FD62A649A7484C
S315080213E00AF056FB4FF4FD62A549A6480AF050FBDF
S315080213F04FF4FD62A449A5480AF04AFB4FF4FD6280
S31508021400A349A4480AF044FB4FF4FD62A249A34843
S315080214100AF03EFB4FF4FD62A149A2480AF038FBE6
S315080214204FF4FD62A049A1480AF032FB4FF4FD626F
S315080214309F49A0480AF02CFB4FF420729E499F4808
S315080214400AF026FB4FF47D629D499E480AF020FB6E
S315080214504FF480729C499D480AF01AFB4FF4207299
S315080214609B499C480AF014FB4FF47D629A499B48B3
S315080214700AF00EFB4FF4807299499A480AF008FB63
S315080214804FF42072984999480AF002FB4FF47D629C
S31508021490974998480AF0FCFA4FF480729649974899
S315080214A00AF0F6FA4FF42072954996480AF0F0FACD
S315080214B04FF47D62944995480AF0EAFA4FF480722D
S315080214C0934994480AF0E4FA4FF4207292499348F1
S315080214D00AF0DEFA4FF47D62914992480AF0D8FA88
S315080214E04FF48072904991480AF0D2FA4FF420726A
S315080214F08F4990480AF0CCFA4FF47D628E498F489C
S315080215000AF0C6FA4FF480728D498E480AF0C0FA7C
S315080215104FF420728C498D480AF0BAFA4FF47D626C
S315080215208B498C480AF0B4FA4FF480728A498B4880
S315080215300AF0AEFA4FF4207289498A480AF0A8FAE4
S315080215404FF47D62884989480AF0A2FA4FF48072FC
S31508021550874988480AF09CFA4FF4207286498748D8
S315080215600AF096FA4FF47D62854986480AF090FA9F
S315080215704FF48072844985480AF08AFA4FF4207239
S31508021580834984480AF084FA4FF47D628249834883
S315080215900AF07EFA4FF48072814982480AF078FA94
S315080215A04FF42072804981480AF072FA4FF47D623C
S315080215B07F4980480AF06CFA4FF480727E497F4868
S315080215C00AF066FA4FF420727D497E480AF060FAFC
S315080215D04FF47D627C497D480AF05AFA4FF48072CC
S315080215E07B497C480AF054FA4FF420727A497B48C0
S315080215F00AF04EFA4FF47D6279497A480AF048FAB7
S315080216004FF48072784979480AF042FA4FF4207208
S31508021610774978480AF03CFA4FF47D62764977486A
S315080216200AF036FA4FF48072754976480AF030FAAB
S315080216304FF48062744975480AF02AFA00BF80BDE1
S31508021640A00C0020900C002098140020881400207A
S31508021650901C0020801C002088240020782400206A
S31508021660802C0020702C002078340020683400205A
S31508021670703C0020603C002068440020584400204A
S31508021680604C0020504C002058540020485400203A
S31508021690505C0020405C002048640020386400202A
S315080216A0406C0020306C002038740020287400201A
S315080216B0307C0020207C0020B4840020A4840020F2
S315080216C074870020348700208497002044970020DE
S315080216D0B8980020A8980020789B0020389B002004
S315080216E088AB002048AB0020BCAC0020ACAC002084
S315080216F07CAF00203CAF00208CBF00204CBF0020EE
S31508021700C0C00020B0C0002080C3002040C3002013
S3150802171090D3002050D30020C4D40020B4D4002093
S3150802172084D7002044D7002094E7002054E70020FD
S31508021730C8E80020B8E8002088EB002048EB002023
S3150802174098FB002058FB0020CCFC0020BCFC0020A3
S315080217508CFF00204CFF00209C0F01205C0F01200B
S31508021760D0100120C010012090130120501301202F
S31508021770A023012060230120D4240120C4240120AF
S315080217809427012054270120A43701206437012019
S31508021790D8380120C8380120983B0120583B01203F
S315080217A0A84B0120684B0120DC4C0120CC4C0120BF
S315080217B09C4F01205C4F0120AC5F01206C5F012029
S315080217C0E0600120D0600120A0630120606301204F
S315080217D0B073012070730120E4740120D4740120CF
S315080217E0A477012064770120B48701207487012039
S315080217F0E8880120D8880120A88B0120688B01205F
S31508021800B89B0120789B0120C89C0120B89C012026
S3150802181080B483B000AF78607B68002B01D10023C7
S3150802182046E07B68012B01D1012341E07B68022B4C
S3150802183001D102233CE07B68032B01D1032337E065
S315080218407B68042B01D1042332E07B68052B01D186
S3150802185005232DE07B68062B01D1062328E07B6849
S31508021860072B01D1072323E07B68082B01D1082324
S315080218701EE07B68092B01D80C2319E07B680A2B2A
S3150802188001D8102314E07B680B2B01D814230FE030
S315080218907B680C2B01D818230AE07B680D2B01D82C
S315080218A0202305E07B680E2B01D8302300E0402375
S315080218B018460C37BD465DF8047B704780B483B082
S315080218C000AF0346FB80FB88002B01D1002346E0CC
S315080218D0FB88012B01D1012341E0FB88022B01D1B0
S315080218E002233CE0FB88032B01D1032337E0FB8864
S315080218F0042B01D1042332E0FB88052B01D10523F1
S315080219002DE0FB88062B01D1062328E0FB88072B4E
S3150802191001D1072323E0FB88082B01D108231EE007
S31508021920FB880C2B01D8092319E0FB88102B01D858
S315080219300A2314E0FB88142B01D80B230FE0FB883B
S31508021940182B01D80C230AE0FB88202B01D80D237B
S3150802195005E0FB88302B01D80E2300E00F2318463A
S315080219600C37BD465DF8047B7047000084B0B0B4FE
S3150802197000AF07F10C0484E80F00074B1D4607F178
S315080219800C040FCC0FC50FCC0FC523682B6000BF04
S31508021990BD46B0BC04B070478084002084B0B0B4A1
S315080219A000AF07F10C0484E80F00074B1D4607F148
S315080219B00C040FCC0FC50FCC0FC523682B6000BFD4
S315080219C0BD46B0BC04B070478498002084B0B0B459
S315080219D000AF07F10C0484E80F00074B1D4607F118
S315080219E00C040FCC0FC50FCC0FC523682B6000BFA4
S315080219F0BD46B0BC04B0704788AC002084B0B0B411
S31508021A0000AF07F10C0484E80F00074B1D4607F1E7
S31508021A100C040FCC0FC50FCC0FC523682B6000BF73
S31508021A20BD46B0BC04B070478CC0002084B0B0B4C8
S31508021A3000AF07F10C0484E80F00074B1D4607F1B7
S31508021A400C040FCC0FC50FCC0FC523682B6000BF43
S31508021A50BD46B0BC04B0704790D4002084B0B0B480
S31508021A6000AF07F10C0484E80F00074B1D4607F187
S31508021A700C040FCC0FC50FCC0FC523682B6000BF13
S31508021A80BD46B0BC04B0704794E8002084B0B0B438
S31508021A9000AF07F10C0484E80F00074B1D4607F157
S31508021AA00C040FCC0FC50FCC0FC523682B6000BFE3
S31508021AB0BD46B0BC04B0704798FC002084B0B0B4F0
S31508021AC000AF07F10C0484E80F00074B1D4607F127
S31508021AD00C040FCC0FC50FCC0FC523682B6000BFB3
S31508021AE0BD46B0BC04B070479C10012084B0B0B4A7
S31508021AF000AF07F10C0484E80F00074B1D4607F1F7
S31508021B000C040FCC0FC50FCC0FC523682B6000BF82
S31508021B10BD46B0BC04B07047A024012084B0B0B45E
S31508021B2000AF07F10C0484E80F00074B1D4607F1C6
S31508021B300C040FCC0FC50FCC0FC523682B6000BF52
S31508021B40BD46B0BC04B07047A438012084B0B0B416
S31508021B5000AF07F10C0484E80F00074B1D4607F196
S31508021B600C040FCC0FC50FCC0FC523682B6000BF22
S31508021B70BD46B0BC04B07047A84C012084B0B0B4CE
S31508021B8000AF07F10C0484E80F00074B1D4607F166
S31508021B900C040FCC0FC50FCC0FC523682B6000BFF2
S31508021BA0BD46B0BC04B07047AC60012084B0B0B486
S31508021BB000AF07F10C0484E80F00074B1D4607F136
S31508021BC00C040FCC0FC50FCC0FC523682B6000BFC2
S31508021BD0BD46B0BC04B07047B074012084B0B0B43E
S31508021BE000AF07F10C0484E80F00074B1D4607F106
S31508021BF00C040FCC0FC50FCC0FC523682B6000BF92
S31508021C00BD46B0BC04B07047B488012080B586B022
S31508021C1000AF78600B467B800023FB7500233B618F
S31508021C200023FB600023BB60424BD3F8C4323B61FE
S31508021C30404B03F58053D3F8D432FB607B681B68AC
S31508021C40BB603A69BB689A4227D13A4B93F8E832A5
S31508021C50002B0AD1374BD3F8D0227B881344354A56
S31508021C60C2F8D0320123FB755FE0324BB3F8EC328F
S31508021C701A467B881344B3F57D6F0BDA2D4BB3F8FE
S31508021C80EC227B8813449AB22A4BA3F8EC2201234E
S31508021C90FB754AE00023FB7547E0FA68BB689A427F
S31508021CA02ED1244B03F5805393F8F832002B0AD130
S31508021CB0204BD3F8D0227B8813441E4AC2F8D0326E
S31508021CC00223FB7531E01B4B03F58053B3F8FC3254
S31508021CD01A467B881344FF2B0FDC164B03F58053F9
S31508021CE0B3F8FC227B8813449AB2124B03F580534D
S31508021CF0A3F8FC220223FB7517E00023FB7514E008
S31508021D003B69002B07D1242279680B481BF063FD37
S31508021D100123FB7509E0FB68002B06D124227968AA
S31508021D2006481BF058FD0223FB75FB7D184618373B
S31508021D30BD4680BD80840020448700205497002039
S31508021D4080B586B000AF78600B467B800023FB75B2
S31508021D5000233B610023FB600023BB60424BD3F8A0
S31508021D60C4323B61404B03F58053D3F8D432FB604F
S31508021D707B681B68BB603A69BB689A4227D13A4BB3
S31508021D8093F8E832002B0AD1374BD3F8D0227B8856
S31508021D901344354AC2F8D0320123FB755FE0324B51
S31508021DA0B3F8EC321A467B881344B3F57D6F0BDA27
S31508021DB02D4BB3F8EC227B8813449AB22A4BA3F82C
S31508021DC0EC220123FB754AE00023FB7547E0FA681B
S31508021DD0BB689A422ED1244B03F5805393F8F83206
S31508021DE0002B0AD1204BD3F8D0227B8813441E4AF3
S31508021DF0C2F8D0320223FB7531E01B4B03F5805340
S31508021E00B3F8FC321A467B881344FF2B0FDC164BB9
S31508021E1003F58053B3F8FC227B8813449AB2124B1B
S31508021E2003F58053A3F8FC220223FB7517E000236F
S31508021E30FB7514E03B69002B07D1242279680B480D
S31508021E401BF0C9FC0123FB7509E0FB68002B06D1D0
S31508021E502422796806481BF0BEFC0223FB75FB7D2B
S31508021E6018461837BD4680BD84980020489B002036
S31508021E7058AB002080B586B000AF78600B467B80F1
S31508021E800023FB7500233B610023FB600023BB6034
S31508021E90424BD3F8C4323B61404B03F58053D3F827
S31508021EA0D432FB607B681B68BB603A69BB689A429E
S31508021EB027D13A4B93F8E832002B0AD1374BD3F89D
S31508021EC0D0227B881344354AC2F8D0320123FB75E7
S31508021ED05FE0324BB3F8EC321A467B881344B3F50B
S31508021EE07D6F0BDA2D4BB3F8EC227B8813449AB23A
S31508021EF02A4BA3F8EC220123FB754AE00023FB7563
S31508021F0047E0FA68BB689A422ED1244B03F5805300
S31508021F1093F8F832002B0AD1204BD3F8D0227B88CB
S31508021F2013441E4AC2F8D0320223FB7531E01B4B1A
S31508021F3003F58053B3F8FC321A467B881344FF2B09
S31508021F400FDC164B03F58053B3F8FC227B88134447
S31508021F509AB2124B03F58053A3F8FC220223FB75AF
S31508021F6017E00023FB7514E03B69002B07D12422F6
S31508021F7079680B481BF02FFC0123FB7509E0FB6807
S31508021F80002B06D12422796806481BF024FC02237A
S31508021F90FB75FB7D18461837BD4680BD88AC002008
S31508021FA04CAF00205CBF002080B586B000AF7860D9
S31508021FB00B467B800023FB7500233B610023FB60F5
S31508021FC00023BB60424BD3F8C4323B61404B03F556
S31508021FD08053D3F8D432FB607B681B68BB603A69CE
S31508021FE0BB689A4227D13A4B93F8E832002B0AD1BA
S31508021FF0374BD3F8D0227B881344354AC2F8D032FD
S315080220000123FB755FE0324BB3F8EC321A467B8844
S315080220101344B3F57D6F0BDA2D4BB3F8EC227B88AC
S3150802202013449AB22A4BA3F8EC220123FB754AE021
S315080220300023FB7547E0FA68BB689A422ED1244B07
S3150802204003F5805393F8F832002B0AD1204BD3F8C4
S31508022050D0227B8813441E4AC2F8D0320223FB756B
S3150802206031E01B4B03F58053B3F8FC321A467B88E2
S315080220701344FF2B0FDC164B03F58053B3F8FC22EF
S315080220807B8813449AB2124B03F58053A3F8FC22B9
S315080220900223FB7517E00023FB7514E03B69002B4E
S315080220A007D1242279680B481BF095FB0123FB759F
S315080220B009E0FB68002B06D12422796806481BF042
S315080220C08AFB0223FB75FB7D18461837BD4680BD81
S315080220D08CC0002050C3002060D3002080B586B093
S315080220E000AF78600B467B800023FB7500233B61BB
S315080220F00023FB600023BB60424BD3F8C4323B612A
S31508022100404B03F58053D3F8D432FB607B681B68D7
S31508022110BB603A69BB689A4227D13A4B93F8E832D0
S31508022120002B0AD1374BD3F8D0227B881344354A81
S31508022130C2F8D0320123FB755FE0324BB3F8EC32BA
S315080221401A467B881344B3F57D6F0BDA2D4BB3F829
S31508022150EC227B8813449AB22A4BA3F8EC22012379
S31508022160FB754AE00023FB7547E0FA68BB689A42AA
S315080221702ED1244B03F5805393F8F832002B0AD15B
S31508022180204BD3F8D0227B8813441E4AC2F8D03299
S315080221900223FB7531E01B4B03F58053B3F8FC327F
S315080221A01A467B881344FF2B0FDC164B03F5805324
S315080221B0B3F8FC227B8813449AB2124B03F5805378
S315080221C0A3F8FC220223FB7517E00023FB7514E033
S315080221D03B69002B07D1242279680B481BF0FBFACE
S315080221E00123FB7509E0FB68002B06D124227968D6
S315080221F006481BF0F0FA0223FB75FB7D18461837D2
S31508022200BD4680BD90D4002054D7002064E7002044
S3150802221080B586B000AF78600B467B800023FB75DD
S3150802222000233B610023FB600023BB60424BD3F8CB
S31508022230C4323B61404B03F58053D3F8D432FB607A
S315080222407B681B68BB603A69BB689A4227D13A4BDE
S3150802225093F8E832002B0AD1374BD3F8D0227B8881
S315080222601344354AC2F8D0320123FB755FE0324B7C
S31508022270B3F8EC321A467B881344B3F57D6F0BDA52
S315080222802D4BB3F8EC227B8813449AB22A4BA3F857
S31508022290EC220123FB754AE00023FB7547E0FA6846
S315080222A0BB689A422ED1244B03F5805393F8F83231
S315080222B0002B0AD1204BD3F8D0227B8813441E4A1E
S315080222C0C2F8D0320223FB7531E01B4B03F580536B
S315080222D0B3F8FC321A467B881344FF2B0FDC164BE5
S315080222E003F58053B3F8FC227B8813449AB2124B47
S315080222F003F58053A3F8FC220223FB7517E000239B
S31508022300FB7514E03B69002B07D1242279680B4838
S315080223101BF061FA0123FB7509E0FB68002B06D165
S315080223202422796806481BF056FA0223FB75FB7DC0
S3150802233018461837BD4680BD94E8002058EB0020A1
S3150802234068FB002080B586B000AF78600B467B80BC
S315080223500023FB7500233B610023FB600023BB605F
S31508022360424BD3F8C4323B61404B03F58053D3F852
S31508022370D432FB607B681B68BB603A69BB689A42C9
S3150802238027D13A4B93F8E832002B0AD1374BD3F8C8
S31508022390D0227B881344354AC2F8D0320123FB7512
S315080223A05FE0324BB3F8EC321A467B881344B3F536
S315080223B07D6F0BDA2D4BB3F8EC227B8813449AB265
S315080223C02A4BA3F8EC220123FB754AE00023FB758E
S315080223D047E0FA68BB689A422ED1244B03F580532C
S315080223E093F8F832002B0AD1204BD3F8D0227B88F7
S315080223F013441E4AC2F8D0320223FB7531E01B4B46
S3150802240003F58053B3F8FC321A467B881344FF2B34
S315080224100FDC164B03F58053B3F8FC227B88134472
S315080224209AB2124B03F58053A3F8FC220223FB75DA
S3150802243017E00023FB7514E03B69002B07D1242221
S3150802244079680B481BF0C7F90123FB7509E0FB689D
S31508022450002B06D12422796806481BF0BCF9022310
S31508022460FB75FB7D18461837BD4680BD98FC0020D3
S315080224705CFF00206C0F012080B586B000AF786043
S315080224800B467B800023FB7500233B610023FB6020
S315080224900023BB60424BD3F8C4323B61404B03F581
S315080224A08053D3F8D432FB607B681B68BB603A69F9
S315080224B0BB689A4227D13A4B93F8E832002B0AD1E5
S315080224C0374BD3F8D0227B881344354AC2F8D03228
S315080224D00123FB755FE0324BB3F8EC321A467B8870
S315080224E01344B3F57D6F0BDA2D4BB3F8EC227B88D8
S315080224F013449AB22A4BA3F8EC220123FB754AE04D
S315080225000023FB7547E0FA68BB689A422ED1244B32
S3150802251003F5805393F8F832002B0AD1204BD3F8EF
S31508022520D0227B8813441E4AC2F8D0320223FB7596
S3150802253031E01B4B03F58053B3F8FC321A467B880D
S315080225401344FF2B0FDC164B03F58053B3F8FC221A
S315080225507B8813449AB2124B03F58053A3F8FC22E4
S315080225600223FB7517E00023FB7514E03B69002B79
S3150802257007D1242279680B481BF02DF90123FB7534
S3150802258009E0FB68002B06D12422796806481BF06D
S3150802259022F90223FB75FB7D18461837BD4680BD16
S315080225A09C100120601301207023012080B586B09B
S315080225B000AF78600B467B800023FB7500233B61E6
S315080225C00023FB600023BB60424BD3F8C4323B6155
S315080225D0404B03F58053D3F8D432FB607B681B6803
S315080225E0BB603A69BB689A4227D13A4B93F8E832FC
S315080225F0002B0AD1374BD3F8D0227B881344354AAD
S31508022600C2F8D0320123FB755FE0324BB3F8EC32E5
S315080226101A467B881344B3F57D6F0BDA2D4BB3F854
S31508022620EC227B8813449AB22A4BA3F8EC220123A4
S31508022630FB754AE00023FB7547E0FA68BB689A42D5
S315080226402ED1244B03F5805393F8F832002B0AD186
S31508022650204BD3F8D0227B8813441E4AC2F8D032C4
S315080226600223FB7531E01B4B03F58053B3F8FC32AA
S315080226701A467B881344FF2B0FDC164B03F580534F
S31508022680B3F8FC227B8813449AB2124B03F58053A3
S31508022690A3F8FC220223FB7517E00023FB7514E05E
S315080226A03B69002B07D1242279680B481BF093F863
S315080226B00123FB7509E0FB68002B06D12422796801
S315080226C006481BF088F80223FB75FB7D1846183767
S315080226D0BD4680BDA024012064270120743701204D
S315080226E080B586B000AF78600B467B800023FB7509
S315080226F000233B610023FB600023BB60424BD3F8F7
S31508022700C4323B61404B03F58053D3F8D432FB60A5
S315080227107B681B68BB603A69BB689A4227D13A4B09
S3150802272093F8E832002B0AD1374BD3F8D0227B88AC
S315080227301344354AC2F8D0320123FB755FE0324BA7
S31508022740B3F8EC321A467B881344B3F57D6F0BDA7D
S315080227502D4BB3F8EC227B8813449AB22A4BA3F882
S31508022760EC220123FB754AE00023FB7547E0FA6871
S31508022770BB689A422ED1244B03F5805393F8F8325C
S31508022780002B0AD1204BD3F8D0227B8813441E4A49
S31508022790C2F8D0320223FB7531E01B4B03F5805396
S315080227A0B3F8FC321A467B881344FF2B0FDC164B10
S315080227B003F58053B3F8FC227B8813449AB2124B72
S315080227C003F58053A3F8FC220223FB7517E00023C6
S315080227D0FB7514E03B69002B07D1242279680B4864
S315080227E01AF0F9FF0123FB7509E0FB68002B06D1F5
S315080227F02422796806481AF0EEFF0223FB75FB7D50
S3150802280018461837BD4680BDA4380120683B01200A
S31508022810784B012080B586B000AF78600B467B8086
S315080228200023FB7500233B610023FB600023BB608A
S31508022830424BD3F8C4323B61404B03F58053D3F87D
S31508022840D432FB607B681B68BB603A69BB689A42F4
S3150802285027D13A4B93F8E832002B0AD1374BD3F8F3
S31508022860D0227B881344354AC2F8D0320123FB753D
S315080228705FE0324BB3F8EC321A467B881344B3F561
S315080228807D6F0BDA2D4BB3F8EC227B8813449AB290
S315080228902A4BA3F8EC220123FB754AE00023FB75B9
S315080228A047E0FA68BB689A422ED1244B03F5805357
S315080228B093F8F832002B0AD1204BD3F8D0227B8822
S315080228C013441E4AC2F8D0320223FB7531E01B4B71
S315080228D003F58053B3F8FC321A467B881344FF2B60
S315080228E00FDC164B03F58053B3F8FC227B8813449E
S315080228F09AB2124B03F58053A3F8FC220223FB7506
S3150802290017E00023FB7514E03B69002B07D124224C
S3150802291079680B481AF05FFF0123FB7509E0FB682B
S31508022920002B06D12422796806481AF054FF02239E
S31508022930FB75FB7D18461837BD4680BDA84C01209D
S315080229406C4F01207C5F012080B586B000AF7860AD
S315080229500B467B800023FB7500233B610023FB604B
S315080229600023BB60424BD3F8C4323B61404B03F5AC
S315080229708053D3F8D432FB607B681B68BB603A6924
S31508022980BB689A4227D13A4B93F8E832002B0AD110
S31508022990374BD3F8D0227B881344354AC2F8D03253
S315080229A00123FB755FE0324BB3F8EC321A467B889B
S315080229B01344B3F57D6F0BDA2D4BB3F8EC227B8803
S315080229C013449AB22A4BA3F8EC220123FB754AE078
S315080229D00023FB7547E0FA68BB689A422ED1244B5E
S315080229E003F5805393F8F832002B0AD1204BD3F81B
S315080229F0D0227B8813441E4AC2F8D0320223FB75C2
S31508022A0031E01B4B03F58053B3F8FC321A467B8838
S31508022A101344FF2B0FDC164B03F58053B3F8FC2245
S31508022A207B8813449AB2124B03F58053A3F8FC220F
S31508022A300223FB7517E00023FB7514E03B69002BA4
S31508022A4007D1242279680B481AF0C5FE0123FB75C3
S31508022A5009E0FB68002B06D12422796806481AF099
S31508022A60BAFE0223FB75FB7D18461837BD4680BDA4
S31508022A70AC600120706301208073012080B586B0A6
S31508022A8000AF78600B467B800023FB7500233B6111
S31508022A900023FB600023BB60424BD3F8C4323B6180
S31508022AA0404B03F58053D3F8D432FB607B681B682E
S31508022AB0BB603A69BB689A4227D13A4B93F8E83227
S31508022AC0002B0AD1374BD3F8D0227B881344354AD8
S31508022AD0C2F8D0320123FB755FE0324BB3F8EC3211
S31508022AE01A467B881344B3F57D6F0BDA2D4BB3F880
S31508022AF0EC227B8813449AB22A4BA3F8EC220123D0
S31508022B00FB754AE00023FB7547E0FA68BB689A4200
S31508022B102ED1244B03F5805393F8F832002B0AD1B1
S31508022B20204BD3F8D0227B8813441E4AC2F8D032EF
S31508022B300223FB7531E01B4B03F58053B3F8FC32D5
S31508022B401A467B881344FF2B0FDC164B03F580537A
S31508022B50B3F8FC227B8813449AB2124B03F58053CE
S31508022B60A3F8FC220223FB7517E00023FB7514E089
S31508022B703B69002B07D1242279680B481AF02BFEF1
S31508022B800123FB7509E0FB68002B06D1242279682C
S31508022B9006481AF020FE0223FB75FB7D18461837F5
S31508022BA0BD4680BDB0740120747701208487012058
S31508022BB080B586B000AF78600B467B800023FB7534
S31508022BC000233B610023FB600023BB60424BD3F822
S31508022BD0C4323B61404B03F58053D3F8D432FB60D1
S31508022BE07B681B68BB603A69BB689A4227D13A4B35
S31508022BF093F8E832002B0AD1374BD3F8D0227B88D8
S31508022C001344354AC2F8D0320123FB755FE0324BD2
S31508022C10B3F8EC321A467B881344B3F57D6F0BDAA8
S31508022C202D4BB3F8EC227B8813449AB22A4BA3F8AD
S31508022C30EC220123FB754AE00023FB7547E0FA689C
S31508022C40BB689A422ED1244B03F5805393F8F83287
S31508022C50002B0AD1204BD3F8D0227B8813441E4A74
S31508022C60C2F8D0320223FB7531E01B4B03F58053C1
S31508022C70B3F8FC321A467B881344FF2B0FDC164B3B
S31508022C8003F58053B3F8FC227B8813449AB2124B9D
S31508022C9003F58053A3F8FC220223FB7517E00023F1
S31508022CA0FB7514E03B69002B07D1242279680B488F
S31508022CB01AF091FD0123FB7509E0FB68002B06D18A
S31508022CC02422796806481AF086FD0223FB75FB7DE5
S31508022CD018461837BD4680BDB4880120788B012076
S31508022CE0889B012080B584B000AF03463960FB712A
S31508022CF01346BB800023FB73FB79012B13D10023F8
S31508022D00FB730AE0FB7B3A6813440122194613480F
S31508022D1008F064FFFB7B0133FB73FB7B9BB2BA882B
S31508022D209A42EFD815E0FB79022B12D10023FB73E6
S31508022D300AE0FB7B3A68134401221946084808F060
S31508022D404DFFFB7B0133FB73FB7B9BB2BA889A422E
S31508022D50EFD800BF1037BD4680BD00BF34870020BC
S31508022D604497002080B584B000AF03463960FB71F2
S31508022D701346BB800023FB73FB79012B13D1002377
S31508022D80FB730AE0FB7B3A6813440122194613488F
S31508022D9008F024FFFB7B0133FB73FB7B9BB2BA88EB
S31508022DA09A42EFD815E0FB79022B12D10023FB7366
S31508022DB00AE0FB7B3A68134401221946084808F0E0
S31508022DC00DFFFB7B0133FB73FB7B9BB2BA889A42EE
S31508022DD0EFD800BF1037BD4680BD00BF389B002024
S31508022DE048AB002080B584B000AF03463960FB715A
S31508022DF01346BB800023FB73FB79012B13D10023F7
S31508022E00FB730AE0FB7B3A6813440122194613480E
S31508022E1008F0E4FEFB7B0133FB73FB7B9BB2BA88AB
S31508022E209A42EFD815E0FB79022B12D10023FB73E5
S31508022E300AE0FB7B3A68134401221946084808F05F
S31508022E40CDFEFB7B0133FB73FB7B9BB2BA889A42AE
S31508022E50EFD800BF1037BD4680BD00BF3CAF00208B
S31508022E604CBF002080B584B000AF03463960FB71C1
S31508022E701346BB800023FB73FB79012B13D1002376
S31508022E80FB730AE0FB7B3A6813440122194613488E
S31508022E9008F0A4FEFB7B0133FB73FB7B9BB2BA886B
S31508022EA09A42EFD815E0FB79022B12D10023FB7365
S31508022EB00AE0FB7B3A68134401221946084808F0DF
S31508022EC08DFEFB7B0133FB73FB7B9BB2BA889A426E
S31508022ED0EFD800BF1037BD4680BD00BF40C30020F3
S31508022EE050D3002080B584B000AF03463960FB7129
S31508022EF01346BB800023FB73FB79012B13D10023F6
S31508022F00FB730AE0FB7B3A6813440122194613480D
S31508022F1008F064FEFB7B0133FB73FB7B9BB2BA882A
S31508022F209A42EFD815E0FB79022B12D10023FB73E4
S31508022F300AE0FB7B3A68134401221946084808F05E
S31508022F404DFEFB7B0133FB73FB7B9BB2BA889A422D
S31508022F50EFD800BF1037BD4680BD00BF44D700205A
S31508022F6054E7002080B584B000AF03463960FB7190
S31508022F701346BB800023FB73FB79012B13D1002375
S31508022F80FB730AE0FB7B3A6813440122194613488D
S31508022F9008F024FEFB7B0133FB73FB7B9BB2BA88EA
S31508022FA09A42EFD815E0FB79022B12D10023FB7364
S31508022FB00AE0FB7B3A68134401221946084808F0DE
S31508022FC00DFEFB7B0133FB73FB7B9BB2BA889A42ED
S31508022FD0EFD800BF1037BD4680BD00BF48EB0020C2
S31508022FE058FB002080B584B000AF03463960FB71F8
S31508022FF01346BB800023FB73FB79012B13D10023F5
S31508023000FB730AE0FB7B3A6813440122194613480C
S3150802301008F0E4FDFB7B0133FB73FB7B9BB2BA88AA
S315080230209A42EFD815E0FB79022B12D10023FB73E3
S315080230300AE0FB7B3A68134401221946084808F05D
S31508023040CDFDFB7B0133FB73FB7B9BB2BA889A42AD
S31508023050EFD800BF1037BD4680BD00BF4CFF002029
S315080230605C0F012080B584B000AF03463960FB715E
S315080230701346BB800023FB73FB79012B13D1002374
S31508023080FB730AE0FB7B3A6813440122194613488C
S3150802309008F0A4FDFB7B0133FB73FB7B9BB2BA886A
S315080230A09A42EFD815E0FB79022B12D10023FB7363
S315080230B00AE0FB7B3A68134401221946084808F0DD
S315080230C08DFDFB7B0133FB73FB7B9BB2BA889A426D
S315080230D0EFD800BF1037BD4680BD00BF5013012090
S315080230E06023012080B584B000AF03463960FB71C6
S315080230F01346BB800023FB73FB79012B13D10023F4
S31508023100FB730AE0FB7B3A6813440122194613480B
S3150802311008F064FDFB7B0133FB73FB7B9BB2BA8829
S315080231209A42EFD815E0FB79022B12D10023FB73E2
S315080231300AE0FB7B3A68134401221946084808F05C
S315080231404DFDFB7B0133FB73FB7B9BB2BA889A422C
S31508023150EFD800BF1037BD4680BD00BF54270120F7
S315080231606437012080B584B000AF03463960FB712D
S315080231701346BB800023FB73FB79012B13D1002373
S31508023180FB730AE0FB7B3A6813440122194613488B
S3150802319008F024FDFB7B0133FB73FB7B9BB2BA88E9
S315080231A09A42EFD815E0FB79022B12D10023FB7362
S315080231B00AE0FB7B3A68134401221946084808F0DC
S315080231C00DFDFB7B0133FB73FB7B9BB2BA889A42EC
S315080231D0EFD800BF1037BD4680BD00BF583B01205F
S315080231E0684B012080B584B000AF03463960FB7195
S315080231F01346BB800023FB73FB79012B13D10023F3
S31508023200FB730AE0FB7B3A6813440122194613480A
S3150802321008F0E4FCFB7B0133FB73FB7B9BB2BA88A9
S315080232209A42EFD815E0FB79022B12D10023FB73E1
S315080232300AE0FB7B3A68134401221946084808F05B
S31508023240CDFCFB7B0133FB73FB7B9BB2BA889A42AC
S31508023250EFD800BF1037BD4680BD00BF5C4F0120C6
S315080232606C5F012080B584B000AF03463960FB71FC
S315080232701346BB800023FB73FB79012B13D1002372
S31508023280FB730AE0FB7B3A6813440122194613488A
S3150802329008F0A4FCFB7B0133FB73FB7B9BB2BA8869
S315080232A09A42EFD815E0FB79022B12D10023FB7361
S315080232B00AE0FB7B3A68134401221946084808F0DB
S315080232C08DFCFB7B0133FB73FB7B9BB2BA889A426C
S315080232D0EFD800BF1037BD4680BD00BF606301202E
S315080232E07073012080B584B000AF03463960FB7164
S315080232F01346BB800023FB73FB79012B13D10023F2
S31508023300FB730AE0FB7B3A68134401221946134809
S3150802331008F064FCFB7B0133FB73FB7B9BB2BA8828
S315080233209A42EFD815E0FB79022B12D10023FB73E0
S315080233300AE0FB7B3A68134401221946084808F05A
S315080233404DFCFB7B0133FB73FB7B9BB2BA889A422B
S31508023350EFD800BF1037BD4680BD00BF6477012095
S315080233607487012080B584B000AF03463960FB71CB
S315080233701346BB800023FB73FB79012B13D1002371
S31508023380FB730AE0FB7B3A68134401221946134889
S3150802339008F024FCFB7B0133FB73FB7B9BB2BA88E8
S315080233A09A42EFD815E0FB79022B12D10023FB7360
S315080233B00AE0FB7B3A68134401221946084808F0DA
S315080233C00DFCFB7B0133FB73FB7B9BB2BA889A42EB
S315080233D0EFD800BF1037BD4680BD00BF688B0120FD
S315080233E0789B012080B582B000AF0346FB71FB1DB6
S315080233F001221946034808F0F1FB00BF0837BD460B
S3150802340080BD00BFA484002080B582B000AF034609
S31508023410FB71FB1D01221946034808F0DFFB00BFBA
S315080234200837BD4680BD00BFA898002080B582B087
S3150802343000AF0346FB71FB1D01221946034808F03B
S31508023440CDFB00BF0837BD4680BD00BFACAC00202F
S3150802345080B582B000AF0346FB71FB1D01221946F7
S31508023460034808F0BBFB00BF0837BD4680BD00BF56
S31508023470B0C0002080B582B000AF0346FB71FB1DC9
S3150802348001221946034808F0A9FB00BF0837BD46C2
S3150802349080BD00BFB4D4002080B582B000AF034619
S315080234A0FB71FB1D01221946034808F097FB00BF72
S315080234B00837BD4680BD00BFB8E8002080B582B097
S315080234C000AF0346FB71FB1D01221946034808F0AB
S315080234D085FB00BF0837BD4680BD00BFBCFC002087
S315080234E080B582B000AF0346FB71FB1D0122194667
S315080234F0034808F073FB00BF0837BD4680BD00BF0E
S31508023500C010012080B582B000AF0346FB71FB1DD7
S3150802351001221946034808F061FB00BF0837BD4679
S3150802352080BD00BFC424012080B582B000AF034627
S31508023530FB71FB1D01221946034808F04FFB00BF29
S315080235400837BD4680BD00BFC838012080B582B0A5
S3150802355000AF0346FB71FB1D01221946034808F01A
S315080235603DFB00BF0837BD4680BD00BFCC4C0120DD
S3150802357080B582B000AF0346FB71FB1D01221946D6
S31508023580034808F02BFB00BF0837BD4680BD00BFC5
S31508023590D060012080B582B000AF0346FB71FB1DE7
S315080235A001221946034808F019FB00BF0837BD4631
S315080235B080BD00BFD474012080B582B000AF034637
S315080235C0FB71FB1D01221946034808F007FB00BFE1
S315080235D00837BD4680BD00BFD888012080B59EB099
S315080235E000AFF860B9601346FB8007F11403642242
S315080235F0002118461AF052F8FB88002B26D04FF005
S315080236008043BB61FB687B610023FB61FB8818462C
S31508023610FEF754F903463B6200237B624FF480139C
S31508023620BB624FF40013FB6200233B6300237B63F8
S31508023630FA8807F114032433B96818461AF0CBF846
S3150802364007F114036421184602F0DEFB00BF78373F
S31508023650BD4680BDF0B5C3B008AFF861B9617A61FD
S31508023660002387F8E730F8690DF069FCC7F8E0002F
S31508023670A84B00221A6079E0A64B1B685A1CA5497A
S315080236800A60B3F5FA7F71D997F8E730013387F8FC
S31508023690E73007F16C031946F8690DF083FDFB6EF6
S315080236A03B613A6FFA60786FB860BB6FFA6FD7F80A
S315080236B08010D7F88400D7F888407C60D7F88C50F9
S315080236C0D7F89060D7F894400794069605957C68D3
S315080236D004940390029101920093BB68FA683969CF
S315080236E08D480AF065FFD7F88030002B07D0FB69B2
S315080236F01B689A69FB691B6822F001029A61F869DC
S315080237000DF01DFCC7F8E000D7F8E010F8690DF0D7
S3150802371022FC804B00221A6080480AF049FF804B3F
S315080237201B78022B2BD07E4B01221A7007F1DC0381
S315080237300221184618F0B9FD07F1980207F1DC03D1
S315080237401146184618F041FE07F19803184618F074
S31508023750BBFD044607F19803184618F0C1FD034657
S315080237601A4621464A20FFF739FF08E00721F86979
S315080237700DF068FD0346002B7FF47EAF00E000BF24
S315080237807A69B969F8690DF096FB0346002B2DD0C4
S3150802379097F8E730013387F8E73062480AF008FFFE
S315080237A05F4B1B78012B21D05D4B01221A7007F162
S315080237B0DC030121184618F078FD07F1980207F193
S315080237C0DC031146184618F000FE07F1980318465E
S315080237D018F07AFD044607F19803184618F080FD9A
S315080237E003461A4621464A20FFF7F8FE97F8E730BD
S315080237F0002B25D14A4B1B78002B21D0484B00229F
S315080238001A7007F1DC030021184618F04EFD07F17D
S31508023810980207F1DC031146184618F0D6FD07F19F
S315080238209803184618F050FD044607F198031846FF
S3150802383018F056FD03461A4621464A20FFF7CEFEE1
S31508023840F86903F055FC03461A46374B9A60F8693D
S3150802385003F018FC0346344A1360F86903F02AFC9D
S315080238600346314A5360304B9B68002B0CD02E4BD3
S315080238701B682D4A526819462C480AF099FE2A4BAB
S315080238809B68184603F07CFC0C222749284819F045
S31508023890F5FE0346002B33D0234B1B68DAB207F139
S315080238A068031146184618F0AFFC1F4B5B68DAB27C
S315080238B007F168031146184618F0C1FC1A4B9B68B3
S315080238C0DAB207F168031146184618F0D3FC07F175
S315080238D0240207F168031146184618F047FD07F156
S315080238E02403184618F0F0FC044607F12403184688
S315080238F018F0F6FC03461A4621464A20FFF76EFEE2
S315080239000B4B094A07CA83E8070000BFEC37BD46D6
S31508023910F0BD00BFE0A001208C0C0408D00C0408FE
S31508023920E4A00120F40C0408C8A00120680C0408CD
S31508023930D4A0012080B592B000AF3B4640220021B8
S31508023940184619F0ABFE0023A7F8423000237B6421
S315080239509C4808F027F9034683F00103DBB2002BE3
S3150802396000F0C480984B93F8E832002B50D1964B5E
S31508023970D3F8D0329AB2944BA3F8EC22924B0F2288
S31508023980C3F8D02210233B703B785AB28E4BB3F859
S31508023990EC321B0A9BB25BB203F00F035BB2134312
S315080239A05BB2DBB23B70884BB3F8EC32DBB27B70AE
S315080239B03B4602333E221946824808F04AF9034634
S315080239C0002B00F0FC80FDF79FFB3B461A467F4919
S315080239D0FFF740FE7C4BB3F8EC323E3B9AB27A4B89
S315080239E0A3F8EC22784BB3F8EA3201339AB2764B53
S315080239F0A3F8EA22744B012283F8E822724BFF22CB
S31508023A0083F8EE22704B4FF4FA62C3F8F022D6E03E
S31508023A106D4B93F8EE32002B05D06B4B93F8EE32D2
S31508023A20012B40F0CC80684BB3F8EC323E2B02D91E
S31508023A3040237B6404E0644BB3F8EC3201337B64C5
S31508023A4020233B703B785AB25F4BB3F8EA325BB23B
S31508023A5003F00F035BB213435BB2DBB23B707B6CC2
S31508023A605A1E3B4601331946564808F0F2F80346F1
S31508023A70002B00F0A4807B6C9BB21846FDF71EFF54
S31508023A800346514AC2F8D032FDF73EFB3B461A4678
S31508023A904E49FFF7DFFD4C4BB3F8EC227B6C9BB229
S31508023AA0D31A9BB201339AB2474BA3F8EC22464B80
S31508023AB0B3F8EA3201339AB2434BA3F8EA22424BED
S31508023AC0B3F8EC32002B7AD1242200213F4819F0B0
S31508023AD0E5FD3D4B002283F8E8223B4B0022A3F882
S31508023AE0EA22394BFF2283F8EE2268E0384808F0CA
S31508023AF059F8034683F00103DBB2002B5FD03B463D
S31508023B0001221946324808F0A4F80346002B53D07E
S31508023B103B781B09DBB2032B14D13B460133022245
S31508023B2019462B4808F095F80346002B47D0264B32
S31508023B300322DA60FDF7E8FA3B461A462249FFF7FE
S31508023B4089FD3CE03B781B09DBB2002B37D13B46AB
S31508023B500133012219461E4808F07BF80346002B5A
S31508023B602CD03B781B029BB203F47063A7F8423051
S31508023B707B781A46B7F842301343A7F84230B7F8AB
S31508023B8042203B4602331946114808F062F80346BA
S31508023B90002B14D0B7F8423002339BB21846FDF711
S31508023BA08DFE0346084AD360FDF7AEFA3B461A462F
S31508023BB00549FFF74FFD02E000BF00E000BF4837A6
S31508023BC0BD4680BD348700208084002044870020BB
S31508023BD0A484002080B592B000AF3B464022002163
S31508023BE0184619F05BFD0023A7F8423000237B64D0
S31508023BF09C4807F0D7FF034683F00103DBB2002B8C
S31508023C0000F0C480984B93F8E832002B50D1964BBB
S31508023C10D3F8D0329AB2944BA3F8EC22924B0F22E5
S31508023C20C3F8D02210233B703B785AB28E4BB3F8B6
S31508023C30EC321B0A9BB25BB203F00F035BB213436F
S31508023C405BB2DBB23B70884BB3F8EC32DBB27B700B
S31508023C503B4602333E221946824807F0FAFF0346DC
S31508023C60002B00F0FC80FDF74FFA3B461A467F49C7
S31508023C70FFF7F0FC7C4BB3F8EC323E3B9AB27A4B38
S31508023C80A3F8EC22784BB3F8EA3201339AB2764BB0
S31508023C90A3F8EA22744B012283F8E822724BFF2228
S31508023CA083F8EE22704B4FF4FA62C3F8F022D6E09C
S31508023CB06D4B93F8EE32002B05D06B4B93F8EE3230
S31508023CC0012B40F0CC80684BB3F8EC323E2B02D97C
S31508023CD040237B6404E0644BB3F8EC3201337B6423
S31508023CE020233B703B785AB25F4BB3F8EA325BB299
S31508023CF003F00F035BB213435BB2DBB23B707B6C20
S31508023D005A1E3B4601331946564807F0A2FF034698
S31508023D10002B00F0A4807B6C9BB21846FDF7CEFD03
S31508023D200346514AC2F8D032FDF7EEF93B461A4627
S31508023D304E49FFF78FFC4C4BB3F8EC227B6C9BB2D7
S31508023D40D31A9BB201339AB2474BA3F8EC22464BDD
S31508023D50B3F8EA3201339AB2434BA3F8EA22424B4A
S31508023D60B3F8EC32002B7AD1242200213F4819F00D
S31508023D7095FC3D4B002283F8E8223B4B0022A3F830
S31508023D80EA22394BFF2283F8EE2268E0384807F028
S31508023D9009FF034683F00103DBB2002B5FD03B46E3
S31508023DA001221946324807F054FF0346002B53D026
S31508023DB03B781B09DBB2032B14D13B4601330222A3
S31508023DC019462B4807F045FF0346002B47D0264BDA
S31508023DD00322DA60FDF798F93B461A462249FFF7AD
S31508023DE039FC3CE03B781B09DBB2002B37D13B465A
S31508023DF00133012219461E4807F02BFF0346002B02
S31508023E002CD03B781B029BB203F47063A7F84230AE
S31508023E107B781A46B7F842301343A7F84230B7F808
S31508023E2042203B4602331946114807F012FF034661
S31508023E30002B14D0B7F8423002339BB21846FDF76E
S31508023E403DFD0346084AD360FDF75EF93B461A462E
S31508023E500549FFF7FFFB02E000BF00E000BF483755
S31508023E60BD4680BD389B002084980020489B0020D0
S31508023E70A898002080B592B000AF3B4640220021A8
S31508023E80184619F00BFC0023A7F8423000237B647E
S31508023E909C4807F087FE034683F00103DBB2002B3A
S31508023EA000F0C480984B93F8E832002B50D1964B19
S31508023EB0D3F8D0329AB2944BA3F8EC22924B0F2243
S31508023EC0C3F8D02210233B703B785AB28E4BB3F814
S31508023ED0EC321B0A9BB25BB203F00F035BB21343CD
S31508023EE05BB2DBB23B70884BB3F8EC32DBB27B7069
S31508023EF03B4602333E221946824807F0AAFE03468B
S31508023F00002B00F0FC80FDF7FFF83B461A467F4976
S31508023F10FFF7A0FB7C4BB3F8EC323E3B9AB27A4BE6
S31508023F20A3F8EC22784BB3F8EA3201339AB2764B0D
S31508023F30A3F8EA22744B012283F8E822724BFF2285
S31508023F4083F8EE22704B4FF4FA62C3F8F022D6E0F9
S31508023F506D4B93F8EE32002B05D06B4B93F8EE328D
S31508023F60012B40F0CC80684BB3F8EC323E2B02D9D9
S31508023F7040237B6404E0644BB3F8EC3201337B6480
S31508023F8020233B703B785AB25F4BB3F8EA325BB2F6
S31508023F9003F00F035BB213435BB2DBB23B707B6C7D
S31508023FA05A1E3B4601331946564807F052FE034647
S31508023FB0002B00F0A4807B6C9BB21846FDF77EFCB2
S31508023FC00346514AC2F8D032FDF79EF83B461A46D6
S31508023FD04E49FFF73FFB4C4BB3F8EC227B6C9BB286
S31508023FE0D31A9BB201339AB2474BA3F8EC22464B3B
S31508023FF0B3F8EA3201339AB2434BA3F8EA22424BA8
S31508024000B3F8EC32002B7AD1242200213F4819F06A
S3150802401045FB3D4B002283F8E8223B4B0022A3F8DE
S31508024020EA22394BFF2283F8EE2268E0384807F085
S31508024030B9FD034683F00103DBB2002B5FD03B4692
S3150802404001221946324807F004FE0346002B53D0D4
S315080240503B781B09DBB2032B14D13B460133022200
S3150802406019462B4807F0F5FD0346002B47D0264B89
S315080240700322DA60FDF748F83B461A462249FFF75B
S31508024080E9FA3CE03B781B09DBB2002B37D13B4609
S315080240900133012219461E4807F0DBFD0346002BB1
S315080240A02CD03B781B029BB203F47063A7F842300C
S315080240B07B781A46B7F842301343A7F84230B7F866
S315080240C042203B4602331946114807F0C2FD034611
S315080240D0002B14D0B7F8423002339BB21846FDF7CC
S315080240E0EDFB0346084AD360FDF70EF83B461A462F
S315080240F00549FFF7AFFA02E000BF00E000BF483704
S31508024100BD4680BD3CAF002088AC00204CAF0020E5
S31508024110ACAC002080B592B000AF3B4640220021ED
S31508024120184619F0BBFA0023A7F8423000237B642D
S315080241309C4807F037FD034683F00103DBB2002BE8
S3150802414000F0C480984B93F8E832002B50D1964B76
S31508024150D3F8D0329AB2944BA3F8EC22924B0F22A0
S31508024160C3F8D02210233B703B785AB28E4BB3F871
S31508024170EC321B0A9BB25BB203F00F035BB213432A
S315080241805BB2DBB23B70884BB3F8EC32DBB27B70C6
S315080241903B4602333E221946824807F05AFD034639
S315080241A0002B00F0FC80FCF7AFFF3B461A467F491E
S315080241B0FFF750FA7C4BB3F8EC323E3B9AB27A4B95
S315080241C0A3F8EC22784BB3F8EA3201339AB2764B6B
S315080241D0A3F8EA22744B012283F8E822724BFF22E3
S315080241E083F8EE22704B4FF4FA62C3F8F022D6E057
S315080241F06D4B93F8EE32002B05D06B4B93F8EE32EB
S31508024200012B40F0CC80684BB3F8EC323E2B02D936
S3150802421040237B6404E0644BB3F8EC3201337B64DD
S3150802422020233B703B785AB25F4BB3F8EA325BB253
S3150802423003F00F035BB213435BB2DBB23B707B6CDA
S315080242405A1E3B4601331946564807F002FD0346F5
S31508024250002B00F0A4807B6C9BB21846FDF72EFB60
S315080242600346514AC2F8D032FCF74EFF3B461A467D
S315080242704E49FFF7EFF94C4BB3F8EC227B6C9BB235
S31508024280D31A9BB201339AB2474BA3F8EC22464B98
S31508024290B3F8EA3201339AB2434BA3F8EA22424B05
S315080242A0B3F8EC32002B7AD1242200213F4819F0C8
S315080242B0F5F93D4B002283F8E8223B4B0022A3F88E
S315080242C0EA22394BFF2283F8EE2268E0384807F0E3
S315080242D069FC034683F00103DBB2002B5FD03B4641
S315080242E001221946324807F0B4FC0346002B53D084
S315080242F03B781B09DBB2032B14D13B46013302225E
S3150802430019462B4807F0A5FC0346002B47D0264B37
S315080243100322DA60FCF7F8FE3B461A462249FFF703
S3150802432099F93CE03B781B09DBB2002B37D13B46B7
S315080243300133012219461E4807F08BFC0346002B5F
S315080243402CD03B781B029BB203F47063A7F8423069
S315080243507B781A46B7F842301343A7F84230B7F8C3
S3150802436042203B4602331946114807F072FC0346BF
S31508024370002B14D0B7F8423002339BB21846FDF729
S315080243809DFA0346084AD360FCF7BEFE3B461A4628
S315080243900549FFF75FF902E000BF00E000BF4837B2
S315080243A0BD4680BD40C300208CC0002050C30020FB
S315080243B0B0C0002080B592B000AF3B464022002133
S315080243C0184619F06BF90023A7F8423000237B64DC
S315080243D09C4807F0E7FB034683F00103DBB2002B98
S315080243E000F0C480984B93F8E832002B50D1964BD4
S315080243F0D3F8D0329AB2944BA3F8EC22924B0F22FE
S31508024400C3F8D02210233B703B785AB28E4BB3F8CE
S31508024410EC321B0A9BB25BB203F00F035BB2134387
S315080244205BB2DBB23B70884BB3F8EC32DBB27B7023
S315080244303B4602333E221946824807F00AFC0346E7
S31508024440002B00F0FC80FCF75FFE3B461A467F49CC
S31508024450FFF700F97C4BB3F8EC323E3B9AB27A4B43
S31508024460A3F8EC22784BB3F8EA3201339AB2764BC8
S31508024470A3F8EA22744B012283F8E822724BFF2240
S3150802448083F8EE22704B4FF4FA62C3F8F022D6E0B4
S315080244906D4B93F8EE32002B05D06B4B93F8EE3248
S315080244A0012B40F0CC80684BB3F8EC323E2B02D994
S315080244B040237B6404E0644BB3F8EC3201337B643B
S315080244C020233B703B785AB25F4BB3F8EA325BB2B1
S315080244D003F00F035BB213435BB2DBB23B707B6C38
S315080244E05A1E3B4601331946564807F0B2FB0346A5
S315080244F0002B00F0A4807B6C9BB21846FDF7DEF910
S315080245000346514AC2F8D032FCF7FEFD3B461A462C
S315080245104E49FFF79FF84C4BB3F8EC227B6C9BB2E3
S31508024520D31A9BB201339AB2474BA3F8EC22464BF5
S31508024530B3F8EA3201339AB2434BA3F8EA22424B62
S31508024540B3F8EC32002B7AD1242200213F4819F025
S31508024550A5F83D4B002283F8E8223B4B0022A3F83C
S31508024560EA22394BFF2283F8EE2268E0384807F040
S3150802457019FB034683F00103DBB2002B5FD03B46EF
S3150802458001221946324807F064FB0346002B53D032
S315080245903B781B09DBB2032B14D13B4601330222BB
S315080245A019462B4807F055FB0346002B47D0264BE6
S315080245B00322DA60FCF7A8FD3B461A462249FFF7B2
S315080245C049F83CE03B781B09DBB2002B37D13B4666
S315080245D00133012219461E4807F03BFB0346002B0E
S315080245E02CD03B781B029BB203F47063A7F84230C7
S315080245F07B781A46B7F842301343A7F84230B7F821
S3150802460042203B4602331946114807F022FB03466D
S31508024610002B14D0B7F8423002339BB21846FDF786
S315080246204DF90346084AD360FCF76EFD3B461A4627
S315080246300549FFF70FF802E000BF00E000BF483760
S31508024640BD4680BD44D7002090D4002054D7002010
S31508024650B4D4002080B592B000AF3B464022002178
S31508024660184619F01BF80023A7F8423000237B648A
S315080246709C4807F097FA034683F00103DBB2002B46
S3150802468000F0C480984B93F8E832002B50D1964B31
S31508024690D3F8D0329AB2944BA3F8EC22924B0F225B
S315080246A0C3F8D02210233B703B785AB28E4BB3F82C
S315080246B0EC321B0A9BB25BB203F00F035BB21343E5
S315080246C05BB2DBB23B70884BB3F8EC32DBB27B7081
S315080246D03B4602333E221946824807F0BAFA034697
S315080246E0002B00F0FC80FCF70FFD3B461A467F497B
S315080246F0FEF7B0FF7C4BB3F8EC323E3B9AB27A4BEC
S31508024700A3F8EC22784BB3F8EA3201339AB2764B25
S31508024710A3F8EA22744B012283F8E822724BFF229D
S3150802472083F8EE22704B4FF4FA62C3F8F022D6E011
S315080247306D4B93F8EE32002B05D06B4B93F8EE32A5
S31508024740012B40F0CC80684BB3F8EC323E2B02D9F1
S3150802475040237B6404E0644BB3F8EC3201337B6498
S3150802476020233B703B785AB25F4BB3F8EA325BB20E
S3150802477003F00F035BB213435BB2DBB23B707B6C95
S315080247805A1E3B4601331946564807F062FA034653
S31508024790002B00F0A4807B6C9BB21846FDF78EF8BE
S315080247A00346514AC2F8D032FCF7AEFC3B461A46DB
S315080247B04E49FEF74FFF4C4BB3F8EC227B6C9BB28B
S315080247C0D31A9BB201339AB2474BA3F8EC22464B53
S315080247D0B3F8EA3201339AB2434BA3F8EA22424BC0
S315080247E0B3F8EC32002B7AD1242200213F4818F084
S315080247F055FF3D4B002283F8E8223B4B0022A3F8E3
S31508024800EA22394BFF2283F8EE2268E0384807F09D
S31508024810C9F9034683F00103DBB2002B5FD03B469E
S3150802482001221946324807F014FA0346002B53D0E0
S315080248303B781B09DBB2032B14D13B460133022218
S3150802484019462B4807F005FA0346002B47D0264B94
S315080248500322DA60FCF758FC3B461A462249FEF761
S31508024860F9FE3CE03B781B09DBB2002B37D13B460D
S315080248700133012219461E4807F0EBF90346002BBD
S315080248802CD03B781B029BB203F47063A7F8423024
S315080248907B781A46B7F842301343A7F84230B7F87E
S315080248A042203B4602331946114807F0D2F903461D
S315080248B0002B14D0B7F8423002339BB21846FCF7E5
S315080248C0FDFF0346084AD360FCF71EFC3B461A4620
S315080248D00549FEF7BFFE02E000BF00E000BF483709
S315080248E0BD4680BD48EB002094E8002058EB002026
S315080248F0B8E8002080B592B000AF3B4640220021BE
S31508024900184618F0CBFE0023A7F8423000237B6432
S315080249109C4807F047F9034683F00103DBB2002BF4
S3150802492000F0C480984B93F8E832002B50D1964B8E
S31508024930D3F8D0329AB2944BA3F8EC22924B0F22B8
S31508024940C3F8D02210233B703B785AB28E4BB3F889
S31508024950EC321B0A9BB25BB203F00F035BB2134342
S315080249605BB2DBB23B70884BB3F8EC32DBB27B70DE
S315080249703B4602333E221946824807F06AF9034645
S31508024980002B00F0FC80FCF7BFFB3B461A467F492A
S31508024990FEF760FE7C4BB3F8EC323E3B9AB27A4B9A
S315080249A0A3F8EC22784BB3F8EA3201339AB2764B83
S315080249B0A3F8EA22744B012283F8E822724BFF22FB
S315080249C083F8EE22704B4FF4FA62C3F8F022D6E06F
S315080249D06D4B93F8EE32002B05D06B4B93F8EE3203
S315080249E0012B40F0CC80684BB3F8EC323E2B02D94F
S315080249F040237B6404E0644BB3F8EC3201337B64F6
S31508024A0020233B703B785AB25F4BB3F8EA325BB26B
S31508024A1003F00F035BB213435BB2DBB23B707B6CF2
S31508024A205A1E3B4601331946564807F012F9034601
S31508024A30002B00F0A4807B6C9BB21846FCF73EFF65
S31508024A400346514AC2F8D032FCF75EFB3B461A4689
S31508024A504E49FEF7FFFD4C4BB3F8EC227B6C9BB23A
S31508024A60D31A9BB201339AB2474BA3F8EC22464BB0
S31508024A70B3F8EA3201339AB2434BA3F8EA22424B1D
S31508024A80B3F8EC32002B7AD1242200213F4818F0E1
S31508024A9005FE3D4B002283F8E8223B4B0022A3F891
S31508024AA0EA22394BFF2283F8EE2268E0384807F0FB
S31508024AB079F8034683F00103DBB2002B5FD03B464D
S31508024AC001221946324807F0C4F80346002B53D090
S31508024AD03B781B09DBB2032B14D13B460133022276
S31508024AE019462B4807F0B5F80346002B47D0264B44
S31508024AF00322DA60FCF708FB3B461A462249FEF710
S31508024B00A9FD3CE03B781B09DBB2002B37D13B46BB
S31508024B100133012219461E4807F09BF80346002B6B
S31508024B202CD03B781B029BB203F47063A7F8423081
S31508024B307B781A46B7F842301343A7F84230B7F8DB
S31508024B4042203B4602331946114807F082F80346CB
S31508024B50002B14D0B7F8423002339BB21846FCF742
S31508024B60ADFE0346084AD360FCF7CEFA3B461A4620
S31508024B700549FEF76FFD02E000BF00E000BF4837B7
S31508024B80BD4680BD4CFF002098FC00205CFF00203B
S31508024B90BCFC002080B592B000AF3B464022002103
S31508024BA0184618F07BFD0023A7F8423000237B64E1
S31508024BB09F4806F0F7FF034683F00103DBB2002B9A
S31508024BC000F0CA809B4B93F8E832002B53D1994BDD
S31508024BD0D3F8D0329AB2974BA3F8EC22954B0F2210
S31508024BE0C3F8D02210233B703B785AB2914BB3F8E4
S31508024BF0EC321B0A9BB25BB203F00F035BB21343A0
S31508024C005BB2DBB23B708B4BB3F8EC32DBB27B7038
S31508024C103B4602333E221946854807F01AF80346F0
S31508024C20002B00F00281844809F0C2FCFCF76CFAFA
S31508024C303B461A468149FEF70DFD7E4BB3F8EC3228
S31508024C403E3B9AB27B4BA3F8EC227A4BB3F8EA3294
S31508024C5001339AB2774BA3F8EA22764B012283F8FC
S31508024C60E822744BFF2283F8EE22724B4FF4FA6263
S31508024C70C3F8F022D9E06F4B93F8EE32002B05D039
S31508024C806C4B93F8EE32012B40F0CF80694BB3F8A8
S31508024C90EC323E2B02D940237B6404E0654BB3F821
S31508024CA0EC3201337B6420233B703B785AB2614B6A
S31508024CB0B3F8EA325BB203F00F035BB213435BB29B
S31508024CC0DBB23B707B6C5A1E3B4601331946584889
S31508024CD006F0BFFF0346002B00F0A780584809F0EC
S31508024CE067FC7B6C9BB21846FCF7E8FD0346514A03
S31508024CF0C2F8D032FCF708FA3B461A464F49FEF785
S31508024D00A9FC4C4BB3F8EC227B6C9BB2D31A9BB230
S31508024D1001339AB2474BA3F8EC22464BB3F8EA3270
S31508024D2001339AB2434BA3F8EA22424BB3F8EC3268
S31508024D30002B7AD124220021404818F0AFFC3D4BC3
S31508024D40002283F8E8223B4B0022A3F8EA22394BD9
S31508024D50FF2283F8EE2268E03A4806F023FF03466C
S31508024D6083F00103DBB2002B5FD03B4601221946D2
S31508024D70344806F06EFF0346002B53D03B781B09D6
S31508024D80DBB2032B14D13B460133022219462D48C6
S31508024D9006F05FFF0346002B47D0264B0322DA6054
S31508024DA0FCF7B2F93B461A462249FEF753FC3CE0A9
S31508024DB03B781B09DBB2002B37D13B460133012274
S31508024DC01946204806F045FF0346002B2CD03B78AF
S31508024DD01B029BB203F47063A7F842307B781A462B
S31508024DE0B7F842301343A7F84230B7F842203B4699
S31508024DF002331946134806F02CFF0346002B14D03B
S31508024E00B7F8423002339BB21846FCF757FD034601
S31508024E10084AD360FCF778F93B461A460549FEF775
S31508024E2019FC02E000BF00E000BF4837BD4680BD5E
S31508024E30501301209C100120180D0408601301204C
S31508024E40240D0408C010012080B592B000AF3B467D
S31508024E5040220021184618F021FC0023A7F8423008
S31508024E6000237B649C4806F09DFE034683F00103FB
S31508024E70DBB2002B00F0C480984B93F8E832002B83
S31508024E8050D1964BD3F8D0329AB2944BA3F8EC226F
S31508024E90924B0F22C3F8D02210233B703B785AB2AA
S31508024EA08E4BB3F8EC321B0A9BB25BB203F00F03CC
S31508024EB05BB213435BB2DBB23B70884BB3F8EC329E
S31508024EC0DBB27B703B4602333E221946824806F025
S31508024ED0C0FE0346002B00F0FC80FCF715F93B46A2
S31508024EE01A467F49FEF7B6FB7C4BB3F8EC323E3BDB
S31508024EF09AB27A4BA3F8EC22784BB3F8EA3201332A
S31508024F009AB2764BA3F8EA22744B012283F8E82276
S31508024F10724BFF2283F8EE22704B4FF4FA62C3F803
S31508024F20F022D6E06D4B93F8EE32002B05D06B4B90
S31508024F3093F8EE32012B40F0CC80684BB3F8EC3292
S31508024F403E2B02D940237B6404E0644BB3F8EC326F
S31508024F5001337B6420233B703B785AB25F4BB3F82C
S31508024F60EA325BB203F00F035BB213435BB2DBB206
S31508024F703B707B6C5A1E3B4601331946564806F06F
S31508024F8068FE0346002B00F0A4807B6C9BB2184691
S31508024F90FCF794FC0346514AC2F8D032FCF7B4F83F
S31508024FA03B461A464E49FEF755FB4C4BB3F8EC22E4
S31508024FB07B6C9BB2D31A9BB201339AB2474BA3F8C6
S31508024FC0EC22464BB3F8EA3201339AB2434BA3F8C2
S31508024FD0EA22424BB3F8EC32002B7AD12422002182
S31508024FE03F4818F05BFB3D4B002283F8E8223B4B17
S31508024FF00022A3F8EA22394BFF2283F8EE2268E060
S31508025000384806F0CFFD034683F00103DBB2002BD6
S315080250105FD03B4601221946324806F01AFE03467D
S31508025020002B53D03B781B09DBB2032B14D13B462A
S315080250300133022219462B4806F00BFE0346002BC3
S3150802504047D0264B0322DA60FCF75EF83B461A463F
S315080250502249FEF7FFFA3CE03B781B09DBB2002B3C
S3150802506037D13B460133012219461E4806F0F1FDA7
S315080250700346002B2CD03B781B029BB203F47063C9
S31508025080A7F842307B781A46B7F842301343A7F896
S315080250904230B7F842203B4602331946114806F019
S315080250A0D8FD0346002B14D0B7F8423002339BB220
S315080250B01846FCF703FC0346084AD360FCF724F8B3
S315080250C03B461A460549FEF7C5FA02E000BF00E06C
S315080250D000BF4837BD4680BD54270120A0240120C1
S315080250E064270120C424012080B592B000AF3B4654
S315080250F040220021184618F0D1FA0023A7F84230B8
S3150802510000237B649C4806F04DFD034683F00103A9
S31508025110DBB2002B00F0C480984B93F8E832002BE0
S3150802512050D1964BD3F8D0329AB2944BA3F8EC22CC
S31508025130924B0F22C3F8D02210233B703B785AB207
S315080251408E4BB3F8EC321B0A9BB25BB203F00F0329
S315080251505BB213435BB2DBB23B70884BB3F8EC32FB
S31508025160DBB27B703B4602333E221946824806F082
S3150802517070FD0346002B00F0FC80FBF7C5FF3B469B
S315080251801A467F49FEF766FA7C4BB3F8EC323E3B89
S315080251909AB27A4BA3F8EC22784BB3F8EA32013387
S315080251A09AB2764BA3F8EA22744B012283F8E822D4
S315080251B0724BFF2283F8EE22704B4FF4FA62C3F861
S315080251C0F022D6E06D4B93F8EE32002B05D06B4BEE
S315080251D093F8EE32012B40F0CC80684BB3F8EC32F0
S315080251E03E2B02D940237B6404E0644BB3F8EC32CD
S315080251F001337B6420233B703B785AB25F4BB3F88A
S31508025200EA325BB203F00F035BB213435BB2DBB263
S315080252103B707B6C5A1E3B4601331946564806F0CC
S3150802522018FD0346002B00F0A4807B6C9BB218463F
S31508025230FCF744FB0346514AC2F8D032FBF764FF37
S315080252403B461A464E49FEF705FA4C4BB3F8EC2292
S315080252507B6C9BB2D31A9BB201339AB2474BA3F823
S31508025260EC22464BB3F8EA3201339AB2434BA3F81F
S31508025270EA22424BB3F8EC32002B7AD124220021DF
S315080252803F4818F00BFA3D4B002283F8E8223B4BC5
S315080252900022A3F8EA22394BFF2283F8EE2268E0BD
S315080252A0384806F07FFC034683F00103DBB2002B85
S315080252B05FD03B4601221946324806F0CAFC03462D
S315080252C0002B53D03B781B09DBB2032B14D13B4688
S315080252D00133022219462B4806F0BBFC0346002B73
S315080252E047D0264B0322DA60FBF70EFF3B461A46E7
S315080252F02249FEF7AFF93CE03B781B09DBB2002BEB
S3150802530037D13B460133012219461E4806F0A1FC55
S315080253100346002B2CD03B781B029BB203F4706326
S31508025320A7F842307B781A46B7F842301343A7F8F3
S315080253304230B7F842203B4602331946114806F076
S3150802534088FC0346002B14D0B7F8423002339BB2CE
S315080253501846FCF7B3FA0346084AD360FBF7D4FEAD
S315080253603B461A460549FEF775F902E000BF00E01A
S3150802537000BF4837BD4680BD583B0120A4380120EE
S31508025380683B0120C838012080B592B000AF3B4681
S3150802539040220021184618F081F90023A7F8423066
S315080253A000237B649C4806F0FDFB034683F0010359
S315080253B0DBB2002B00F0C480984B93F8E832002B3E
S315080253C050D1964BD3F8D0329AB2944BA3F8EC222A
S315080253D0924B0F22C3F8D02210233B703B785AB265
S315080253E08E4BB3F8EC321B0A9BB25BB203F00F0387
S315080253F05BB213435BB2DBB23B70884BB3F8EC3259
S31508025400DBB27B703B4602333E221946824806F0DF
S3150802541020FC0346002B00F0FC80FBF775FE3B469A
S315080254201A467F49FEF716F97C4BB3F8EC323E3B37
S315080254309AB27A4BA3F8EC22784BB3F8EA320133E4
S315080254409AB2764BA3F8EA22744B012283F8E82231
S31508025450724BFF2283F8EE22704B4FF4FA62C3F8BE
S31508025460F022D6E06D4B93F8EE32002B05D06B4B4B
S3150802547093F8EE32012B40F0CC80684BB3F8EC324D
S315080254803E2B02D940237B6404E0644BB3F8EC322A
S3150802549001337B6420233B703B785AB25F4BB3F8E7
S315080254A0EA325BB203F00F035BB213435BB2DBB2C1
S315080254B03B707B6C5A1E3B4601331946564806F02A
S315080254C0C8FB0346002B00F0A4807B6C9BB21846EF
S315080254D0FCF7F4F90346514AC2F8D032FBF714FE38
S315080254E03B461A464E49FEF7B5F84C4BB3F8EC2242
S315080254F07B6C9BB2D31A9BB201339AB2474BA3F881
S31508025500EC22464BB3F8EA3201339AB2434BA3F87C
S31508025510EA22424BB3F8EC32002B7AD1242200213C
S315080255203F4818F0BBF83D4B002283F8E8223B4B74
S315080255300022A3F8EA22394BFF2283F8EE2268E01A
S31508025540384806F02FFB034683F00103DBB2002B33
S315080255505FD03B4601221946324806F07AFB0346DB
S31508025560002B53D03B781B09DBB2032B14D13B46E5
S315080255700133022219462B4806F06BFB0346002B21
S3150802558047D0264B0322DA60FBF7BEFD3B461A4696
S315080255902249FEF75FF83CE03B781B09DBB2002B99
S315080255A037D13B460133012219461E4806F051FB04
S315080255B00346002B2CD03B781B029BB203F4706384
S315080255C0A7F842307B781A46B7F842301343A7F851
S315080255D04230B7F842203B4602331946114806F0D4
S315080255E038FB0346002B14D0B7F8423002339BB27D
S315080255F01846FCF763F90346084AD360FBF784FDAD
S315080256003B461A460549FEF725F802E000BF00E0C8
S3150802561000BF4837BD4680BD5C4F0120A84C01201B
S315080256206C4F0120CC4C012080B592B000AF3B46AE
S3150802563040220021184618F031F80023A7F8423014
S3150802564000237B649C4806F0ADFA034683F0010307
S31508025650DBB2002B00F0C480984B93F8E832002B9B
S3150802566050D1964BD3F8D0329AB2944BA3F8EC2287
S31508025670924B0F22C3F8D02210233B703B785AB2C2
S315080256808E4BB3F8EC321B0A9BB25BB203F00F03E4
S315080256905BB213435BB2DBB23B70884BB3F8EC32B6
S315080256A0DBB27B703B4602333E221946824806F03D
S315080256B0D0FA0346002B00F0FC80FBF725FD3B469B
S315080256C01A467F49FDF7C6FF7C4BB3F8EC323E3BE0
S315080256D09AB27A4BA3F8EC22784BB3F8EA32013342
S315080256E09AB2764BA3F8EA22744B012283F8E8228F
S315080256F0724BFF2283F8EE22704B4FF4FA62C3F81C
S31508025700F022D6E06D4B93F8EE32002B05D06B4BA8
S3150802571093F8EE32012B40F0CC80684BB3F8EC32AA
S315080257203E2B02D940237B6404E0644BB3F8EC3287
S3150802573001337B6420233B703B785AB25F4BB3F844
S31508025740EA325BB203F00F035BB213435BB2DBB21E
S315080257503B707B6C5A1E3B4601331946564806F087
S3150802576078FA0346002B00F0A4807B6C9BB218469D
S31508025770FCF7A4F80346514AC2F8D032FBF7C4FC38
S315080257803B461A464E49FDF765FF4C4BB3F8EC22E9
S315080257907B6C9BB2D31A9BB201339AB2474BA3F8DE
S315080257A0EC22464BB3F8EA3201339AB2434BA3F8DA
S315080257B0EA22424BB3F8EC32002B7AD1242200219A
S315080257C03F4817F06BFF3D4B002283F8E8223B4B1C
S315080257D00022A3F8EA22394BFF2283F8EE2268E078
S315080257E0384806F0DFF9034683F00103DBB2002BE3
S315080257F05FD03B4601221946324806F02AFA03468A
S31508025800002B53D03B781B09DBB2032B14D13B4642
S315080258100133022219462B4806F01BFA0346002BCF
S3150802582047D0264B0322DA60FBF76EFC3B461A4644
S315080258302249FDF70FFF3CE03B781B09DBB2002B40
S3150802584037D13B460133012219461E4806F001FAB2
S315080258500346002B2CD03B781B029BB203F47063E1
S31508025860A7F842307B781A46B7F842301343A7F8AE
S315080258704230B7F842203B4602331946114806F031
S31508025880E8F90346002B14D0B7F8423002339BB22C
S315080258901846FCF713F80346084AD360FBF734FCAC
S315080258A03B461A460549FDF7D5FE02E000BF00E071
S315080258B000BF4837BD4680BD60630120AC60012049
S315080258C070630120D060012080B592B000AF3B46DC
S315080258D040220021184617F0E1FE0023A7F84230BD
S315080258E000237B649C4806F05DF9034683F00103B6
S315080258F0DBB2002B00F0C480984B93F8E832002BF9
S3150802590050D1964BD3F8D0329AB2944BA3F8EC22E4
S31508025910924B0F22C3F8D02210233B703B785AB21F
S315080259208E4BB3F8EC321B0A9BB25BB203F00F0341
S315080259305BB213435BB2DBB23B70884BB3F8EC3213
S31508025940DBB27B703B4602333E221946824806F09A
S3150802595080F90346002B00F0FC80FBF7D5FB3B469B
S315080259601A467F49FDF776FE7C4BB3F8EC323E3B8E
S315080259709AB27A4BA3F8EC22784BB3F8EA3201339F
S315080259809AB2764BA3F8EA22744B012283F8E822EC
S31508025990724BFF2283F8EE22704B4FF4FA62C3F879
S315080259A0F022D6E06D4B93F8EE32002B05D06B4B06
S315080259B093F8EE32012B40F0CC80684BB3F8EC3208
S315080259C03E2B02D940237B6404E0644BB3F8EC32E5
S315080259D001337B6420233B703B785AB25F4BB3F8A2
S315080259E0EA325BB203F00F035BB213435BB2DBB27C
S315080259F03B707B6C5A1E3B4601331946564806F0E5
S31508025A0028F90346002B00F0A4807B6C9BB218464B
S31508025A10FBF754FF0346514AC2F8D032FBF774FB30
S31508025A203B461A464E49FDF715FE4C4BB3F8EC2297
S31508025A307B6C9BB2D31A9BB201339AB2474BA3F83B
S31508025A40EC22464BB3F8EA3201339AB2434BA3F837
S31508025A50EA22424BB3F8EC32002B7AD124220021F7
S31508025A603F4817F01BFE3D4B002283F8E8223B4BCA
S31508025A700022A3F8EA22394BFF2283F8EE2268E0D5
S31508025A80384806F08FF8034683F00103DBB2002B91
S31508025A905FD03B4601221946324806F0DAF8034639
S31508025AA0002B53D03B781B09DBB2032B14D13B46A0
S31508025AB00133022219462B4806F0CBF80346002B7F
S31508025AC047D0264B0322DA60FBF71EFB3B461A46F3
S31508025AD02249FDF7BFFD3CE03B781B09DBB2002BF0
S31508025AE037D13B460133012219461E4806F0B1F862
S31508025AF00346002B2CD03B781B029BB203F470633F
S31508025B00A7F842307B781A46B7F842301343A7F80B
S31508025B104230B7F842203B4602331946114806F08E
S31508025B2098F80346002B14D0B7F8423002339BB2DA
S31508025B301846FBF7C3FE0346084AD360FBF7E4FAA6
S31508025B403B461A460549FDF785FD02E000BF00E01F
S31508025B5000BF4837BD4680BD64770120B074012076
S31508025B6074770120D474012080B592B000AF3B4609
S31508025B7040220021184617F091FD0023A7F842306B
S31508025B8000237B649C4806F00DF8034683F0010364
S31508025B90DBB2002B00F0C480984B93F8E832002B56
S31508025BA050D1964BD3F8D0329AB2944BA3F8EC2242
S31508025BB0924B0F22C3F8D02210233B703B785AB27D
S31508025BC08E4BB3F8EC321B0A9BB25BB203F00F039F
S31508025BD05BB213435BB2DBB23B70884BB3F8EC3271
S31508025BE0DBB27B703B4602333E221946824806F0F8
S31508025BF030F80346002B00F0FC80FBF785FA3B469B
S31508025C001A467F49FDF726FD7C4BB3F8EC323E3B3C
S31508025C109AB27A4BA3F8EC22784BB3F8EA320133FC
S31508025C209AB2764BA3F8EA22744B012283F8E82249
S31508025C30724BFF2283F8EE22704B4FF4FA62C3F8D6
S31508025C40F022D6E06D4B93F8EE32002B05D06B4B63
S31508025C5093F8EE32012B40F0CC80684BB3F8EC3265
S31508025C603E2B02D940237B6404E0644BB3F8EC3242
S31508025C7001337B6420233B703B785AB25F4BB3F8FF
S31508025C80EA325BB203F00F035BB213435BB2DBB2D9
S31508025C903B707B6C5A1E3B4601331946564805F043
S31508025CA0D8FF0346002B00F0A4807B6C9BB21846F3
S31508025CB0FBF704FE0346514AC2F8D032FBF724FA30
S31508025CC03B461A464E49FDF7C5FC4C4BB3F8EC2247
S31508025CD07B6C9BB2D31A9BB201339AB2474BA3F899
S31508025CE0EC22464BB3F8EA3201339AB2434BA3F895
S31508025CF0EA22424BB3F8EC32002B7AD12422002155
S31508025D003F4817F0CBFC3D4B002283F8E8223B4B79
S31508025D100022A3F8EA22394BFF2283F8EE2268E032
S31508025D20384805F03FFF034683F00103DBB2002B38
S31508025D305FD03B4601221946324805F08AFF0346E0
S31508025D40002B53D03B781B09DBB2032B14D13B46FD
S31508025D500133022219462B4805F07BFF0346002B26
S31508025D6047D0264B0322DA60FBF7CEF93B461A46A2
S31508025D702249FDF76FFC3CE03B781B09DBB2002B9E
S31508025D8037D13B460133012219461E4805F061FF09
S31508025D900346002B2CD03B781B029BB203F470639C
S31508025DA0A7F842307B781A46B7F842301343A7F869
S31508025DB04230B7F842203B4602331946114805F0ED
S31508025DC048FF0346002B14D0B7F8423002339BB281
S31508025DD01846FBF773FD0346084AD360FBF794F9A6
S31508025DE03B461A460549FDF735FC02E000BF00E0CE
S31508025DF000BF4837BD4680BD688B0120B4880120A4
S31508025E00788B0120D888012080B582B000AF7860EF
S31508025E100B467B807B881A467968034805F0DEFEC6
S31508025E2000BF0837BD4680BDB89C012080B59AB030
S31508025E3000AF3B1D64220021184617F02FFC0F48BD
S31508025E4005F0B0FE034683F00103DBB2002B11D046
S31508025E503B1D64221946094805F0FBFE0346002B42
S31508025E6008D0FBF751F93B1D03F124023B1D1946E5
S31508025E70FDF7F0FB00BF6837BD4680BDB89C012020
S31508025E8080B500AF174B93F8E832002B28D0154B94
S31508025E9093F8EE32FF2B23D1124BD3F8F032002BB4
S31508025EA007D0104BD3F8F032013B0E4AC2F8F03253
S31508025EB016E0242200210C4817F0F0FB4FF47D620D
S31508025EC00A490B4805F0E4FD064B002283F8E8224E
S31508025ED0044B0022A3F8EA22024BFF2283F8EE22A1
S31508025EE000BF80BD8084002044870020748700207C
S31508025EF03487002080B500AF174B93F8E832002BA1
S31508025F0028D0154B93F8EE32FF2B23D1124BD3F838
S31508025F10F032002B07D0104BD3F8F032013B0E4A71
S31508025F20C2F8F03216E0242200210C4817F0B6FB1C
S31508025F304FF47D620A490B4805F0AAFD064B00227A
S31508025F4083F8E822044B0022A3F8EA22024BFF2236
S31508025F5083F8EE2200BF80BD84980020489B00206B
S31508025F60789B0020389B002080B500AF174B93F82A
S31508025F70E832002B28D0154B93F8EE32FF2B23D1AB
S31508025F80124BD3F8F032002B07D0104BD3F8F0326D
S31508025F90013B0E4AC2F8F03216E0242200210C48D0
S31508025FA017F07CFB4FF47D620A490B4805F070FD39
S31508025FB0064B002283F8E822044B0022A3F8EA22C1
S31508025FC0024BFF2283F8EE2200BF80BD88AC002078
S31508025FD04CAF00207CAF00203CAF002080B500AF5C
S31508025FE0174B93F8E832002B28D0154B93F8EE326C
S31508025FF0FF2B23D1124BD3F8F032002B07D0104BCC
S31508026000D3F8F032013B0E4AC2F8F03216E02422E7
S3150802601000210C4817F042FB4FF47D620A490B48EF
S3150802602005F036FD064B002283F8E822044B0022CF
S31508026030A3F8EA22024BFF2283F8EE2200BF80BDB4
S315080260408CC0002050C3002080C3002040C300201B
S3150802605080B500AF174B93F8E832002B28D0154BC2
S3150802606093F8EE32FF2B23D1124BD3F8F032002BE2
S3150802607007D0104BD3F8F032013B0E4AC2F8F03281
S3150802608016E0242200210C4817F008FB4FF47D6223
S315080260900A490B4805F0FCFC064B002283F8E82265
S315080260A0044B0022A3F8EA22024BFF2283F8EE22CF
S315080260B000BF80BD90D4002054D7002084D700208A
S315080260C044D7002080B500AF174B93F8E832002B6F
S315080260D028D0154B93F8EE32FF2B23D1124BD3F867
S315080260E0F032002B07D0104BD3F8F032013B0E4AA0
S315080260F0C2F8F03216E0242200210C4817F0CEFA34
S315080261004FF47D620A490B4805F0C2FC064B002291
S3150802611083F8E822044B0022A3F8EA22024BFF2264
S3150802612083F8EE2200BF80BD94E8002058EB0020D9
S3150802613088EB002048EB002080B500AF174B93F898
S31508026140E832002B28D0154B93F8EE32FF2B23D1D9
S31508026150124BD3F8F032002B07D0104BD3F8F0329B
S31508026160013B0E4AC2F8F03216E0242200210C48FE
S3150802617017F094FA4FF47D620A490B4805F088FC39
S31508026180064B002283F8E822044B0022A3F8EA22EF
S31508026190024BFF2283F8EE2200BF80BD98FC002046
S315080261A05CFF00208CFF00204CFF002080B500AF6A
S315080261B0194B93F8E832002B2BD0174B93F8EE3293
S315080261C0FF2B26D1144BD3F8F032002B07D0124BF3
S315080261D0D3F8F032013B104AC2F8F03219E0242211
S315080261E000210E4817F05AFA4FF47D620C490D4801
S315080261F005F04EFC084B002283F8E822064B0022E3
S31508026200A3F8EA22044BFF2283F8EE22064808F096
S31508026210CFF900BF80BD00BF9C100120601301208A
S315080262209013012050130120300D040880B500AFE9
S31508026230174B93F8E832002B28D0154B93F8EE3219
S31508026240FF2B23D1124BD3F8F032002B07D0104B79
S31508026250D3F8F032013B0E4AC2F8F03216E0242295
S3150802626000210C4817F01AFA4FF47D620A490B48C6
S3150802627005F00EFC064B002283F8E822044B0022A6
S31508026280A3F8EA22024BFF2283F8EE2200BF80BD62
S31508026290A0240120642701209427012054270120E5
S315080262A080B500AF174B93F8E832002B28D0154B70
S315080262B093F8EE32FF2B23D1124BD3F8F032002B90
S315080262C007D0104BD3F8F032013B0E4AC2F8F0322F
S315080262D016E0242200210C4817F0E0F94FF47D62FB
S315080262E00A490B4805F0D4FB064B002283F8E8223C
S315080262F0044B0022A3F8EA22024BFF2283F8EE227D
S3150802630000BF80BDA4380120683B0120983B0120CC
S31508026310583B012080B500AF174B93F8E832002BA3
S3150802632028D0154B93F8EE32FF2B23D1124BD3F814
S31508026330F032002B07D0104BD3F8F032013B0E4A4D
S31508026340C2F8F03216E0242200210C4817F0A6F90A
S315080263504FF47D620A490B4805F09AFB064B002268
S3150802636083F8E822044B0022A3F8EA22024BFF2212
S3150802637083F8EE2200BF80BDA84C01206C4F012095
S315080263809C4F01205C4F012080B500AF174B93F854
S31508026390E832002B28D0154B93F8EE32FF2B23D187
S315080263A0124BD3F8F032002B07D0104BD3F8F03249
S315080263B0013B0E4AC2F8F03216E0242200210C48AC
S315080263C017F06CF94FF47D620A490B4805F060FB39
S315080263D0064B002283F8E822044B0022A3F8EA229D
S315080263E0024BFF2283F8EE2200BF80BDAC6001207B
S315080263F070630120A06301206063012080B500AFAD
S31508026400174B93F8E832002B28D0154B93F8EE3247
S31508026410FF2B23D1124BD3F8F032002B07D0104BA7
S31508026420D3F8F032013B0E4AC2F8F03216E02422C3
S3150802643000210C4817F032F94FF47D620A490B48DD
S3150802644005F026FB064B002283F8E822044B0022BD
S31508026450A3F8EA22024BFF2283F8EE2200BF80BD90
S31508026460B074012074770120A47701206477012093
S3150802647080B500AF174B93F8E832002B28D0154B9E
S3150802648093F8EE32FF2B23D1124BD3F8F032002BBE
S3150802649007D0104BD3F8F032013B0E4AC2F8F0325D
S315080264A016E0242200210C4817F0F8F84FF47D6212
S315080264B00A490B4805F0ECFA064B002283F8E82253
S315080264C0044B0022A3F8EA22024BFF2283F8EE22AB
S315080264D000BF80BDB4880120788B0120A88B0120DB
S315080264E0688B012080B582B000AF78600B467B804E
S315080264F0786803F0A3F800BF0837BD4680BD80B5AB
S3150802650082B000AF78600B467B80786803F09AF910
S3150802651000BF0837BD4680BD80B582B000AF78603F
S315080265200B467B80786803F08FFA00BF0837BD46B2
S3150802653080BD80B582B000AF78600B467B807868F4
S3150802654003F086FB00BF0837BD4680BD80B582B022
S3150802655000AF78600B467B80786803F07BFC00BF4F
S315080265600837BD4680BD80B582B000AF78600B465D
S315080265707B80786803F072FD00BF0837BD4680BD90
S3150802658080B582B000AF78600B467B80786803F0EE
S3150802659067FE00BF0837BD4680BD80B582B000AF32
S315080265A078600B467B80786803F05EFF00BF083789
S315080265B0BD4680BD80B582B000AF78600B467B8051
S315080265C0786804F08DF800BF0837BD4680BD80B5EF
S315080265D082B000AF78600B467B80786804F084F955
S315080265E000BF0837BD4680BD80B582B000AF78606F
S315080265F00B467B80786804F079FA00BF0837BD46F7
S3150802660080BD80B582B000AF78600B467B80786823
S3150802661004F070FB00BF0837BD4680BD80B582B066
S3150802662000AF78600B467B80786804F065FC00BF93
S315080266300837BD4680BD80B582B000AF78600B468C
S315080266407B80786804F05CFD00BF0837BD4680BDD4
S3150802665080B582B000AF78600B467B80786805F01B
S315080266603FF800BF0837BD4680BD000080B582B03E
S3150802667000AF78600B467B807B881A4679680348A8
S3150802668005F0ACFA00BF0837BD4680BD900C002065
S3150802669080B582B000AF78600B467B807B881A464D
S315080266A07968034805F09AFA00BF0837BD4680BDE7
S315080266B08814002080B582B000AF78600B467B80D4
S315080266C07B881A467968034805F088FA00BF0837B6
S315080266D0BD4680BD801C002080B582B000AF7860C0
S315080266E00B467B807B881A467968034805F076FA5A
S315080266F000BF0837BD4680BD7824002080B582B029
S3150802670000AF78600B467B807B881A467968034817
S3150802671005F064FA00BF0837BD4680BD702C00201C
S3150802672080B582B000AF78600B467B807B881A46BC
S315080267307968034805F052FA00BF0837BD4680BD9E
S315080267406834002080B582B000AF78600B467B8043
S315080267507B881A467968034805F040FA00BF08376D
S31508026760BD4680BD603C002080B582B000AF78602F
S315080267700B467B807B881A467968034805F02EFA11
S3150802678000BF0837BD4680BD5844002080B582B098
S3150802679000AF78600B467B807B881946064807F06F
S315080267A007FF7B881A467968044805F017FA00BF7E
S315080267B00837BD4680BD00BF3C0D0408504C00207A
S315080267C080B582B000AF78600B467B807B881A461C
S315080267D07968034805F002FA00BF0837BD4680BD4E
S315080267E04854002080B582B000AF78600B467B80A3
S315080267F07B881A467968034805F0F0F900BF08371E
S31508026800BD4680BD405C002080B582B000AF78608E
S315080268100B467B807B881A467968034805F0DEF9C1
S3150802682000BF0837BD4680BD3864002080B582B0F7
S3150802683000AF78600B467B807B881A4679680348E6
S3150802684005F0CCF900BF0837BD4680BD306C002084
S3150802685080B582B000AF78600B467B807B881A468B
S315080268607968034805F0BAF900BF0837BD4680BD06
S315080268702874002080B582B000AF78600B467B8012
S315080268807B881A467968034805F0A8F900BF0837D5
S31508026890BD4680BD207C002080B59AB000AF3B463D
S315080268A068220021184616F0F9FE0E4805F07AF914
S315080268B0034683F00103DBB2002B0ED004E03B460D
S315080268C068211846FFF70EFE3B4668221946054818
S315080268D005F0BFF90346002BF1D100BF6837BD4664
S315080268E080BD00BF900C002080B59AB000AF3B4631
S315080268F068220021184616F0D1FE0E4805F052F914
S31508026900034683F00103DBB2002B0ED004E03B46BC
S3150802691068211846FFF7F3FD3B46682219460548E3
S3150802692005F097F90346002BF1D100BF6837BD463B
S3150802693080BD00BF8814002080B59AB000AF3B46E0
S3150802694068220021184616F0A9FE0E4805F02AF913
S31508026950034683F00103DBB2002B0ED004E03B466C
S3150802696068211846FFF7D8FD3B46682219460548AE
S3150802697005F06FF90346002BF1D100BF6837BD4613
S3150802698080BD00BF801C002080B59AB000AF3B4690
S3150802699068220021184616F081FE0E4805F002F913
S315080269A0034683F00103DBB2002B0ED004E03B461C
S315080269B068211846FFF7BDFD3B4668221946054879
S315080269C005F047F90346002BF1D100BF6837BD46EB
S315080269D080BD00BF7824002080B59AB000AF3B4640
S315080269E068220021184616F059FE0E4805F0DAF814
S315080269F0034683F00103DBB2002B0ED004E03B46CC
S31508026A0068211846FFF7A2FD3B4668221946054843
S31508026A1005F01FF90346002BF1D100BF6837BD46C2
S31508026A2080BD00BF702C002080B59AB000AF3B46EF
S31508026A3068220021184616F031FE0E4805F0B2F813
S31508026A40034683F00103DBB2002B0ED004E03B467B
S31508026A5068211846FFF787FD3B466822194605480E
S31508026A6005F0F7F80346002BF1D100BF6837BD469B
S31508026A7080BD00BF6834002080B59AB000AF3B469F
S31508026A8068220021184616F009FE0E4805F08AF813
S31508026A90034683F00103DBB2002B0ED004E03B462B
S31508026AA068211846FFF76CFD3B46682219460548D9
S31508026AB005F0CFF80346002BF1D100BF6837BD4673
S31508026AC080BD00BF603C002080B59AB000AF3B464F
S31508026AD068220021184616F0E1FD0E4805F062F814
S31508026AE0034683F00103DBB2002B0ED004E03B46DB
S31508026AF068211846FFF751FD3B46682219460548A4
S31508026B0005F0A7F80346002BF1D100BF6837BD464A
S31508026B1080BD00BF5844002080B59AB000AF3B46FE
S31508026B2068220021184616F0B9FD0E4805F03AF813
S31508026B30034683F00103DBB2002B0ED004E03B468A
S31508026B4068211846FFF736FD3B466822194605486E
S31508026B5005F07FF80346002BF1D100BF6837BD4622
S31508026B6080BD00BF504C002080B59AB000AF3B46AE
S31508026B7068220021184616F091FD0E4805F012F813
S31508026B80034683F00103DBB2002B0ED004E03B463A
S31508026B9068211846FFF71BFD3B4668221946054839
S31508026BA005F057F80346002BF1D100BF6837BD46FA
S31508026BB080BD00BF4854002080B59AB000AF3B465E
S31508026BC068220021184616F069FD0E4804F0EAFF0D
S31508026BD0034683F00103DBB2002B0ED004E03B46EA
S31508026BE068211846FFF700FD3B4668221946054804
S31508026BF005F02FF80346002BF1D100BF6837BD46D2
S31508026C0080BD00BF405C002080B59AB000AF3B460D
S31508026C1068220021184616F041FD0E4804F0C2FF0C
S31508026C20034683F00103DBB2002B0ED004E03B4699
S31508026C3068211846FFF7E5FC3B46682219460548CF
S31508026C4005F007F80346002BF1D100BF6837BD46A9
S31508026C5080BD00BF3864002080B59AB000AF3B46BD
S31508026C6068220021184616F019FD0E4804F09AFF0C
S31508026C70034683F00103DBB2002B0ED004E03B4649
S31508026C8068211846FFF7CAFC3B466822194605489A
S31508026C9004F0DFFF0346002BF1D100BF6837BD467B
S31508026CA080BD00BF306C002080B59AB000AF3B466D
S31508026CB068220021184616F0F1FC0E4804F072FF0D
S31508026CC0034683F00103DBB2002B0ED004E03B46F9
S31508026CD068211846FFF7AFFC3B4668221946054865
S31508026CE004F0B7FF0346002BF1D100BF6837BD4653
S31508026CF080BD00BF2874002080B59AB000AF3B461D
S31508026D0068220021184616F0C9FC0E4804F04AFF0C
S31508026D10034683F00103DBB2002B0ED004E03B46A8
S31508026D2068211846FFF794FC3B466822194605482F
S31508026D3004F08FFF0346002BF1D100BF6837BD462A
S31508026D4080BD00BF207C002080B582B000AF78608D
S31508026D506D4A7B681360FAF713FB242200216B48FD
S31508026D6016F09CFC24220021694816F097FC24227E
S31508026D700021684816F092FC24220021664816F083
S31508026D808DFC24220021654816F088FC2422002165
S31508026D90634816F083FC24220021624816F07EFC22
S31508026DA024220021604816F079FC242200215F483B
S31508026DB016F074FC242200215D4816F06FFC24228A
S31508026DC000215C4816F06AFC242200215A4816F073
S31508026DD065FC24220021594816F060FC2422002171
S31508026DE0574816F05BFC24220021564816F056FC3A
S31508026DF024220021544816F051FC2422002153482B
S31508026E0016F04CFC24220021514816F047FC242295
S31508026E100021504816F042FC242200214E4816F062
S31508026E203DFC242200214D4816F038FC242200217C
S31508026E304B4816F033FC242200214A4816F02EFC51
S31508026E4024220021484816F029FC2422002147481A
S31508026E5016F024FC24220021454816F01FFC2422A1
S31508026E600021444816F01AFC24220021424816F052
S31508026E7015FC24220021414816F010FC2422002188
S31508026E803F4816F00BFC242200213E4816F006FC69
S31508026E90242200213C4816F001FC242200213B480A
S31508026EA016F0FCFB24220021394816F0F7FB2422AF
S31508026EB00021384816F0F2FB24220021364816F043
S31508026EC0EDFB24220021354816F0E8FB2422002196
S31508026ED0334816F0E3FB24220021324816F0DEFB83
S31508026EE024220021304816F0D9FB242200212F48FB
S31508026EF016F0D4FB242200212D4816F0CFFB00BF42
S31508026F000837BD4680BD00BF8C0C00208084002057
S31508026F10448700205497002084980020489B00202C
S31508026F2058AB002088AC00204CAF00205CBF002084
S31508026F308CC0002050C3002060D3002090D40020CB
S31508026F4054D7002064E7002094E8002058EB00207C
S31508026F5068FB002098FC00205CFF00206C0F0120D3
S31508026F609C1001206013012070230120A024012017
S31508026F706427012074370120A4380120683B0120C8
S31508026F80784B0120A84C01206C4F01207C5F012020
S31508026F90AC6001207063012080730120B074012067
S31508026FA07477012084870120B4880120788B012018
S31508026FB0889B012080B58AB002AF78600B467B8039
S31508026FC013463B800023BB600023FB607B683B6162
S31508026FD001237B617B88BB613B88FB610A4B1B688B
S31508026FE007F108021146184609F0B2FE064B186860
S31508026FF00123009301230222022109F003FF00BFA5
S315080270002037BD4680BD00BF8C0C002080B58CB0F1
S3150802701002AFF860B9607A604FF080433B610023A3
S315080270207B61FB68BB610123FB61BB683B627B68D2
S315080270307B620A4B1B6807F110021146184609F0D3
S3150802704087FE064B186801230093012302220221B8
S3150802705009F0D8FE00BF2837BD4680BD8C0C00203B
S3150802706080B500AF064B1B68184609F0FCFE044BB8
S315080270701B680022012118460AF018F900BF80BDD4
S315080270808C0C002080B485B000AF78607B681B68E2
S315080270901B6CBB600023FB60BB68DBB2002B02D013
S315080270A0BB68DBB2FB60FB6818461437BD465DF861
S315080270B0047B704780B485B000AF78607B681B6834
S315080270C01B6CBB600023FB60BB6803F4FE43002B0A
S315080270D006D0BB6803F4FE43FB60FB681B0AFB6031
S315080270E0FB6818461437BD465DF8047B70470000F6
S315080270F080B485B000AF78607B681B685B6CBB6048
S315080271000023FB60BB6803F00703002B2FD0BB6884
S3150802711003F00703013B052B20D801A252F823F0FE
S31508027120397102083F710208457102084B7102085B
S3150802713051710208577102080123FB600FE002230E
S31508027140FB600CE00323FB6009E00423FB6006E016
S315080271500523FB6003E00623FB6000E000BF7B68B3
S315080271601B685A6C7B681B6822F007025A64FB6824
S31508027170DBB218461437BD465DF8047B704700BF7C
S3150802718080B582B000AF78607B68013B052B27D8B3
S3150802719001A252F823F000BFB1710208B9710208C0
S315080271A0C1710208C9710208D1710208D9710208AF
S315080271B00D4807F0FDF913E00C4807F0F9F90FE05E
S315080271C00B4807F0F5F90BE00A4807F0F1F907E072
S315080271D0094807F0EDF903E0084807F0E9F900BFA6
S315080271E000BF0837BD4680BD480D0408540D040883
S315080271F0600D0408780D04088C0D0408A00D040817
S3150802720080B400AF034B1B781846BD465DF8047B75
S31508027210704700BF0000002080B400AF024B18463A
S31508027220BD465DF8047B704704A1012080B582B093
S3150802723000AF78600B467B807B881A4679684FF4E4
S31508027240006001F0DBFF00BF0837BD4680BD0000C5
S3150802725090B589B002AFF860B9601346FB80042086
S3150802726004F0CEF803460133DBB23B75CE237B75B9
S31508027270D623BB753B7D1946BB681B781A460B4855
S3150802728007F096F906F048FD044606F03BFD01466E
S3150802729007F11402FB880093BB68204614F0D7FC5A
S315080272A000BF00BF1C37BD4690BD00BFAC0D040829
S315080272B080B500AF4FF480720249034804F0E8FB38
S315080272C000BF80BD50AA0120E8A0012080B500AF0A
S315080272D0FFF7EEFF034B044A0449054814F003F985
S315080272E000BF80BD2D7202085172020804A1012056
S315080272F0F8A0012080B400AF024B1846BD465DF8DF
S31508027300047B70476CAB012080B582B000AF786011
S315080273100B467B807B881A4679684FF4803001F0E9
S315080273206DFF00BF0837BD4680BD000090B589B025
S3150802733002AFF860B9601346FB80082004F060F8D3
S3150802734003460133DBB23B75CE237B75D623BB7569
S315080273503B7D1946BB681B781A460B4807F028F985
S3150802736006F0DAFC044606F0CDFC014607F11402E3
S31508027370FB880093BB68204614F069FC00BF00BF77
S315080273801C37BD4690BD00BFD40D040880B500AFBA
S315080273904FF480720249034804F07AFB00BF80BDAD
S315080273A0B8B4012050AB012080B500AFFFF7EEFF5D
S315080273B0034B044A0449054814F095F800BF80BDFA
S315080273C0097302082D7302086CAB012060AB012019
S315080273D080B400AF024B1846BD465DF8047B704781
S315080273E0D4B5012080B582B000AF78600B467B80A9
S315080273F07B881A4679684FF4003001F0FFFE00BF19
S315080274000837BD4680BD000090B589B002AFF86066
S31508027410B9601346FB80092003F0F2FF03460133E5
S31508027420DBB23B75CE237B75D623BB753B7D1946EE
S31508027430BB681B781A46FB880A4807F0B9F806F0B3
S315080274406BFC044606F05EFC014607F11402FB8853
S315080274500093BB68204614F0FAFB00BF00BF1C3736
S31508027460BD4690BDFC0D040880B500AF4FF480728E
S315080274700249034804F00CFB00BF80BD20BF01206F
S31508027480B8B5012080B500AFFFF7EEFF034B044AFB
S315080274900449054814F027F800BF80BDE5730208C1
S315080274A009740208D4B50120C8B5012080B400AF1A
S315080274B0024B1846BD465DF8047B70473CC0012066
S315080274C080B582B000AF78600B467B807B881A460F
S315080274D079684FF4005001F091FE00BF0837BD46A7
S315080274E080BD000090B589B002AFF860B960134656
S315080274F0FB80052003F084FF03460133DBB23B75AC
S31508027500CE237B75D623BB753B7D1946BB681B7894
S315080275101A460B4807F04CF806F0FEFB044606F03E
S31508027520F1FB014607F11402FB880093BB6820466B
S3150802753014F08DFB00BF00BF1C37BD4690BD00BFCF
S315080275402C0E040880B500AF4FF480720249034836
S3150802755004F09EFA00BF80BD88C9012020C0012020
S3150802756080B500AFFFF7EEFF034B044A044905480E
S3150802757013F0B9FF00BF80BDC1740208E5740208A2
S315080275803CC0012030C0012080B400AF024B18462F
S31508027590BD465DF8047B7047A4CA012080B582B057
S315080275A000AF78600B467B807B881A4679684FF471
S315080275B0802001F023FE00BF0837BD4680BD0000CB
S315080275C090B589B002AFF860B9601346FB800A200D
S315080275D003F016FF03460133DBB23B75CE237B75F8
S315080275E0D623BB753B7D1946BB681B781A460B48E2
S315080275F006F0DEFF06F090FB044606F083FB014622
S3150802760007F11402FB880093BB68204614F01FFB9F
S3150802761000BF00BF1C37BD4690BD00BF540E04080C
S3150802762080B500AF4FF480720249034804F030FA7D
S3150802763000BF80BDF0D3012088CA012080B500AF03
S31508027640FFF7EEFF034B044A0449054813F04BFFC4
S3150802765000BF80BD9D750208C1750208A4CA012033
S3150802766098CA012080B400AF024B1846BD465DF8A1
S31508027670047B70470CD5012080B582B000AF7860D4
S315080276800B467B807B881A4679684FF4002001F006
S31508027690B5FD00BF0837BD4680BD000090B589B06C
S315080276A002AFF860B9601346FB800B2003F0A8FE10
S315080276B003460133DBB23B75CE237B75D623BB75F6
S315080276C03B7D1946BB681B781A460B4806F070FFC5
S315080276D006F022FB044606F015FB014607F11402E2
S315080276E0FB880093BB68204614F0B1FA00BF00BFBE
S315080276F01C37BD4690BD00BF7C0E040880B500AF9E
S315080277004FF480720249034804F0C2F900BF80BDF3
S3150802771058DE0120F0D4012080B500AFFFF7EEFF56
S31508027720034B044A0449054813F0DDFE00BF80BD39
S31508027730797602089D7602080CD5012000D501202B
S31508027740B0B5A4B006AFF860B9601346FB80002353
S31508027750A7F87630FB683B65FFF752FD0346002B18
S3150802776003D04FF080437B6501E000237B6500234D
S31508027770BB65FB8802339BB21846FAF79FF80346A5
S31508027780FB6500233B664FF480137B664FF40013B8
S31508027790BB660023FB6600233B6700233B743B7CE6
S315080277A05AB2FB881B0A9BB25BB203F00F035BB2A9
S315080277B013435BB2DBB23B74FB88DBB27B740223F6
S315080277C0A7F8763010E0B7F87630023BBA681A4462
S315080277D0B7F87630127878333B4403F8682CB7F852
S315080277E076300133A7F87630B7F87620FB8801336E
S315080277F09A42E8DD0023A7F876300DE0B7F876302E
S3150802780078333B4413F8683C1846FBF7EBFDB7F8A8
S3150802781076300133A7F87630B7F87620FB8801333D
S315080278209A42EBDD6D4607F160040FCC0FC523685B
S315080278302B6007F150030FCBFAF798F800BF783799
S31508027840BD46B0BDB0B5A4B006AFF860B960134680
S31508027850FB800023A7F87630FB683B65FFF7D0FC70
S315080278600346002B03D04FF080437B6501E00023DB
S315080278707B650023BB65FB8802339BB21846FAF781
S315080278801DF80346FB6500233B664FF480137B66AF
S315080278904FF40013BB660023FB6600233B670023F5
S315080278A03B743B7C5AB2FB881B0A9BB25BB203F061
S315080278B00F035BB213435BB2DBB23B74FB88DBB2EA
S315080278C07B740223A7F8763010E0B7F87630023BCD
S315080278D0BA681A44B7F87630127878333B4403F814
S315080278E0682CB7F876300133A7F87630B7F87620E1
S315080278F0FB8801339A42E8DD0023A7F876300DE0CB
S31508027900B7F8763078333B4413F8683C1846FBF7E9
S315080279107BFDB7F876300133A7F87630B7F87620CC
S31508027920FB8801339A42EBDD6D4607F160040FCC02
S315080279300FC523682B6007F150030FCBFAF72EF811
S3150802794000BF7837BD46B0BDB0B5A4B006AFF86083
S31508027950B9601346FB800023A7F87630FB683B65BF
S31508027960FFF74EFC0346002B03D04FF080437B659E
S3150802797001E000237B650023BB65FB8802339BB2CB
S315080279801846F9F79BFF0346FB6500233B664FF44F
S3150802799080137B664FF40013BB660023FB66002345
S315080279A03B6700233B743B7C5AB2FB881B0A9BB29B
S315080279B05BB203F00F035BB213435BB2DBB23B74F9
S315080279C0FB88DBB27B740223A7F8763010E0B7F89F
S315080279D07630023BBA681A44B7F8763012787833AA
S315080279E03B4403F8682CB7F876300133A7F87630AB
S315080279F0B7F87620FB8801339A42E8DD0023A7F818
S31508027A0076300DE0B7F8763078333B4413F8683CA5
S31508027A101846FBF70BFDB7F876300133A7F8763030
S31508027A20B7F87620FB8801339A42EBDD6D4607F1FB
S31508027A3060040FCC0FC523682B6007F150030FCBE8
S31508027A40F9F7C4FF00BF7837BD46B0BDB0B5A4B0DC
S31508027A5006AFF860B9601346FB800023A7F87630B4
S31508027A60FB683B65FFF7CCFB0346002B03D04FF0C0
S31508027A7080437B6501E000237B650023BB65FB88A9
S31508027A8002339BB21846F9F719FF0346FB65002332
S31508027A903B664FF480137B664FF40013BB660023E4
S31508027AA0FB6600233B6700233B743B7C5AB2FB8888
S31508027AB01B0A9BB25BB203F00F035BB213435BB2C2
S31508027AC0DBB23B74FB88DBB27B740223A7F8763001
S31508027AD010E0B7F87630023BBA681A44B7F876303F
S31508027AE0127878333B4403F8682CB7F876300133BA
S31508027AF0A7F87630B7F87620FB8801339A42E8DD94
S31508027B000023A7F876300DE0B7F8763078333B4491
S31508027B1013F8683C1846FBF79BFCB7F87630013336
S31508027B20A7F87630B7F87620FB8801339A42EBDD60
S31508027B306D4607F160040FCC0FC523682B6007F169
S31508027B4050030FCBF9F75AFF00BF7837BD46B0BDD1
S31508027B50B0B5A4B006AFF860B9601346FB8000233F
S31508027B60A7F87630FB683B65FFF74AFB0346002B0E
S31508027B7003D04FF080437B6501E000237B65002339
S31508027B80BB65FB8802339BB21846F9F797FE034694
S31508027B90FB6500233B664FF480137B664FF40013A4
S31508027BA0BB660023FB6600233B6700233B743B7CD2
S31508027BB05AB2FB881B0A9BB25BB203F00F035BB295
S31508027BC013435BB2DBB23B74FB88DBB27B740223E2
S31508027BD0A7F8763010E0B7F87630023BBA681A444E
S31508027BE0B7F87630127878333B4403F8682CB7F83E
S31508027BF076300133A7F87630B7F87620FB8801335A
S31508027C009A42E8DD0023A7F876300DE0B7F8763019
S31508027C1078333B4413F8683C1846FBF72BFCB7F855
S31508027C2076300133A7F87630B7F87620FB88013329
S31508027C309A42EBDD6D4607F160040FCC0FC5236847
S31508027C402B6007F150030FCBF9F7F0FE00BF783728
S31508027C50BD46B0BDB0B5A4B006AFF860B96013466C
S31508027C60FB800023A7F87630FB683B65FFF7C8FA66
S31508027C700346002B03D04FF080437B6501E00023C7
S31508027C807B650023BB65FB8802339BB21846F9F76E
S31508027C9015FE0346FB6500233B664FF480137B669D
S31508027CA04FF40013BB660023FB6600233B670023E1
S31508027CB03B743B7C5AB2FB881B0A9BB25BB203F04D
S31508027CC00F035BB213435BB2DBB23B74FB88DBB2D6
S31508027CD07B740223A7F8763010E0B7F87630023BB9
S31508027CE0BA681A44B7F87630127878333B4403F800
S31508027CF0682CB7F876300133A7F87630B7F87620CD
S31508027D00FB8801339A42E8DD0023A7F876300DE0B6
S31508027D10B7F8763078333B4413F8683C1846FBF7D5
S31508027D20BBFBB7F876300133A7F87630B7F876207A
S31508027D30FB8801339A42EBDD6D4607F160040FCCEE
S31508027D400FC523682B6007F150030FCBF9F786FEA0
S31508027D5000BF7837BD46B0BDB0B5A4B006AFF8606F
S31508027D60B9601346FB800023A7F87630FB683B65AB
S31508027D70FFF746FA0346002B03D04FF080437B6594
S31508027D8001E000237B650023BB65FB8802339BB2B7
S31508027D901846F9F793FD0346FB6500233B664FF445
S31508027DA080137B664FF40013BB660023FB66002331
S31508027DB03B6700233B743B7C5AB2FB881B0A9BB287
S31508027DC05BB203F00F035BB213435BB2DBB23B74E5
S31508027DD0FB88DBB27B740223A7F8763010E0B7F88B
S31508027DE07630023BBA681A44B7F876301278783396
S31508027DF03B4403F8682CB7F876300133A7F8763097
S31508027E00B7F87620FB8801339A42E8DD0023A7F803
S31508027E1076300DE0B7F8763078333B4413F8683C91
S31508027E201846FBF74BFBB7F876300133A7F87630DE
S31508027E30B7F87620FB8801339A42EBDD6D4607F1E7
S31508027E4060040FCC0FC523682B6007F150030FCBD4
S31508027E50F9F71CFE00BF7837BD46B0BDB0B5A4B071
S31508027E6006AFF860B9601346FB800023A7F87630A0
S31508027E70FB683B65FFF7C4F90346002B03D04FF0B6
S31508027E8080437B6501E000237B650023BB65FB8895
S31508027E9002339BB21846F9F711FD0346FB65002328
S31508027EA03B664FF480137B664FF40013BB660023D0
S31508027EB0FB6600233B6700233B743B7C5AB2FB8874
S31508027EC01B0A9BB25BB203F00F035BB213435BB2AE
S31508027ED0DBB23B74FB88DBB27B740223A7F87630ED
S31508027EE010E0B7F87630023BBA681A44B7F876302B
S31508027EF0127878333B4403F8682CB7F876300133A6
S31508027F00A7F87630B7F87620FB8801339A42E8DD7F
S31508027F100023A7F876300DE0B7F8763078333B447D
S31508027F2013F8683C1846FBF7DBFAB7F876300133E4
S31508027F30A7F87630B7F87620FB8801339A42EBDD4C
S31508027F406D4607F160040FCC0FC523682B6007F155
S31508027F5050030FCBF9F7B2FD00BF7837BD46B0BD67
S31508027F60B0B5A4B006AFF860B9601346FB8000232B
S31508027F70A7F87630FB683B65FFF742F90346002B04
S31508027F8003D04FF080437B6501E000237B65002325
S31508027F90BB65FB8802339BB21846F9F78FFC03468A
S31508027FA0FB6500233B664FF480137B664FF4001390
S31508027FB0BB660023FB6600233B6700233B743B7CBE
S31508027FC05AB2FB881B0A9BB25BB203F00F035BB281
S31508027FD013435BB2DBB23B74FB88DBB27B740223CE
S31508027FE0A7F8763010E0B7F87630023BBA681A443A
S31508027FF0B7F87630127878333B4403F8682CB7F82A
S3150802800076300133A7F87630B7F87620FB88013345
S315080280109A42E8DD0023A7F876300DE0B7F8763005
S3150802802078333B4413F8683C1846FBF76BFAB7F803
S3150802803076300133A7F87630B7F87620FB88013315
S315080280409A42EBDD6D4607F160040FCC0FC5236833
S315080280502B6007F150030FCBF9F748FD00BF7837BD
S31508028060BD46B0BDB0B5A4B006AFF860B960134658
S31508028070FB800023A7F87630FB683B65FFF7C0F85C
S315080280800346002B03D04FF080437B6501E00023B3
S315080280907B650023BB65FB8802339BB21846F9F75A
S315080280A00DFC0346FB6500233B664FF480137B6693
S315080280B04FF40013BB660023FB6600233B670023CD
S315080280C03B743B7C5AB2FB881B0A9BB25BB203F039
S315080280D00F035BB213435BB2DBB23B74FB88DBB2C2
S315080280E07B740223A7F8763010E0B7F87630023BA5
S315080280F0BA681A44B7F87630127878333B4403F8EC
S31508028100682CB7F876300133A7F87630B7F87620B8
S31508028110FB8801339A42E8DD0023A7F876300DE0A2
S31508028120B7F8763078333B4413F8683C1846FBF7C1
S31508028130FBF9B7F876300133A7F87630B7F8762028
S31508028140FB8801339A42EBDD6D4607F160040FCCDA
S315080281500FC523682B6007F150030FCBF9F7DEFC36
S3150802816000BF7837BD46B0BDB0B5A4B006AFF8605B
S31508028170B9601346FB800023A7F87630FB683B6597
S31508028180FFF73EF80346002B03D04FF080437B658A
S3150802819001E000237B650023BB65FB8802339BB2A3
S315080281A01846F9F78BFB0346FB6500233B664FF43B
S315080281B080137B664FF40013BB660023FB6600231D
S315080281C03B6700233B743B7C5AB2FB881B0A9BB273
S315080281D05BB203F00F035BB213435BB2DBB23B74D1
S315080281E0FB88DBB27B740223A7F8763010E0B7F877
S315080281F07630023BBA681A44B7F876301278783382
S315080282003B4403F8682CB7F876300133A7F8763082
S31508028210B7F87620FB8801339A42E8DD0023A7F8EF
S3150802822076300DE0B7F8763078333B4413F8683C7D
S315080282301846FBF78BF9B7F876300133A7F876308C
S31508028240B7F87620FB8801339A42EBDD6D4607F1D3
S3150802825060040FCC0FC523682B6007F150030FCBC0
S31508028260F9F774FC00BF7837BD46B0BDB0B5A4B007
S3150802827006AFF860B9601346FB800023A7F876308C
S31508028280FB683B65FEF7BCFF0346002B03D04FF0A5
S3150802829080437B6501E000237B650023BB65FB8881
S315080282A002339BB21846F9F709FB0346FB6500231E
S315080282B03B664FF480137B664FF40013BB660023BC
S315080282C0FB6600233B6700233B743B7C5AB2FB8860
S315080282D01B0A9BB25BB203F00F035BB213435BB29A
S315080282E0DBB23B74FB88DBB27B740223A7F87630D9
S315080282F010E0B7F87630023BBA681A44B7F8763017
S31508028300127878333B4403F8682CB7F87630013391
S31508028310A7F87630B7F87620FB8801339A42E8DD6B
S315080283200023A7F876300DE0B7F8763078333B4469
S3150802833013F8683C1846FBF71BF9B7F87630013391
S31508028340A7F87630B7F87620FB8801339A42EBDD38
S315080283506D4607F160040FCC0FC523682B6007F141
S3150802836050030FCBF9F70AFC00BF7837BD46B0BDFC
S31508028370B0B5A4B006AFF860B9601346FB80002317
S31508028380A7F87630FB683B65FEF73AFF0346002BF3
S3150802839003D04FF080437B6501E000237B65002311
S315080283A0BB65FB8802339BB21846F9F787FA034680
S315080283B0FB6500233B664FF480137B664FF400137C
S315080283C0BB660023FB6600233B6700233B743B7CAA
S315080283D05AB2FB881B0A9BB25BB203F00F035BB26D
S315080283E013435BB2DBB23B74FB88DBB27B740223BA
S315080283F0A7F8763010E0B7F87630023BBA681A4426
S31508028400B7F87630127878333B4403F8682CB7F815
S3150802841076300133A7F87630B7F87620FB88013331
S315080284209A42E8DD0023A7F876300DE0B7F87630F1
S3150802843078333B4413F8683C1846FBF7ABF8B7F8B1
S3150802844076300133A7F87630B7F87620FB88013301
S315080284509A42EBDD6D4607F160040FCC0FC523681F
S315080284602B6007F150030FCBF9F7A0FB00BF783753
S31508028470BD46B0BDB0B5A4B006AFF860B960134644
S31508028480FB800023A7F87630FB683B65FEF7B8FE4B
S315080284900346002B03D04FF080437B6501E000239F
S315080284A07B650023BB65FB8802339BB21846F9F746
S315080284B005FA0346FB6500233B664FF480137B6689
S315080284C04FF40013BB660023FB6600233B670023B9
S315080284D03B743B7C5AB2FB881B0A9BB25BB203F025
S315080284E00F035BB213435BB2DBB23B74FB88DBB2AE
S315080284F07B740223A7F8763010E0B7F87630023B91
S31508028500BA681A44B7F87630127878333B4403F8D7
S31508028510682CB7F876300133A7F87630B7F87620A4
S31508028520FB8801339A42E8DD0023A7F876300DE08E
S31508028530B7F8763078333B4413F8683C1846FBF7AD
S315080285403BF8B7F876300133A7F87630B7F87620D5
S31508028550FB8801339A42EBDD6D4607F160040FCCC6
S315080285600FC523682B6007F150030FCBF9F736FBCB
S3150802857000BF7837BD46B0BD80B58EB000AFF86093
S31508028580B9601346FB80002387F83730FB683B61E6
S31508028590FEF736FE0346002B03D04FF080437B617D
S315080285A001E000237B610023BB61FB88FB6100239A
S315080285B03B624FF480137B624FF40013BB620023C5
S315080285C0FB6200233B63FA8807F11003114618463B
S315080285D0F9F71CFB034687F8373097F83730002B34
S315080285E006D0FA8897F83730B9681846FAF77AFB48
S315080285F000BF3837BD4680BD80B58EB000AFF86083
S31508028600B9601346FB80002387F83730FB683B6165
S31508028610FEF7F6FD0346002B03D04FF080437B613D
S3150802862001E000237B610023BB61FB88FB61002319
S315080286303B624FF480137B624FF40013BB62002344
S31508028640FB6200233B63FA8807F1100311461846BA
S31508028650F9F776FB034687F8373097F83730002B59
S3150802866006D0FA8897F83730B9681846FAF77AFBC7
S3150802867000BF3837BD4680BD80B58EB000AFF86002
S31508028680B9601346FB80002387F83730FB683B61E5
S31508028690FEF7B6FD0346002B03D04FF080437B61FD
S315080286A001E000237B610023BB61FB88FB61002399
S315080286B03B624FF480137B624FF40013BB620023C4
S315080286C0FB6200233B63FA8807F11003114618463A
S315080286D0F9F7D0FB034687F8373097F83730002B7F
S315080286E006D0FA8897F83730B9681846FAF77AFB47
S315080286F000BF3837BD4680BD80B58EB000AFF86082
S31508028700B9601346FB80002387F83730FB683B6164
S31508028710FEF776FD0346002B03D04FF080437B61BC
S3150802872001E000237B610023BB61FB88FB61002318
S315080287303B624FF480137B624FF40013BB62002343
S31508028740FB6200233B63FA8807F1100311461846B9
S31508028750F9F72AFC034687F8373097F83730002BA3
S3150802876006D0FA8897F83730B9681846FAF77AFBC6
S3150802877000BF3837BD4680BD80B58EB000AFF86001
S31508028780B9601346FB80002387F83730FB683B61E4
S31508028790FEF736FD0346002B03D04FF080437B617C
S315080287A001E000237B610023BB61FB88FB61002398
S315080287B03B624FF480137B624FF40013BB620023C3
S315080287C0FB6200233B63FA8807F110031146184639
S315080287D0F9F784FC034687F8373097F83730002BC9
S315080287E006D0FA8897F83730B9681846FAF77AFB46
S315080287F000BF3837BD4680BD80B58EB000AFF86081
S31508028800B9601346FB80002387F83730FB683B6163
S31508028810FEF7F6FC0346002B03D04FF080437B613C
S3150802882001E000237B610023BB61FB88FB61002317
S315080288303B624FF480137B624FF40013BB62002342
S31508028840FB6200233B63FA8807F1100311461846B8
S31508028850F9F7DEFC034687F8373097F83730002BEE
S3150802886006D0FA8897F83730B9681846FAF77AFBC5
S3150802887000BF3837BD4680BD80B58EB000AFF86000
S31508028880B9601346FB80002387F83730FB683B61E3
S31508028890FEF7B6FC0346002B03D04FF080437B61FC
S315080288A001E000237B610023BB61FB88FB61002397
S315080288B03B624FF480137B624FF40013BB620023C2
S315080288C0FB6200233B63FA8807F110031146184638
S315080288D0F9F738FD034687F8373097F83730002B13
S315080288E006D0FA8897F83730B9681846FAF77AFB45
S315080288F000BF3837BD4680BD80B58EB000AFF86080
S31508028900B9601346FB80002387F83730FB683B6162
S31508028910FEF776FC0346002B03D04FF080437B61BB
S3150802892001E000237B610023BB61FB88FB61002316
S315080289303B624FF480137B624FF40013BB62002341
S31508028940FB6200233B63FA8807F1100311461846B7
S31508028950F9F792FD034687F8373097F83730002B38
S3150802896006D0FA8897F83730B9681846FAF77AFBC4
S3150802897000BF3837BD4680BD80B58EB000AFF860FF
S31508028980B9601346FB80002387F83730FB683B61E2
S31508028990FEF736FC0346002B03D04FF080437B617B
S315080289A001E000237B610023BB61FB88FB61002396
S315080289B03B624FF480137B624FF40013BB620023C1
S315080289C0FB6200233B63FA8807F110031146184637
S315080289D0F9F7ECFD034687F8373097F83730002B5E
S315080289E006D0FA8897F83730B9681846FAF77AFB44
S315080289F000BF3837BD4680BD80B58EB000AFF8607F
S31508028A00B9601346FB80002387F83730FB683B6161
S31508028A10FEF7F6FB0346002B03D04FF080437B613B
S31508028A2001E000237B610023BB61FB88FB61002315
S31508028A303B624FF480137B624FF40013BB62002340
S31508028A40FB6200233B63FA8807F1100311461846B6
S31508028A50F9F746FE034687F8373097F83730002B82
S31508028A6006D0FA8897F83730B9681846FAF77AFBC3
S31508028A7000BF3837BD4680BD80B58EB000AFF860FE
S31508028A80B9601346FB80002387F83730FB683B61E1
S31508028A90FEF7B6FB0346002B03D04FF080437B61FB
S31508028AA001E000237B610023BB61FB88FB61002395
S31508028AB03B624FF480137B624FF40013BB620023C0
S31508028AC0FB6200233B63FA8807F110031146184636
S31508028AD0F9F7A0FE034687F8373097F83730002BA8
S31508028AE006D0FA8897F83730B9681846FAF77AFB43
S31508028AF000BF3837BD4680BD80B58EB000AFF8607E
S31508028B00B9601346FB80002387F83730FB683B6160
S31508028B10FEF776FB0346002B03D04FF080437B61BA
S31508028B2001E000237B610023BB61FB88FB61002314
S31508028B303B624FF480137B624FF40013BB6200233F
S31508028B40FB6200233B63FA8807F1100311461846B5
S31508028B50F9F7FAFE034687F8373097F83730002BCD
S31508028B6006D0FA8897F83730B9681846FAF77AFBC2
S31508028B7000BF3837BD4680BD80B58EB000AFF860FD
S31508028B80B9601346FB80002387F83730FB683B61E0
S31508028B90FEF736FB0346002B03D04FF080437B617A
S31508028BA001E000237B610023BB61FB88FB61002394
S31508028BB03B624FF480137B624FF40013BB620023BF
S31508028BC0FB6200233B63FA8807F110031146184635
S31508028BD0F9F754FF034687F8373097F83730002BF2
S31508028BE006D0FA8897F83730B9681846FAF77AFB42
S31508028BF000BF3837BD4680BD80B58EB000AFF8607D
S31508028C00B9601346FB80002387F83730FB683B615F
S31508028C10FEF7F6FA0346002B03D04FF080437B613A
S31508028C2001E000237B610023BB61FB88FB61002313
S31508028C303B624FF480137B624FF40013BB6200233E
S31508028C40FB6200233B63FA8807F1100311461846B4
S31508028C50F9F7AEFF034687F8373097F83730002B17
S31508028C6006D0FA8897F83730B9681846FAF77AFBC1
S31508028C7000BF3837BD4680BD80B59CB000AF78606E
S31508028C80084611461A460346FB700B46BB70134646
S31508028C907B707B68FB64FEF7B3FA0346002B03D0AE
S31508028CA04FF080433B6501E000233B6500237B656B
S31508028CB00323BB650023FB654FF480133B664FF421
S31508028CC000137B660023BB660023FB6630233B73D7
S31508028CD03B7B5AB297F9033003F00F035BB2134397
S31508028CE05BB2DBB23B73BB787B737B78BB7308489A
S31508028CF005F05EFCF8F708FA07F10C0207F14C03D7
S31508028D001946FAF7A7FC00BF7037BD4680BD00BFFB
S31508028D10A40E040880B59CB000AF786008461146D8
S31508028D201A460346FB700B46BB7013467B707B687C
S31508028D30FB64FEF765FA0346002B03D04FF0804327
S31508028D403B6501E000233B6500237B650323BB6586
S31508028D500023FB654FF480133B664FF400137B66D2
S31508028D600023BB660023FB6630233B733B7B5AB268
S31508028D7097F9033003F00F035BB213435BB2DBB21E
S31508028D803B73BB787B737B78BB73F8F7BDF907F146
S31508028D900C0207F14C031946FAF75CFC00BF703760
S31508028DA0BD4680BD80B59CB000AF786008461146C6
S31508028DB01A460346FB700B46BB7013467B707B68EC
S31508028DC0FB64FEF71DFA0346002B03D04FF08043DF
S31508028DD03B6501E000233B6500237B650323BB65F6
S31508028DE00023FB654FF480133B664FF400137B6642
S31508028DF00023BB660023FB6630233B733B7B5AB2D8
S31508028E0097F9033003F00F035BB213435BB2DBB28D
S31508028E103B73BB787B737B78BB73F8F775F907F1FD
S31508028E200C0207F14C031946FAF714FC00BF703717
S31508028E30BD4680BD80B59CB000AF78600846114635
S31508028E401A460346FB700B46BB7013467B707B685B
S31508028E50FB64FEF7D5F90346002B03D04FF0804397
S31508028E603B6501E000233B6500237B650323BB6565
S31508028E700023FB654FF480133B664FF400137B66B1
S31508028E800023BB660023FB6630233B733B7B5AB247
S31508028E9097F9033003F00F035BB213435BB2DBB2FD
S31508028EA03B73BB787B737B78BB73F8F72DF907F1B5
S31508028EB00C0207F14C031946FAF7CCFB00BF7037D0
S31508028EC0BD4680BD80B59CB000AF786008461146A5
S31508028ED01A460346FB700B46BB7013467B707B68CB
S31508028EE0FB64FEF78DF90346002B03D04FF080434F
S31508028EF03B6501E000233B6500237B650323BB65D5
S31508028F000023FB654FF480133B664FF400137B6620
S31508028F100023BB660023FB6630233B733B7B5AB2B6
S31508028F2097F9033003F00F035BB213435BB2DBB26C
S31508028F303B73BB787B737B78BB73F8F7E5F807F16D
S31508028F400C0207F14C031946FAF784FB00BF703787
S31508028F50BD4680BD80B59CB000AF78600846114614
S31508028F601A460346FB700B46BB7013467B707B683A
S31508028F70FB64FEF745F90346002B03D04FF0804306
S31508028F803B6501E000233B6500237B650323BB6544
S31508028F900023FB654FF480133B664FF400137B6690
S31508028FA00023BB660023FB6630233B733B7B5AB226
S31508028FB097F9033003F00F035BB213435BB2DBB2DC
S31508028FC03B73BB787B737B78BB73F8F79DF807F125
S31508028FD00C0207F14C031946FAF73CFB00BF70373F
S31508028FE0BD4680BD80B59CB000AF78600846114684
S31508028FF01A460346FB700B46BB7013467B707B68AA
S31508029000FB64FEF7FDF80346002B03D04FF08043BE
S315080290103B6501E000233B6500237B650323BB65B3
S315080290200023FB654FF480133B664FF400137B66FF
S315080290300023BB660023FB6630233B733B7B5AB295
S3150802904097F9033003F00F035BB213435BB2DBB24B
S315080290503B73BB787B737B78BB73F8F755F807F1DC
S315080290600C0207F14C031946FAF7F4FA00BF7037F7
S31508029070BD4680BD80B582B000AF7860002300226D
S3150802908000217868FFF7F8FD00BF0837BD4680BDA6
S3150802909080B582B000AF786000230022002178688C
S315080290A0FFF738FE00BF0837BD4680BD80B582B0DF
S315080290B000AF78600023002200217868FFF772FE6D
S315080290C000BF0837BD4680BD80B582B000AF786064
S315080290D00023002200217868FFF7ACFE00BF08379C
S315080290E0BD4680BD80B582B000AF786000230022FD
S315080290F000217868FFF7E6FE00BF0837BD4680BD47
S3150802910080B582B000AF786000230022002178681B
S31508029110FFF720FF00BF0837BD4680BD80B582B085
S3150802912000AF78600023002200217868FFF75AFF13
S3150802913000BF0837BD4680BD80B582B000AF7860F3
S315080291400023002200217868FFF796FD00BF083742
S31508029150BD4680BD80B582B000AF7860002300228C
S3150802916000217868FFF788FD00BF0837BD4680BD35
S3150802917080B582B000AF78600023002200217868AB
S31508029180FFF77AFD00BF0837BD4680BD80B582B0BD
S3150802919000AF78600023002200217868FFF76CFD93
S315080291A000BF0837BD4680BD80B582B000AF786083
S315080291B00023002200217868FFF75EFD00BF08370A
S315080291C0BD4680BD80B582B000AF7860002300221C
S315080291D000217868FFF750FD00BF0837BD4680BDFD
S315080291E080B582B000AF786000230022002178683B
S315080291F0FFF742FD00BF0837BD4680BD80B586B081
S3150802920000AFF860B9601346FB80FB687B61FB68B8
S31508029210B3F5007F06D1FB881A46B968786900F06B
S3150802922093F88DE0FB68B3F5806F06D1FB881A4682
S31508029230B968786900F0A3F882E0FB68B3F5006FB5
S3150802924006D1FB881A46B968786900F0B3F877E060
S31508029250FB68B3F5805F06D1FB881A46B968786958
S3150802926000F0C3F86CE0FB68B3F5005F06D1FB8833
S315080292701A46B968786900F0D3F861E0FB68B3F575
S31508029280804F06D1FB881A46B968786900F0E3F878
S3150802929056E0FB68B3F5004F06D1FB881A46B96853
S315080292A0786900F0F3F84BE0FB68B3F5803F06D126
S315080292B0FB881A46B968786900F003F940E0FB684A
S315080292C0B3F5003F06D1FB881A46B968786900F0FB
S315080292D013F935E0FB68B3F5802F06D1FB881A46E9
S315080292E0B968786900F023F92AE0FB68B3F5002F1C
S315080292F006D1FB881A46B968786900F033F91FE087
S31508029300FB68B3F5801F06D1FB881A46B9687869E7
S3150802931000F043F914E0FB68B3F5001F06D1FB8899
S315080293201A46B968786900F053F909E0FB68B3F59B
S31508029330800F05D1FB881A46B968786900F063F987
S3150802934000BF1837BD4680BD80B584B000AFF8604F
S31508029350B9601346FB80FB883E2B06D8FB881A4663
S31508029360B968F868FEF7ECF905E0FB881A46B968A9
S31508029370F868FFF701F900BF1037BD4680BD80B512
S3150802938084B000AFF860B9601346FB80FB883E2BB9
S3150802939006D8FB881A46B968F868FEF753FA05E054
S315080293A0FB881A46B968F868FFF726F900BF10372E
S315080293B0BD4680BD80B584B000AFF860B96013467B
S315080293C0FB80FB883E2B06D8FB881A46B968F868E4
S315080293D0FEF7BAFA05E0FB881A46B968F868FFF795
S315080293E04BF900BF1037BD4680BD80B584B000AFCB
S315080293F0F860B9601346FB80FB883E2B06D8FB88CB
S315080294001A46B968F868FEF721FB05E0FB881A4692
S31508029410B968F868FFF770F900BF1037BD4680BD16
S3150802942080B584B000AFF860B9601346FB80FB884C
S315080294303E2B06D8FB881A46B968F868FEF788FBF9
S3150802944005E0FB881A46B968F868FFF795F900BF80
S315080294501037BD4680BD80B584B000AFF860B960EC
S315080294601346FB80FB883E2B06D8FB881A46B9684A
S31508029470F868FEF7EFFB05E0FB881A46B968F86854
S31508029480FFF7BAF900BF1037BD4680BD80B584B074
S3150802949000AFF860B9601346FB80FB883E2B06D8FE
S315080294A0FB881A46B968F868FEF756FC05E0FB8899
S315080294B01A46B968F868FFF7DFF900BF1037BD46E4
S315080294C080BD80B584B000AFF860B9601346FB80F2
S315080294D0FB883E2B06D8FB881A46B968F868FEF759
S315080294E0BDFC05E0FB881A46B968F868FFF704FA76
S315080294F000BF1037BD4680BD80B584B000AFF860A6
S31508029500B9601346FB80FB883E2B06D8FB881A46B1
S31508029510B968F868FEF724FD05E0FB881A46B968BB
S31508029520F868FFF729FA00BF1037BD4680BD80B537
S3150802953084B000AFF860B9601346FB80FB883E2B07
S3150802954006D8FB881A46B968F868FEF78BFD05E067
S31508029550FB881A46B968F868FFF74EFA00BF103753
S31508029560BD4680BD80B584B000AFF860B9601346C9
S31508029570FB80FB883E2B06D8FB881A46B968F86832
S31508029580FEF7F2FD05E0FB881A46B968F868FFF7A8
S3150802959073FA00BF1037BD4680BD80B584B000AFF0
S315080295A0F860B9601346FB80FB883E2B06D8FB8819
S315080295B01A46B968F868FEF759FE05E0FB881A46A6
S315080295C0B968F868FFF798FA00BF1037BD4680BD3C
S315080295D080B584B000AFF860B9601346FB80FB889B
S315080295E03E2B06D8FB881A46B968F868FEF7C0FE0D
S315080295F005E0FB881A46B968F868FFF7BDFA00BFA6
S315080296001037BD4680BD80B584B000AFF860B9603A
S315080296101346FB80FB883E2B06D8FB881A46B96898
S31508029620F868FEF727FF05E0FB881A46B968F86866
S31508029630FFF7E2FA00BF1037BD4680BD80B588B095
S3150802964000AF78600023FB83FF23FB7500233B6191
S315080296500023BB610023FB817B68BB60BB6893F870
S3150802966028301B09FB75BB681B683B613B6940F2E6
S315080296700112934202D14FF40073BB61FB7D032BA7
S3150802968000F2D68001A252F823F000BF9D96020886
S31508029690FB9602085F970208C7970208BB6893F809
S315080296A0283003F00F039AB2634B1A80624B1B8869
S315080296B01B029AB2604B1A80BB6893F829301A4685
S315080296C05D4B1B8813439AB25B4B1A800223FB83BA
S315080296D00CE005F0D7FBFB8BBA68134493F82830E5
S315080296E0194612F029FBFB8B0133FB83FA8B524B8B
S315080296F01B8801339A42ECDD9AE0BB6893F828305E
S3150802970003F00F039AB24C4B1A804B4B1B881B0271
S315080297109AB2494B1A80BB6893F829301A46464BC7
S315080297201B8813439AB2444B1A80444B01221A707F
S315080297300223FB830CE005F0A5FBFB8BBA681344F6
S3150802974093F82830194612F0F7FAFB8B0133FB839C
S31508029750FB8B3F2BEFD9B869FFF78CFC68E0374BD8
S315080297601B781A46BB6893F8283003F00F039A420F
S315080297705BD1BB68DB681846F8F74AF80346013B33
S31508029780FB810123FB830CE005F07CFBFB8BBA68AB
S31508029790134493F82830194612F0CEFAFB8B01339C
S315080297A0FB83FA8BFB899A42EED9244B1B78013349
S315080297B0DAB2224B1A70214B1B780F2B35D91F4B65
S315080297C000221A7031E01E4BD3F8C432BA699A42A3
S315080297D00FD1BB6893F8283003F00F03DAB2184B9F
S315080297E083F8EE22BB6893F82920154B83F8EF22FB
S315080297F01DE0134B03F58053D3F8D432BA699A4263
S3150802980015D1BB6893F8283003F00F03DAB20C4B74
S3150802981003F5805383F8FE22BB6893F82920084B88
S3150802982003F5805383F8FF2201E000BF00E000BF82
S3150802983000BF2037BD4680BD58DF01205ADF012010
S315080298408084002080B588B000AF78600023FB834F
S31508029850FF23FB7500233B610023BB610023FB81C9
S315080298607B68BB60BB6893F828301B09FB75BB682D
S315080298701B683B613B69B3F5817F02D14FF4806374
S31508029880BB61FB7D032B00F2D58001A252F823F0BF
S31508029890A1980208FF98020863990208CB99020860
S315080298A0BB6893F8283003F00F039AB2634B1A8009
S315080298B0624B1B881B029AB2604B1A80BB6893F8EC
S315080298C029301A465D4B1B8813439AB25B4B1A80A2
S315080298D00223FB830CE005F043FBFB8BBA681344B7
S315080298E093F82830194612F027FAFB8B0133FB83CB
S315080298F0FA8B524B1B8801339A42ECDD9AE0BB681D
S3150802990093F8283003F00F039AB24C4B1A804B4B4C
S315080299101B881B029AB2494B1A80BB6893F82930F6
S315080299201A46464B1B8813439AB2444B1A80444B39
S3150802993001221A700223FB830CE005F011FBFB8B54
S31508029940BA68134493F82830194612F0F5F9FB8BD6
S315080299500133FB83FB8B3F2BEFD9B869FFF798FBE3
S3150802996068E0374B1B781A46BB6893F8283003F031
S315080299700F039A425BD1BB68DB681846F7F748FFC4
S315080299800346013BFB810123FB830CE005F0E8FA61
S31508029990FB8BBA68134493F82830194612F0CCF9AF
S315080299A0FB8B0133FB83FA8BFB899A42EED9244B54
S315080299B01B780133DAB2224B1A70214B1B780F2B14
S315080299C035D91F4B00221A7031E01E4BD3F8C43228
S315080299D0BA699A420FD1BB6893F8283003F00F038D
S315080299E0DAB2184B83F8EE22BB6893F82920154B96
S315080299F083F8EF221DE0134B03F58053D3F8D432D4
S31508029A00BA699A4215D1BB6893F8283003F00F0356
S31508029A10DAB20C4B03F5805383F8FE22BB6893F83F
S31508029A202920084B03F5805383F8FF2201E000BF83
S31508029A3000E000BF00BF2037BD4680BD5CDF0120C5
S31508029A405EDF01208498002080B588B000AF786078
S31508029A500023FB83FF23FB7500233B610023BB61C5
S31508029A600023FB817B68BB60BB6893F828301B091F
S31508029A70FB75BB681B683B613B6940F20312934264
S31508029A8002D14FF40063BB61FB7D032B00F2D68043
S31508029A9001A252F823F000BFA99A0208079B0208FE
S31508029AA06B9B0208D39B0208BB6893F8283003F025
S31508029AB00F039AB2634B1A80624B1B881B029AB237
S31508029AC0604B1A80BB6893F829301A465D4B1B888F
S31508029AD013439AB25B4B1A800223FB830CE0FDF711
S31508029AE09BFBFB8BBA68134493F82830194612F08D
S31508029AF023F9FB8B0133FB83FA8B524B1B88013309
S31508029B009A42ECDD9AE0BB6893F8283003F00F031B
S31508029B109AB24C4B1A804B4B1B881B029AB2494B82
S31508029B201A80BB6893F829301A46464B1B8813439A
S31508029B309AB2444B1A80444B01221A700223FB83C1
S31508029B400CE0FDF769FBFB8BBA68134493F82830DF
S31508029B50194612F0F1F8FB8B0133FB83FB8B3F2B83
S31508029B60EFD9B869FFF7A2FA68E0374B1B781A46AD
S31508029B70BB6893F8283003F00F039A425BD1BB689F
S31508029B80DB681846F7F744FE0346013BFB810123CF
S31508029B90FB830CE0FDF740FBFB8BBA68134493F892
S31508029BA02830194612F0C8F8FB8B0133FB83FA8B6F
S31508029BB0FB899A42EED9244B1B780133DAB2224B3F
S31508029BC01A70214B1B780F2B35D91F4B00221A709E
S31508029BD031E01E4BD3F8C432BA699A420FD1BB6838
S31508029BE093F8283003F00F03DAB2184B83F8EE2203
S31508029BF0BB6893F82920154B83F8EF221DE0134B17
S31508029C0003F58053D3F8D432BA699A4215D1BB68A0
S31508029C1093F8283003F00F03DAB20C4B03F580539E
S31508029C2083F8FE22BB6893F82920084B03F5805374
S31508029C3083F8FF2201E000BF00E000BF00BF203723
S31508029C40BD4680BD60DF012062DF012088AC0020AE
S31508029C5080B588B000AF78600023FB83FF23FB75CD
S31508029C6000233B610023BB610023FB817B68BB6049
S31508029C70BB6893F828301B09FB75BB681B683B61F8
S31508029C803B69B3F5827F02D14FF48053BB61FB7DFA
S31508029C90032B00F2D58001A252F823F0AD9C0208EC
S31508029CA00B9D02086F9D0208D79D0208BB6893F8B0
S31508029CB0283003F00F039AB2634B1A80624B1B8853
S31508029CC01B029AB2604B1A80BB6893F829301A466F
S31508029CD05D4B1B8813439AB25B4B1A800223FB83A4
S31508029CE00CE001F0F9FDFB8BBA68134493F82830AF
S31508029CF0194612F021F8FB8B0133FB83FA8B524B80
S31508029D001B8801339A42ECDD9AE0BB6893F8283047
S31508029D1003F00F039AB24C4B1A804B4B1B881B025B
S31508029D209AB2494B1A80BB6893F829301A46464BB1
S31508029D301B8813439AB2444B1A80444B01221A7069
S31508029D400223FB830CE001F0C7FDFB8BBA681344C0
S31508029D5093F82830194611F0EFFFFB8B0133FB838A
S31508029D60FB8B3F2BEFD9B869FFF7AEF968E0374BA3
S31508029D701B781A46BB6893F8283003F00F039A42F9
S31508029D805BD1BB68DB681846F7F742FD0346013B21
S31508029D90FB810123FB830CE001F09EFDFB8BBA6875
S31508029DA0134493F82830194611F0C6FFFB8B01338A
S31508029DB0FB83FA8BFB899A42EED9244B1B78013333
S31508029DC0DAB2224B1A70214B1B780F2B35D91F4B4F
S31508029DD000221A7031E01E4BD3F8C432BA699A428D
S31508029DE00FD1BB6893F8283003F00F03DAB2184B89
S31508029DF083F8EE22BB6893F82920154B83F8EF22E5
S31508029E001DE0134B03F58053D3F8D432BA699A424C
S31508029E1015D1BB6893F8283003F00F03DAB20C4B5E
S31508029E2003F5805383F8FE22BB6893F82920084B72
S31508029E3003F5805383F8FF2201E000BF00E000BF6C
S31508029E4000BF2037BD4680BD64DF012066DF0120E2
S31508029E508CC0002080B588B000AF78600023FB83F1
S31508029E60FF23FB7500233B610023BB610023FB81B3
S31508029E707B68BB60BB6893F828301B09FB75BB6817
S31508029E801B683B613B6940F20512934202D14FF4CB
S31508029E900053BB61FB7D032B00F2D68001A252F868
S31508029EA023F000BFB59E0208139F0208779F020897
S31508029EB0DF9F0208BB6893F8283003F00F039AB2B3
S31508029EC0634B1A80624B1B881B029AB2604B1A803C
S31508029ED0BB6893F829301A465D4B1B8813439AB21E
S31508029EE05B4B1A800223FB830CE0FDF7DFFAFB8B40
S31508029EF0BA68134493F82830194611F01DFFFB8BF4
S31508029F000133FB83FA8B524B1B8801339A42ECDDF1
S31508029F109AE0BB6893F8283003F00F039AB24C4BC9
S31508029F201A804B4B1B881B029AB2494B1A80BB6894
S31508029F3093F829301A46464B1B8813439AB2444B68
S31508029F401A80444B01221A700223FB830CE0FDF7A8
S31508029F50ADFAFB8BBA68134493F82830194611F008
S31508029F60EBFEFB8B0133FB83FB8B3F2BEFD9B869E7
S31508029F70FFF7B8F868E0374B1B781A46BB6893F8C0
S31508029F80283003F00F039A425BD1BB68DB68184698
S31508029F90F7F73EFC0346013BFB810123FB830CE0FA
S31508029FA0FDF784FAFB8BBA68134493F828301946EE
S31508029FB011F0C2FEFB8B0133FB83FA8BFB899A42B3
S31508029FC0EED9244B1B780133DAB2224B1A70214B95
S31508029FD01B780F2B35D91F4B00221A7031E01E4B06
S31508029FE0D3F8C432BA699A420FD1BB6893F82830BB
S31508029FF003F00F03DAB2184B83F8EE22BB6893F824
S3150802A0002920154B83F8EF221DE0134B03F58053E5
S3150802A010D3F8D432BA699A4215D1BB6893F8283074
S3150802A02003F00F03DAB20C4B03F5805383F8FE22D2
S3150802A030BB6893F82920084B03F5805383F8FF225F
S3150802A04001E000BF00E000BF00BF2037BD4680BD6B
S3150802A05068DF01206ADF012090D4002080B588B02D
S3150802A06000AF78600023FB83FF23FB7500233B6167
S3150802A0700023BB610023FB817B68BB60BB6893F846
S3150802A08028301B09FB75BB681B683B613B69B3F546
S3150802A090837F02D14FF48043BB61FB7D032B00F221
S3150802A0A0D58001A252F823F0B9A0020817A1020826
S3150802A0B07BA10208E3A10208BB6893F8283003F0E3
S3150802A0C00F039AB2634B1A80624B1B881B029AB221
S3150802A0D0604B1A80BB6893F829301A465D4B1B8879
S3150802A0E013439AB25B4B1A800223FB830CE0F6F702
S3150802A0F09DFFFB8BBA68134493F82830194611F072
S3150802A1001BFEFB8B0133FB83FA8B524B1B880133F5
S3150802A1109A42ECDD9AE0BB6893F8283003F00F0305
S3150802A1209AB24C4B1A804B4B1B881B029AB2494B6C
S3150802A1301A80BB6893F829301A46464B1B88134384
S3150802A1409AB2444B1A80444B01221A700223FB83AB
S3150802A1500CE0F6F76BFFFB8BBA68134493F82830CA
S3150802A160194611F0E9FDFB8B0133FB83FB8B3F2B71
S3150802A170EFD9B869FEF7C4FF68E0374B1B781A4671
S3150802A180BB6893F8283003F00F039A425BD1BB6889
S3150802A190DB681846F7F73CFB0346013BFB810123C4
S3150802A1A0FB830CE0F6F742FFFB8BBA68134493F87D
S3150802A1B02830194611F0C0FDFB8B0133FB83FA8B5D
S3150802A1C0FB899A42EED9244B1B780133DAB2224B29
S3150802A1D01A70214B1B780F2B35D91F4B00221A7088
S3150802A1E031E01E4BD3F8C432BA699A420FD1BB6822
S3150802A1F093F8283003F00F03DAB2184B83F8EE22ED
S3150802A200BB6893F82920154B83F8EF221DE0134B00
S3150802A21003F58053D3F8D432BA699A4215D1BB688A
S3150802A22093F8283003F00F03DAB20C4B03F5805388
S3150802A23083F8FE22BB6893F82920084B03F580535E
S3150802A24083F8FF2201E000BF00E000BF00BF20370D
S3150802A250BD4680BD6CDF01206EDF012094E8002038
S3150802A26080B588B000AF78600023FB83FF23FB75B7
S3150802A27000233B610023BB610023FB817B68BB6033
S3150802A280BB6893F828301B09FB75BB681B683B61E2
S3150802A2903B6940F20712934202D14FF40043BB6175
S3150802A2A0FB7D032B00F2D68001A252F823F000BFF1
S3150802A2B0C1A202081FA3020883A30208EBA302088D
S3150802A2C0BB6893F8283003F00F039AB2634B1A80DF
S3150802A2D0624B1B881B029AB2604B1A80BB6893F8C2
S3150802A2E029301A465D4B1B8813439AB25B4B1A8078
S3150802A2F00223FB830CE001F05DFBFB8BBA68134477
S3150802A30093F82830194611F017FDFB8B0133FB83AE
S3150802A310FA8B524B1B8801339A42ECDD9AE0BB68F2
S3150802A32093F8283003F00F039AB24C4B1A804B4B22
S3150802A3301B881B029AB2494B1A80BB6893F82930CC
S3150802A3401A46464B1B8813439AB2444B1A80444B0F
S3150802A35001221A700223FB830CE001F02BFBFB8B14
S3150802A360BA68134493F82830194611F0E5FCFB8BBA
S3150802A3700133FB83FB8B3F2BEFD9B869FEF7CEFE81
S3150802A38068E0374B1B781A46BB6893F8283003F007
S3150802A3900F039A425BD1BB68DB681846F7F738FAAF
S3150802A3A00346013BFB810123FB830CE001F002FB20
S3150802A3B0FB8BBA68134493F82830194611F0BCFC93
S3150802A3C0FB8B0133FB83FA8BFB899A42EED9244B2A
S3150802A3D01B780133DAB2224B1A70214B1B780F2BEA
S3150802A3E035D91F4B00221A7031E01E4BD3F8C432FE
S3150802A3F0BA699A420FD1BB6893F8283003F00F0363
S3150802A400DAB2184B83F8EE22BB6893F82920154B6B
S3150802A41083F8EF221DE0134B03F58053D3F8D432A9
S3150802A420BA699A4215D1BB6893F8283003F00F032C
S3150802A430DAB20C4B03F5805383F8FE22BB6893F815
S3150802A4402920084B03F5805383F8FF2201E000BF59
S3150802A45000E000BF00BF2037BD4680BD70DF012087
S3150802A46072DF012098FC002080B588B000AF7860C2
S3150802A4700023FB83FF23FB7500233B610023BB619B
S3150802A4800023FB817B68BB60BB6893F828301B09F5
S3150802A490FB75BB681B683B613B69B3F5847F02D1D8
S3150802A4A04FF48033BB61FB7D032B00F2FA8001A2D5
S3150802A4B052F823F0C5A4020823A50208ABA5020890
S3150802A4C039A60208BB6893F8283003F00F039AB23C
S3150802A4D0794B1A80784B1B881B029AB2764B1A80E4
S3150802A4E0BB6893F829301A46734B1B8813439AB2F2
S3150802A4F0714B1A800223FB830CE0FCF7FBFEFB8BF5
S3150802A500BA68134493F82830194611F015FCFB8BE8
S3150802A5100133FB83FA8B684B1B8801339A42ECDDC5
S3150802A520C6E0BB6893F8283003F00F039AB2624B71
S3150802A5301A80614B1B881B029AB25F4B1A80BB6852
S3150802A54093F829301A465C4B1B8813439AB25A4B26
S3150802A5501A805A4B01221A70594804F029F8594BA5
S3150802A5601B78002B04D0584804F022F8FCF71CFF8D
S3150802A5700223FB830CE0FCF7BDFEFB8BBA6813448F
S3150802A58093F82830194611F0D7FBFB8B0133FB836E
S3150802A590FB8B3F2BEFD94D4804F00AF8B869FEF752
S3150802A5A0CBFD484B01221A7082E0464B00221A70F4
S3150802A5B0424B1B781A46BB6893F8283003F00F0300
S3150802A5C09A4232D13D4B1B781946414803F0F0FFB7
S3150802A5D0BB68DB681846F7F71BF90346013BFB81A4
S3150802A5E00123FB830CE0FCF785FEFB8BBA68134458
S3150802A5F093F82830194611F09FFBFB8B0133FB8336
S3150802A600FA8BFB899A42EED9304803F0D1FF2B4BDD
S3150802A6101B780133DAB2294B1A70284B1B780F2B99
S3150802A62043D9264B00221A703FE0244B1B78194661
S3150802A630274803F0BDFF38E0264BD3F8C432BA697F
S3150802A6409A4212D1BB6893F8283003F00F03DAB2A4
S3150802A650204B83F8EE22BB6893F829201D4B83F81A
S3150802A660EF221D4803F0A4FF21E01A4B03F580539D
S3150802A670D3F8D432BA699A4219D1BB6893F828300A
S3150802A68003F00F03DAB2134B03F5805383F8FE2265
S3150802A690BB6893F829200F4B03F5805383F8FF22F2
S3150802A6A005E00E4803F084FF02E000BF00E000BFA9
S3150802A6B000BF2037BD4680BD74DF012076DF01204A
S3150802A6C0B00E040877DF0120BC0E0408C80E040881
S3150802A6D0CC0E04089C100120D80E0408E00E0408CB
S3150802A6E080B588B000AF78600023FB83FF23FB7533
S3150802A6F000233B610023BB610023FB817B68BB60AF
S3150802A700BB6893F828301B09FB75BB681B683B615D
S3150802A7103B6940F20912934202D14FF40033BB61FE
S3150802A720FB7D032B00F2D68001A252F823F000BF6C
S3150802A73041A702089FA7020803A802086BA80208F5
S3150802A740BB6893F8283003F00F039AB2634B1A805A
S3150802A750624B1B881B029AB2604B1A80BB6893F83D
S3150802A76029301A465D4B1B8813439AB25B4B1A80F3
S3150802A7700223FB830CE0FCF72BFEFB8BBA6813441F
S3150802A78093F82830194611F0D7FAFB8B0133FB836D
S3150802A790FA8B524B1B8801339A42ECDD9AE0BB686E
S3150802A7A093F8283003F00F039AB24C4B1A804B4B9E
S3150802A7B01B881B029AB2494B1A80BB6893F8293048
S3150802A7C01A46464B1B8813439AB2444B1A80444B8B
S3150802A7D001221A700223FB830CE0FCF7F9FDFB8BBE
S3150802A7E0BA68134493F82830194611F0A5FAFB8B78
S3150802A7F00133FB83FB8B3F2BEFD9B869FEF7AAFC23
S3150802A80068E0374B1B781A46BB6893F8283003F082
S3150802A8100F039A425BD1BB68DB681846F6F7F8FF66
S3150802A8200346013BFB810123FB830CE0FCF7D0FDC9
S3150802A830FB8BBA68134493F82830194611F07CFA50
S3150802A840FB8B0133FB83FA8BFB899A42EED9244BA5
S3150802A8501B780133DAB2224B1A70214B1B780F2B65
S3150802A86035D91F4B00221A7031E01E4BD3F8C43279
S3150802A870BA699A420FD1BB6893F8283003F00F03DE
S3150802A880DAB2184B83F8EE22BB6893F82920154BE7
S3150802A89083F8EF221DE0134B03F58053D3F8D43225
S3150802A8A0BA699A4215D1BB6893F8283003F00F03A8
S3150802A8B0DAB20C4B03F5805383F8FE22BB6893F891
S3150802A8C02920084B03F5805383F8FF2201E000BFD5
S3150802A8D000E000BF00BF2037BD4680BD78DF0120FB
S3150802A8E07ADF0120A024012080B588B000AF786005
S3150802A8F00023FB83FF23FB7500233B610023BB6117
S3150802A9000023FB817B68BB60BB6893F828301B0970
S3150802A910FB75BB681B683B613B69B3F5857F02D152
S3150802A9204FF48023BB61FB7D032B00F2D58001A285
S3150802A93052F823F045A90208A3A9020807AA0208A1
S3150802A9406FAA0208BB6893F8283003F00F039AB27D
S3150802A950634B1A80624B1B881B029AB2604B1A80A1
S3150802A960BB6893F829301A465D4B1B8813439AB283
S3150802A9705B4B1A800223FB830CE0FCF705FEFB8B7C
S3150802A980BA68134493F82830194611F0D5F9FB8BA7
S3150802A9900133FB83FA8B524B1B8801339A42ECDD57
S3150802A9A09AE0BB6893F8283003F00F039AB24C4B2F
S3150802A9B01A804B4B1B881B029AB2494B1A80BB68FA
S3150802A9C093F829301A46464B1B8813439AB2444BCE
S3150802A9D01A80444B01221A700223FB830CE0FCF70F
S3150802A9E0D3FDFB8BBA68134493F82830194611F045
S3150802A9F0A3F9FB8B0133FB83FB8B3F2BEFD9B8699A
S3150802AA00FEF7B6FB68E0374B1B781A46BB6893F825
S3150802AA10283003F00F039A425BD1BB68DB681846FD
S3150802AA20F6F7F6FE0346013BFB810123FB830CE0A6
S3150802AA30FCF7AAFDFB8BBA68134493F8283019462B
S3150802AA4011F07AF9FB8B0133FB83FA8BFB899A4265
S3150802AA50EED9244B1B780133DAB2224B1A70214BFA
S3150802AA601B780F2B35D91F4B00221A7031E01E4B6B
S3150802AA70D3F8C432BA699A420FD1BB6893F8283020
S3150802AA8003F00F03DAB2184B83F8EE22BB6893F889
S3150802AA902920154B83F8EF221DE0134B03F580534B
S3150802AAA0D3F8D432BA699A4215D1BB6893F82830DA
S3150802AAB003F00F03DAB20C4B03F5805383F8FE2238
S3150802AAC0BB6893F82920084B03F5805383F8FF22C5
S3150802AAD001E000BF00E000BF00BF2037BD4680BDD1
S3150802AAE07CDF01207EDF0120A438012080B588B0F2
S3150802AAF000AF78600023FB83FF23FB7500233B61CD
S3150802AB000023BB610023FB817B68BB60BB6893F8AB
S3150802AB1028301B09FB75BB681B683B613B6940F221
S3150802AB200B12934202D14FF40023BB61FB7D032B28
S3150802AB3000F2D68001A252F823F000BF4DAB0208FC
S3150802AB40ABAB02080FAC020877AC0208BB6893F8F5
S3150802AB50283003F00F039AB2634B1A80624B1B88A4
S3150802AB601B029AB2604B1A80BB6893F829301A46C0
S3150802AB705D4B1B8813439AB25B4B1A800223FB83F5
S3150802AB800CE0FCF76FFDFB8BBA68134493F8283088
S3150802AB90194611F0D1F8FB8B0133FB83FA8B524B22
S3150802ABA01B8801339A42ECDD9AE0BB6893F8283099
S3150802ABB003F00F039AB24C4B1A804B4B1B881B02AD
S3150802ABC09AB2494B1A80BB6893F829301A46464B03
S3150802ABD01B8813439AB2444B1A80444B01221A70BB
S3150802ABE00223FB830CE0FCF73DFDFB8BBA6813449A
S3150802ABF093F82830194611F09FF8FB8B0133FB8333
S3150802AC00FB8B3F2BEFD9B869FEF7C0FA68E0374BE2
S3150802AC101B781A46BB6893F8283003F00F039A424A
S3150802AC205BD1BB68DB681846F6F7F2FD0346013BC3
S3150802AC30FB810123FB830CE0FCF714FDFB8BBA684E
S3150802AC40134493F82830194611F076F8FB8B013332
S3150802AC50FB83FA8BFB899A42EED9244B1B78013384
S3150802AC60DAB2224B1A70214B1B780F2B35D91F4BA0
S3150802AC7000221A7031E01E4BD3F8C432BA699A42DE
S3150802AC800FD1BB6893F8283003F00F03DAB2184BDA
S3150802AC9083F8EE22BB6893F82920154B83F8EF2236
S3150802ACA01DE0134B03F58053D3F8D432BA699A429E
S3150802ACB015D1BB6893F8283003F00F03DAB20C4BB0
S3150802ACC003F5805383F8FE22BB6893F82920084BC4
S3150802ACD003F5805383F8FF2201E000BF00E000BFBE
S3150802ACE000BF2037BD4680BD80DF012082DF0120FC
S3150802ACF0A84C012080B588B000AF78600023FB839A
S3150802AD00FF23FB7500233B610023BB610023FB8104
S3150802AD107B68BB60BB6893F828301B09FB75BB6868
S3150802AD201B683B613B69B3F5867F02D14FF48013FA
S3150802AD30BB61FB7D032B00F2D58001A252F823F0FA
S3150802AD4051AD0208AFAD020813AE02087BAE020887
S3150802AD50BB6893F8283003F00F039AB2634B1A8044
S3150802AD60624B1B881B029AB2604B1A80BB6893F827
S3150802AD7029301A465D4B1B8813439AB25B4B1A80DD
S3150802AD800223FB830CE000F0BDFAFB8BBA6813447E
S3150802AD9093F82830194610F0CFFFFB8B0133FB835B
S3150802ADA0FA8B524B1B8801339A42ECDD9AE0BB6858
S3150802ADB093F8283003F00F039AB24C4B1A804B4B88
S3150802ADC01B881B029AB2494B1A80BB6893F8293032
S3150802ADD01A46464B1B8813439AB2444B1A80444B75
S3150802ADE001221A700223FB830CE000F08BFAFB8B1C
S3150802ADF0BA68134493F82830194610F09DFFFB8B66
S3150802AE000133FB83FB8B3F2BEFD9B869FEF7CCF9ED
S3150802AE1068E0374B1B781A46BB6893F8283003F06C
S3150802AE200F039A425BD1BB68DB681846F6F7F0FC5B
S3150802AE300346013BFB810123FB830CE000F062FA27
S3150802AE40FB8BBA68134493F82830194610F074FF3E
S3150802AE50FB8B0133FB83FA8BFB899A42EED9244B8F
S3150802AE601B780133DAB2224B1A70214B1B780F2B4F
S3150802AE7035D91F4B00221A7031E01E4BD3F8C43263
S3150802AE80BA699A420FD1BB6893F8283003F00F03C8
S3150802AE90DAB2184B83F8EE22BB6893F82920154BD1
S3150802AEA083F8EF221DE0134B03F58053D3F8D4320F
S3150802AEB0BA699A4215D1BB6893F8283003F00F0392
S3150802AEC0DAB20C4B03F5805383F8FE22BB6893F87B
S3150802AED02920084B03F5805383F8FF2201E000BFBF
S3150802AEE000E000BF00BF2037BD4680BD84DF0120D9
S3150802AEF086DF0120AC60012080B588B000AF78609B
S3150802AF000023FB83FF23FB7500233B610023BB6100
S3150802AF100023FB817B68BB60BB6893F828301B095A
S3150802AF20FB75BB681B683B613B6940F20D12934295
S3150802AF3002D14FF40013BB61FB7D032B00F2D680CE
S3150802AF4001A252F823F000BF59AF0208B7AF0208B0
S3150802AF501BB0020883B00208BB6893F8283003F0D6
S3150802AF600F039AB2634B1A80624B1B881B029AB272
S3150802AF70604B1A80BB6893F829301A465D4B1B88CA
S3150802AF8013439AB25B4B1A800223FB830CE000F050
S3150802AF90C7FBFB8BBA68134493F82830194610F09E
S3150802AFA0CBFEFB8B0133FB83FA8B524B1B88013397
S3150802AFB09A42ECDD9AE0BB6893F8283003F00F0357
S3150802AFC09AB24C4B1A804B4B1B881B029AB2494BBE
S3150802AFD01A80BB6893F829301A46464B1B881343D6
S3150802AFE09AB2444B1A80444B01221A700223FB83FD
S3150802AFF00CE000F095FBFB8BBA68134493F82830F3
S3150802B000194610F099FEFB8B0133FB83FB8B3F2B12
S3150802B010EFD9B869FEF7D6F868E0374B1B781A46B7
S3150802B020BB6893F8283003F00F039A425BD1BB68DA
S3150802B030DB681846F6F7ECFB0346013BFB81012366
S3150802B040FB830CE000F06CFBFB8BBA68134493F8A5
S3150802B0502830194610F070FEFB8B0133FB83FA8BFE
S3150802B060FB899A42EED9244B1B780133DAB2224B7A
S3150802B0701A70214B1B780F2B35D91F4B00221A70D9
S3150802B08031E01E4BD3F8C432BA699A420FD1BB6873
S3150802B09093F8283003F00F03DAB2184B83F8EE223E
S3150802B0A0BB6893F82920154B83F8EF221DE0134B52
S3150802B0B003F58053D3F8D432BA699A4215D1BB68DC
S3150802B0C093F8283003F00F03DAB20C4B03F58053DA
S3150802B0D083F8FE22BB6893F82920084B03F58053B0
S3150802B0E083F8FF2201E000BF00E000BF00BF20375F
S3150802B0F0BD4680BD88DF01208ADF0120B0740120A9
S3150802B10080B588B000AF78600023FB83FF23FB7508
S3150802B11000233B610023BB610023FB817B68BB6084
S3150802B120BB6893F828301B09FB75BB681B683B6133
S3150802B1303B69B3F5877F02D14FF48003BB61FB7D80
S3150802B140032B00F2D58001A252F823F05DB1020862
S3150802B150BBB102081FB2020887B20208BB6893F89D
S3150802B160283003F00F039AB2634B1A80624B1B888E
S3150802B1701B029AB2604B1A80BB6893F829301A46AA
S3150802B1805D4B1B8813439AB25B4B1A800223FB83DF
S3150802B1900CE000F033FBFB8BBA68134493F82830B3
S3150802B1A0194610F0C9FDFB8B0133FB83FA8B524B10
S3150802B1B01B8801339A42ECDD9AE0BB6893F8283083
S3150802B1C003F00F039AB24C4B1A804B4B1B881B0297
S3150802B1D09AB2494B1A80BB6893F829301A46464BED
S3150802B1E01B8813439AB2444B1A80444B01221A70A5
S3150802B1F00223FB830CE000F001FBFB8BBA681344C5
S3150802B20093F82830194610F097FDFB8B0133FB8320
S3150802B210FB8B3F2BEFD9B869FDF7E2FF68E0374BA6
S3150802B2201B781A46BB6893F8283003F00F039A4234
S3150802B2305BD1BB68DB681846F6F7EAFA0346013BB8
S3150802B240FB810123FB830CE000F0D8FAFB8BBA687A
S3150802B250134493F82830194610F06EFDFB8B013320
S3150802B260FB83FA8BFB899A42EED9244B1B7801336E
S3150802B270DAB2224B1A70214B1B780F2B35D91F4B8A
S3150802B28000221A7031E01E4BD3F8C432BA699A42C8
S3150802B2900FD1BB6893F8283003F00F03DAB2184BC4
S3150802B2A083F8EE22BB6893F82920154B83F8EF2220
S3150802B2B01DE0134B03F58053D3F8D432BA699A4288
S3150802B2C015D1BB6893F8283003F00F03DAB20C4B9A
S3150802B2D003F5805383F8FE22BB6893F82920084BAE
S3150802B2E003F5805383F8FF2201E000BF00E000BFA8
S3150802B2F000BF2037BD4680BD8CDF01208EDF0120CE
S3150802B300B488012080B400AF024B1846BD465DF8EA
S3150802B310047B7047ACDF012080B582B000AF78604D
S3150802B3200B467B807B881A4679684FF48010FDF7B6
S3150802B33065FF00BF0837BD4680BD000090B589B0DD
S3150802B34002AFF860B9601346FB800C2000F058F88B
S3150802B35003460133DBB23B75CE237B75D623BB7519
S3150802B3603B7D1946BB681B781A46FB880A4803F0D8
S3150802B3701FF902F0D1FC044602F0C4FC014607F1AB
S3150802B3801402FB880093BB68204610F060FC00BFDD
S3150802B39000BF1C37BD4690BDF40E040880B500AF49
S3150802B3A04FF480720249034800F072FB00BF80BD69
S3150802B3B0F8E8012090DF012080B500AFFFF7EEFF25
S3150802B3C0034B044A0449054810F08DF800BF80BDB6
S3150802B3D019B302083DB30208ACDF0120A0DF012041
S3150802B3E080B483B000AF0346FB71FB79034AD35C92
S3150802B3F018460C37BD465DF8047B704704000020EA
S3150802B40080B485B000AF0346FB710023FB730023AB
S3150802B410FB730AE0FB7B0A4AD35CFA799A4201D1AA
S3150802B420FB7B06E0FB7B0133FB73FB7B142BF1D919
S3150802B430FF2318461437BD465DF8047B704700BFE4
S3150802B4400400002080B400AF034B1B781846BD46A3
S3150802B4505DF8047B704700BF3100002080B584B0D8
S3150802B46000AF0346FB710023FB730023FB730DE059
S3150802B470FB7B1B4AD35CFA799A4204D1FB7B194AB5
S3150802B4807821D15428E0FB7B0133FB73FB7B142B19
S3150802B490EED90023FB731CE0FB7B114AD35CFF2B1E
S3150802B4A014D1FB7B0E49FA79CA540F4B1B78013328
S3150802B4B0DAB20D4B1A70FB7BFA7919460B4803F080
S3150802B4C077F8FB7B074A7821D15405E0FB7B0133E9
S3150802B4D0FB73FB7B142BDFD91037BD4680BD00BF3B
S3150802B4E0040000201C00002031000020240F04085C
S3150802B4F080B582B000AF0023FB710123FB7119E00E
S3150802B500FB791846FFF76CFF0346FF2B0FD0FB7932
S3150802B5100C4AD25C013AD1B20A4AD154FB79094A99
S3150802B520D35C002B03D1FB79074AFF21D154FB795F
S3150802B5300133FB71FB79142BE2D900BF00BF083730
S3150802B540BD4680BD1C0000200400002080B582B0E4
S3150802B55000AF0346FB711E220021514812F09EF8E5
S3150802B560FB790E2B00F2968001A252F823F000BF57
S3150802B570ADB50208B9B50208C1B50208CDB50208CB
S3150802B580DDB50208EDB50208FDB5020813B60208D4
S3150802B59025B6020831B602083DB6020853B60208B5
S3150802B5A069B6020875B6020885B602083C4B3D4ADA
S3150802B5B007CA83E807006EE0394B3B4A1A606AE01D
S3150802B5C0374B3A4A07CA03C31A7064E0344B384AFF
S3150802B5D092E803001860043319805CE0304B354A60
S3150802B5E092E8030018600433198054E02C4B324A5F
S3150802B5F092E803001860043319704CE0284B2F4A6E
S3150802B60092E8030018600433198002330A0C1A7090
S3150802B61041E0234B2A4A1268114619800233120C5A
S3150802B6201A7038E01E4B274A07CA03C31A7032E05B
S3150802B6301B4B254A07CA03C31A702CE0184B234A28
S3150802B64092E8030018600433198002330A0C1A7050
S3150802B65021E0134B1E4A92E803001860043319804E
S3150802B66002330A0C1A7016E00D4B1A4A07CA83E807
S3150802B670070010E00A4B184A92E8030018600433E0
S3150802B680197008E0064B154A92E80300186004335D
S3150802B690197000E000BF024B18460837BD4680BD48
S3150802B6A0F8E90120340F040849434500400F04080D
S3150802B6B04C0F0408540F04085C0F0408640F0408AE
S3150802B6C06C0F0408700F04087C0F0408880F04081E
S3150802B6D0900F0408980F0408A40F0408AC0F040876
S3150802B6E080B584B000AF78607B68FB600023BB60DE
S3150802B6F0FB681B68BB60BB68B3F5807F0BD1FB6830
S3150802B70093F82830002B06D1FB6893F8293018469F
S3150802B710FFF7A4FE00BF00BF1037BD4680BD00007C
S3150802B72080B400AF024B1846BD465DF8047B7047ED
S3150802B73034EA012080B582B000AF78600B467B8080
S3150802B7407B881A4679684FF40010FDF757FD00BF4B
S3150802B7500837BD4680BD000090B589B002AFF860D3
S3150802B760B9601346FB800D20FFF74AFE03460133F4
S3150802B770DBB23B75CE237B75D623BB753B7D19465B
S3150802B780BB681B781A460B4802F012FF02F0C4FA8D
S3150802B790044602F0B7FA014607F11402FB88009341
S3150802B7A0BB68204610F053FA00BF00BF1C37BD46DF
S3150802B7B090BD00BFB40F040880B500AF4FF4807285
S3150802B7C00249034800F064F900BF80BD80F30120F6
S3150802B7D018EA012080B500AFFFF7EEFF034B044AD3
S3150802B7E0044905480FF07FFE00BF80BD35B7020841
S3150802B7F059B7020834EA012028EA012080B400AFCA
S3150802B800024B1846BD465DF8047B70479CF401203E
S3150802B81080B582B000AF78600B467B807B881A467B
S3150802B82079684FF48000FDF7E9FC00BF0837BD468A
S3150802B83080BD000090B589B002AFF860B9601346C2
S3150802B840FB800E20FFF7DCFD03460133DBB23B75B6
S3150802B850CE237B75D623BB753B7D1946BB681B7801
S3150802B8601A460B4802F0A4FE02F056FA044602F003
S3150802B87049FA014607F11402FB880093BB68204681
S3150802B88010F0E5F900BF00BF1C37BD4690BD00BFEA
S3150802B890DC0F040880B500AF4FF4807202490348F2
S3150802B8A000F0F6F800BF80BDE8FD012080F4012013
S3150802B8B080B500AFFFF7EEFF034B044A044905487B
S3150802B8C00FF011FE00BF80BD11B8020835B8020894
S3150802B8D09CF4012090F4012080B400AF024B184674
S3150802B8E0BD465DF8047B704704FF012080B582B02F
S3150802B8F000AF78600B467B807B881A4679684FF4DE
S3150802B9008050FDF77BFC00BF0837BD4680BD0000AE
S3150802B91090B589B002AFF860B9601346FB80032080
S3150802B920FFF76EFD03460133DBB23B75CE237B750B
S3150802B930D623BB753B7D1946BB681B781A460B484E
S3150802B94002F036FE02F0E8F9044602F0DBF9014697
S3150802B95007F11402FB880093BB68204610F077F9BA
S3150802B96000BF00BF1C37BD4690BD00BF04100408C7
S3150802B97080B500AF4FF480720249034800F088F898
S3150802B98000BF80BD50080220E8FE012080B500AF46
S3150802B990FFF7EEFF034B044A044905480FF0A3FDDF
S3150802B9A000BF80BDEDB8020811B9020804FF0120E4
S3150802B9B0F8FE012080B400AF024B1846BD465DF87A
S3150802B9C0047B70476C09022080B582B000AF7860AC
S3150802B9D00B467B807B881A4679684FF40040FDF750
S3150802B9E00DFC00BF0837BD4680BD000090B589B082
S3150802B9F002AFF860B9601346FB800720FFF700FD27
S3150802BA0003460133DBB23B75CE237B75D623BB7562
S3150802BA103B7D1946BB681B781A460B4802F0C8FDDF
S3150802BA2002F07AF9044602F06DF9014607F11402AA
S3150802BA30FB880093BB68204610F009F900BF00BFD7
S3150802BA401C37BD4690BD00BF2C10040880B500AF58
S3150802BA504FF480720249034800F01AF800BF80BD0D
S3150802BA60B81202205009022080B500AFFFF7EEFF98
S3150802BA70034B044A044905480FF035FD00BF80BD53
S3150802BA80C9B90208EDB902086C0902206009022048
S3150802BA9080B485B000AFF860B9607A60FB68002BA5
S3150802BAA002D14FF0FF3319E0FB68BA681A60FB68E7
S3150802BAB01B68002B02D14FF0FF330FE0FB681A68B0
S3150802BAC07B68013B1A44FB685A60FB681A68FB6884
S3150802BAD09A60FB689A68FB68DA600023184614378E
S3150802BAE0BD465DF8047B704780B485B000AF7860C8
S3150802BAF07B68002B03D07B681B68002B01D10023CF
S3150802BB001FE07B68DA687B689B689A420CD37B687D
S3150802BB105A687B68DB68D21A7B6899687B681B68F7
S3150802BB20CB1A1344FB6005E07B689A687B68DB687E
S3150802BB30D31AFB60FB68002B02D0FB68013BFB6053
S3150802BB40FB6818461437BD465DF8047B704780B417
S3150802BB5083B000AF78607B68002B03D07B681B68D4
S3150802BB60002B02D14FF0FF3316E07B68DA687B6858
S3150802BB709B689A4205D37B68DA687B689B68D31A06
S3150802BB800AE07B685A687B689B68D21A7B68D96820
S3150802BB907B681B68CB1A134418460C37BD465DF8FA
S3150802BBA0047B704780B483B000AF78607B68002B53
S3150802BBB003D07B681B68002B01D1012308E07B6850
S3150802BBC09A687B68DB689A420CBF01230023DBB2C2
S3150802BBD018460C37BD465DF8047B704780B586B0BB
S3150802BBE000AFF860B9607A60FB68002B03D0FB6887
S3150802BBF01B68002B01D1002327E07B687B61F8686C
S3150802BC00FFF772FF02467B69934201D900231CE0C3
S3150802BC10FB68DB683B610FE0BA68531CBB603B6993
S3150802BC20591C396112781A70FB685B683A699A423C
S3150802BC3002D1FB681B683B617B695A1E7A61002B3D
S3150802BC40EAD1FB683A69DA607B6818461837BD4656
S3150802BC5080BD80B586B000AFF860B9607A60FB68CF
S3150802BC60002B03D0FB681B68002B01D100232DE0B3
S3150802BC70F868FFF76CFF78617A697B689A4202D99D
S3150802BC807B687B6105E07A687B699A4201D97B69A0
S3150802BC907B60FB689B683B610FE03A69531C3B611A
S3150802BCA0BB68591CB96012781A70FB685B683A69F6
S3150802BCB09A4202D1FB681B683B617B695A1E7A610C
S3150802BCC0002BEAD1FB683A699A607B6818461837EE
S3150802BCD0BD4680BD90B5ADF2FC5D00AF044607F5E2
S3150802BCE0BF60A0F5BE60016007F5BF61A1F2F4511D
S3150802BCF00A6007F5BF62A2F5BF62136007F5BF6364
S3150802BD00A3F2E95322461A7007F5BF63A3F5BE6389
S3150802BD101B68002B07D007F5BF63A3F5BE631B6834
S3150802BD201B68002B01D10023C2E007F5BF63A3F20B
S3150802BD30E9531B78002B11D107F5BF63A3F5BE6340
S3150802BD401868FFF7D1FE024607F5BF63A3F5BF637E
S3150802BD501B6802339A4226D80023A9E007F5BF6377
S3150802BD60A3F5BE631868FFF7BFFE024607F5BF6371
S3150802BD70A3F5BF631B6802339A420DD8012387F8DD
S3150802BD80EF3507F1100207F5BF63A3F5BE63114647
S3150802BD90186800F0A3F802E0002387F8EF3597F851
S3150802BDA0EF35012BDAD007F5BF63A3F5BE631B682F
S3150802BDB0DB68C7F8F035D7F8F0355A1CC7F8F0250E
S3150802BDC007F5BF62A2F5BF621268D2B21A7007F50A
S3150802BDD0BF63A3F5BE631B685B68D7F8F0259A4272
S3150802BDE007D107F5BF63A3F5BE631B681B68C7F8CF
S3150802BDF0F03507F5BF63A3F5BF631B68190AD7F8C1
S3150802BE00F0355A1CC7F8F025CAB21A7007F5BF638F
S3150802BE10A3F5BE631B685B68D7F8F0259A4207D17B
S3150802BE2007F5BF63A3F5BE631B681B68C7F8F03541
S3150802BE3007F5BF63A3F5BF631B68C7F8F43523E0AC
S3150802BE4007F5BF63A3F2F4531A6807F5BF63A3F2B3
S3150802BE50F453511C1960D7F8F035591CC7F8F01578
S3150802BE6012781A7007F5BF63A3F5BE631B685B6891
S3150802BE70D7F8F0259A4207D107F5BF63A3F5BE6343
S3150802BE801B681B68C7F8F035D7F8F4355A1EC7F889
S3150802BE90F425002BD4D107F5BF63A3F5BE631B684F
S3150802BEA0D7F8F025DA6007F5BF63A3F5BF631B6809
S3150802BEB0184607F2FC57BD4690BD80B584B000AF60
S3150802BEC0F860B9607A607B68BA68F9680020FFF79B
S3150802BED001FF034618461037BD4680BD80B586B0B9
S3150802BEE000AF786039607B68002B03D07B681B68DB
S3150802BEF0002B01D1002353E07B689A687B68DB68D4
S3150802BF009A4201D100234BE07B689B683B613B69FF
S3150802BF105A1C3A611B787B617B685B683A699A426C
S3150802BF2002D17B681B683B613B695A1C3A611B78E4
S3150802BF301B027A6913437B617B685B683A699A429A
S3150802BF4002D17B681B683B617B69FB607868FFF7F7
S3150802BF50FEFD0246FB68934219D97B681A687B681C
S3150802BF609A607B689A687B68DA60002318E03A6907
S3150802BF70531C3B613B68591C396012781A707B68FE
S3150802BF805B683A699A4202D17B681B683B617B69A6
S3150802BF905A1E7A61002BEAD17B683A699A60FB6875
S3150802BFA018461837BD4680BD80B483B000AF7860A6
S3150802BFB07B681B68B3F1804F02D10C4B01221A70C1
S3150802BFC07B681B680A4A934202D10A4B01221A70FD
S3150802BFD07B681B68084A934202D1084B01221A70F1
S3150802BFE000BF0C37BD465DF8047B7047B8130220C4
S3150802BFF000040040BA13022000080040BB130220C6
S3150802C00080B500AF05480BF09FFF05480BF09CFF73
S3150802C01004480BF099FF00BF80BD00BF4C140220F4
S3150802C02098140220E414022090B593B000AF474B4F
S3150802C030D3F8F430002B09DA454802F0B9FA07F1C9
S3150802C04044030621184610F0C4F85DE03F4BD3F8C6
S3150802C050F43003F08043002B09D03E4802F0A8FAD8
S3150802C06007F144030521184610F0B3F84CE0374BA4
S3150802C070D3F8F43003F00053002B09D0364802F007
S3150802C08097FA07F144030421184610F0A2F83BE098
S3150802C0902E4BD3F8F43003F08053002B09D02F48E7
S3150802C0A002F086FA07F144030321184610F091F8C4
S3150802C0B02AE0264BD3F8F43003F00063002B09D0AC
S3150802C0C0274802F075FA07F144030221184610F0D0
S3150802C0D080F819E01D4BD3F8F43003F08063002B87
S3150802C0E009D0204802F064FA07F1440301211846F0
S3150802C0F010F06FF808E01C4802F05AFA07F14403F8
S3150802C1000021184610F065F8104BD3F8F4300F4AA0
S3150802C11043F40003C2F8F4303A4607F144031146E1
S3150802C120184610F004F93B46184610F0CDF80446B6
S3150802C1303B46184610F0D4F803461A4621464A20CA
S3150802C140F7F74CFA00BF4C37BD4690BD000C0244C7
S3150802C150501004086C10040888100408A410040877
S3150802C160C4100408DC100408F410040890B583B05F
S3150802C17000AF0023FB710023BB71134802F018FAC3
S3150802C1800023FB7116E0FB791846FFF729F90346E7
S3150802C190BB71BB79FF2B0AD0FC79BB791846FFF72E
S3150802C1A0D5F903461A462146084802F001FAFB79F0
S3150802C1B00133FB71FB79142BE5D9054802F0F8F92E
S3150802C1C000BF0C37BD4690BD101104083C11040887
S3150802C1D044110408B0B5ADF5047D00AF804B1B7859
S3150802C1E0002B00F09E807E4B00221A70FAF754FB51
S3150802C1F0F7F7A0FBF9F744FEFAF776FBF7F7EAFC3E
S3150802C200F9F778FEFAF798FBF7F734FEF9F7ACFE7A
S3150802C210FAF7BAFBF7F77EFFF9F7E0FEFAF7DCFB67
S3150802C220F8F7C8F8F9F714FFFAF7FEFBF8F712FA67
S3150802C230F9F748FFFAF720FCF8F75CFBF9F77CFFF9
S3150802C240FAF742FCF8F7A6FCF9F7B0FFFAF764FC2E
S3150802C250F8F7FAFDF9F7EAFFFAF786FCF8F744FF6A
S3150802C260FAF71EF8FAF7A8FCF9F78EF8FAF752F871
S3150802C270FAF7CAFCF9F7D8F9FAF786F8FAF7ECFCEE
S3150802C280F9F722FBFAF7BAF8FAF70EFDF9F76CFC9A
S3150802C290FAF7EEF8F9F7CAFDFAF72EFD514B1B78B5
S3150802C2A0002B3ED007F50473A3F504744E4B2046C3
S3150802C2B019466C231A4611F08EFA04F16C03002211
S3150802C2C01A605A609A60DA601A616023C7F8043203
S3150802C2D007F5027300221A609A80444B1B78012BD9
S3150802C2E007D102F03DFE3B466B2219460FF00CFEC3
S3150802C2F011E03E4B1B780A2B0DD902F031FE07F5E9
S3150802C3000173012219460FF0FFFD364B00221A70FF
S3150802C310364B00221A70354B1B780133DAB2334B8F
S3150802C3201A70334B1B78002B20D0314B00221A701F
S3150802C33001F0AEFC02F046F802F0A2F802F04AFA60
S3150802C34002F088F902F0D8FA02F064FB294B1B883E
S3150802C35001339AB2274B1A80264B1B88042B05D920
S3150802C360244B00221A80244B01221A70224B1B7876
S3150802C370002B02D0204B00221A70204B1B78002B70
S3150802C38012D01E4B00221A701D4B1B8801339AB21B
S3150802C3901B4B1A801A4B1B88092B05D9184B0022EE
S3150802C3A01A80184B01221A70164B1B78002B61D083
S3150802C3B0144B00221A70144B1B68002B04D0124B24
S3150802C3C01B680133104A1360FFF792F800F02CF944
S3150802C3D00346002B1CD00D4802F0EAF81AE000BF0B
S3150802C3E0BB130220D013022090110408D113022095
S3150802C3F0B8130220C0130220B9130220BA1302206E
S3150802C400C2130220BC130220CC13022070110408A6
S3150802C41000F0F4F8404B1B8801339AB23E4B1A805F
S3150802C4203D4B1B88012B05D93B4B00221A803B4BFF
S3150802C43001221A703A4B1B8801339AB2384B1A807A
S3150802C440374B1B88092B05D9354B00221A80354BE9
S3150802C45001221A70344B1B8801339AB2324B1A8066
S3150802C460314B1B881D2B05D92F4B00221A802F4BC7
S3150802C47001221A70294B1B78002B15D0274B002254
S3150802C4801A7001212A4805F089FC0220FEF7B8FF36
S3150802C4900346FF2B08D0274B1B78002B04D1254BCC
S3150802C4A001221A70FFF7C0FD1E4B1B78002B24D001
S3150802C4B01C4B00221A700FF073FA0346002B05D1A3
S3150802C4C001F016FC034618460FF091F93B46194649
S3150802C4D019480EF0C2FF01F00BFC04463B4618460B
S3150802C4E00EF088FF05463B4618460EF08FFF0346B8
S3150802C4F01A462946204600F035FD0C4B1B78002BC0
S3150802C50004D00A4B00221A70FFF730FE00BF07F567
S3150802C5100477BD46B0BD00BFC6130220BE13022073
S3150802C520C4130220BD130220C8130220BF1302201F
S3150802C53000140242CA1302208011040880B400AF14
S3150802C54000BFBD465DF8047B704780B400AF00BFEC
S3150802C550BD465DF8047B704780B500AF064802F019
S3150802C56027F806480CF076FD04480CF0DDFC034873
S3150802C5700CF048FB00BF80BD10120408EC1602201E
S3150802C58080B500AF00F0A4FB02F082F900BF80BDBF
S3150802C59080B500AF02480CF035FB00BF80BD00BF76
S3150802C5A08017022080B500AF00F046FB02F0D0F8F3
S3150802C5B000BF80BD80B500AF02480CF023FB00BF68
S3150802C5C080BD00BF3015022080B500AF00F034FBF5
S3150802C5D002F0EEF900BF80BD80B500AF02480CF04C
S3150802C5E011FB00BF80BD00BFC415022080B500AF95
S3150802C5F000F022FB02F08CFA00BF80BD80B500AFC6
S3150802C600024805F06DFC00BF80BD00BF3814022049
S3150802C61080B400AF034B01221A7000BFBD465DF815
S3150802C620047B7047C818022080B400AF034B1B78FE
S3150802C6301846BD465DF8047B704700BFC81802203D
S3150802C64080B500AF384B394A9A6062B600BF02F02D
S3150802C6501FFD00F071F800F0D3FB00F01FF900F09F
S3150802C660D5F800F03BF900F05BF900F04DFA00F05E
S3150802C67097FA00F0E1FA00F02BFB00F075FB00F0E8
S3150802C68057F900F0A3F900F0F1F9FFF7B9FC01F048
S3150802C6907FFF01F067FE02F0FBF802F0D3FB02F01F
S3150802C6A057F802F0B7FC02F083F902F045FC02F0F3
S3150802C6B02FFAFAF755FFFAF709FEFFF767F9F4F7C3
S3150802C6C00FFDFFF7D1F9FAF76FFEFAF7DBFEFAF775
S3150802C6D0B5FFFBF721F8FEF76FFEFFF77BF8FFF7CA
S3150802C6E0E7F8D6200FF068F91148FAF72DFBFAF7A2
S3150802C6F087FD0346002B07D04FF480726FF0604126
S3150802C7000220FAF783FC06E04FF480724FF6FF71B7
S3150802C7100220FAF74FFCFAF7A3FC0621054801F0B6
S3150802C72015FFFFF757FDFCE700ED00E000000208E1
S3150802C730D41302202812040880B59CB000AF07F172
S3150802C740200350220021184610F0A8FF07F108031B
S3150802C75000221A605A609A60DA601A615A612A4B94
S3150802C7601B69294A43F030031361274B1B6903F0FF
S3150802C77030037B607B6800BF234B5B6903F00803C9
S3150802C780082BF9D109233B624FF480337B624FF0C1
S3150802C7908063BB630223BB640323FB6403233B65F9
S3150802C7A07D237B650223BB650223FB6502233B6669
S3150802C7B008237B660023BB660023FB6607F120037A
S3150802C7C0184605F09DFB0346002B01D000F0C4FB7A
S3150802C7D01F23BB600323FB6000233B6100237B61AD
S3150802C7E00023BB610023FB6107F1080305211846F4
S3150802C7F005F0BEFF0346002B01D000F0ADFB00BFDB
S3150802C8007037BD4680BD00BF0008024480B500AF40
S3150802C810204B214A1A601F4B00225A601D4B4FF4C7
S3150802C82040729A601B4B0022DA601A4B00221A7475
S3150802C830184B00225A74174B00229A74154B05227C
S3150802C8405A61144B0A229A61124B2722DA61114B5A
S3150802C8500A221A620F4B05225A620E4B02229A626A
S3150802C8600C4B0722DA620B4B02221A63094B01228E
S3150802C8705A63084B01229A63064B0022DA6305487B
S3150802C88004F00CF90346002B01D000F065FB00BF4B
S3150802C89080BD00BFD413022000A4004080B582B038
S3150802C8A000AF0D4BD3F888300B4A43F00103C2F8A8
S3150802C8B08830094BD3F8883003F001037B607B6824
S3150802C8C0002200211B2002F05EFD1B2002F075FDEE
S3150802C8D000BF0837BD4680BD000C024480B500AFD4
S3150802C8E00D4B0E4A1A600C4B05225A600A4B40F24F
S3150802C8F0EE22DA60084B40F2EE229A60064B0022DC
S3150802C9001A61054805F064FA0346002B01D000F0C7
S3150802C91023FB00BF80BD00BF381402200030004050
S3150802C92080B400AF00BFBD465DF8047B70470000C7
S3150802C93080B588B000AF07F1100300221A605A606A
S3150802C9409A60DA603B1D00221A605A609A601E4B92
S3150802C9504FF080421A601C4B4CF24F325A601A4B07
S3150802C96000229A60184B3122DA60174B00221A61AC
S3150802C970154B00229A6114480BF08EFA0346002BD7
S3150802C98001D000F0E9FA4FF480533B6107F1100336
S3150802C99019460D480BF0D0FC0346002B01D000F0D7
S3150802C9A0DBFA00237B600023FB603B1D1946064821
S3150802C9B00BF0C2FF0346002B01D000F0CDFA00BFF0
S3150802C9C02037BD4680BD00BF4C14022080B588B012
S3150802C9D000AF07F1100300221A605A609A60DA6003
S3150802C9E03B1D00221A605A609A601E4B1E4A1A6044
S3150802C9F01C4B4CF24F325A601A4B00229A60194B62
S3150802CA0040F2F312DA60174B00221A61154B002224
S3150802CA109A6114480BF040FA0346002B01D000F045
S3150802CA209BFA4FF480533B6107F1100319460D48F0
S3150802CA300BF082FC0346002B01D000F08DFA00238E
S3150802CA407B600023FB603B1D194606480BF074FF0A
S3150802CA500346002B01D000F07FFA00BF2037BD46FF
S3150802CA6080BD00BF981402200004004080B588B03B
S3150802CA7000AF07F1100300221A605A609A60DA6062
S3150802CA803B1D00221A605A609A601D4B1D4A1A60A5
S3150802CA901B4B4CF24F325A60194B00229A60184BC4
S3150802CAA00422DA60164B00221A61154B00229A619B
S3150802CAB013480BF0F1F90346002B01D000F04CFAAB
S3150802CAC04FF480533B6107F1100319460C480BF0EB
S3150802CAD033FC0346002B01D000F03EFA00237B60AC
S3150802CAE00023FB603B1D194605480BF025FF03464C
S3150802CAF0002B01D000F030FA00BF2037BD4680BDBA
S3150802CB00E41402200008004080B500AF224B234AF5
S3150802CB101A60214B4FF4E1325A601F4B00229A6089
S3150802CB201D4B0022DA601C4B00221A611A4B0C229A
S3150802CB305A61194B00229A61174B0022DA61164B89
S3150802CB4000221A62144B00225A62134B00229A627E
S3150802CB5011480CF007F80346002B01D000F0FCF947
S3150802CB6000210D480EF07BFB0346002B01D000F096
S3150802CB70F3F9002108480EF0B0FB0346002B01D05A
S3150802CB8000F0EAF904480EF031FB0346002B01D007
S3150802CB9000F0E2F900BF80BD30150220004C0040CB
S3150802CBA080B500AF224B234A1A60214B4FF4E1327B
S3150802CBB05A601F4B00229A601D4B0022DA601C4BFA
S3150802CBC000221A611A4B0C225A61194B00229A61E9
S3150802CBD0174B0022DA61164B00221A62144B002206
S3150802CBE05A62134B00229A6211480BF0BBFF0346A6
S3150802CBF0002B01D000F0B0F900210D480EF02FFBF2
S3150802CC000346002B01D000F0A7F9002108480EF0D0
S3150802CC1064FB0346002B01D000F09EF904480EF08F
S3150802CC20E5FA0346002B01D000F096F900BF80BD55
S3150802CC30C41502200050004080B500AF224B234A9B
S3150802CC401A60214B4FF4E1325A601F4B00229A6058
S3150802CC501D4B0022DA601C4B00221A611A4B0C2269
S3150802CC605A61194B00229A61174B0022DA61164B58
S3150802CC7000221A62144B00225A62134B00229A624D
S3150802CC8011480BF06FFF0346002B01D000F064F940
S3150802CC9000210D480EF0E3FA0346002B01D000F0FE
S3150802CCA05BF9002108480EF018FB0346002B01D059
S3150802CCB000F052F904480EF099FA0346002B01D007
S3150802CCC000F04AF900BF80BD58160220003801401C
S3150802CCD080B500AF224B234A1A60214B4FF4E1324A
S3150802CCE05A601F4B00229A601D4B0022DA601C4BC9
S3150802CCF000221A611A4B0C225A61194B00229A61B8
S3150802CD00174B0022DA61164B00221A62144B0022D4
S3150802CD105A62134B00229A6211480BF023FF03460C
S3150802CD20002B01D000F018F900210D480EF097FAF1
S3150802CD300346002B01D000F00FF9002108480EF037
S3150802CD40CCFA0346002B01D000F006F904480EF08F
S3150802CD504DFA0346002B01D000F0FEF800BF80BD55
S3150802CD60EC1602200044004080B500AF224B234A4D
S3150802CD701A60214B4FF4E1325A601F4B00229A6027
S3150802CD801D4B0022DA601C4B00221A611A4B0C2238
S3150802CD905A61194B00229A61174B0022DA61164B27
S3150802CDA000221A62144B00225A62134B00229A621C
S3150802CDB011480BF0D7FE0346002B01D000F0CCF841
S3150802CDC000210D480EF04BFA0346002B01D000F065
S3150802CDD0C3F8002108480EF080FA0346002B01D05A
S3150802CDE000F0BAF804480EF001FA0346002B01D007
S3150802CDF000F0B2F800BF80BD80170220004800404C
S3150802CE0080B58CB000AF07F11C0300221A605A6085
S3150802CE109A60DA601A614C4BD3F88C304A4A43F06E
S3150802CE202003C2F88C30484BD3F88C3003F0200329
S3150802CE30BB61BB69444BD3F88C30434A43F0800349
S3150802CE40C2F88C30404BD3F88C3003F080037B61F8
S3150802CE507B693D4BD3F88C303B4A43F00403C2F856
S3150802CE608C30394BD3F88C3003F004033B613B69B1
S3150802CE70354BD3F88C30344A43F00103C2F88C3070
S3150802CE80314BD3F88C3003F00103FB60FB682E4B61
S3150802CE90D3F88C302C4A43F00203C2F88C302A4B62
S3150802CEA0D3F88C3003F00203BB60BB68264BD3F879
S3150802CEB08C30254A43F00803C2F88C30224BD3F84B
S3150802CEC08C3003F008037B607B68002201211F482F
S3150802CED004F04CFF00220F211D4804F047FF0122EF
S3150802CEE04FF480611B4804F041FF0123FB610123D3
S3150802CEF03B6200237B620323BB6207F11C031946CC
S3150802CF00124804F025FD0F23FB6101233B6200232F
S3150802CF107B620123BB6207F11C0319460C4804F025
S3150802CF2017FD4FF48063FB6101233B6200237B629A
S3150802CF300123BB6207F11C031946064804F008FDE3
S3150802CF4000BF3037BD4680BD000C024400140242C1
S3150802CF50000802420004024280B400AF72B600BF63
S3150802CF6000BFFDE780B58CB002AFF860B960134622
S3150802CF70FB80FB689B683B62FB685B68FB6100237E
S3150802CF80FB820023FB843B6A03F58063BB610023B3
S3150802CF90FB840CE0FB8CBA6813441A7807F1160373
S3150802CFA01946B8690EF087FAFB8C0133FB84FA8CB2
S3150802CFB0FB889A42EED30EF0C3FC01463B6A03F5A0
S3150802CFC08062FB8A009313460A46396AF8690EF0AC
S3150802CFD03EFE00BF2837BD4680BD80B400AF00BF05
S3150802CFE0BD465DF8047B704780B5CCB000AF07F547
S3150802CFF09873A3F59673186007F58E7300221A6064
S3150802D0005A609A60DA601A6107F59873A3F5907305
S3150802D01018464FF484731A46002110F03FFB07F5B1
S3150802D0209873A3F596731B681B68384A934267D1AF
S3150802D03007F59873A3F590714FF000024FF00403B9
S3150802D040C1E9002307F59873A3F590734FF480722C
S3150802D050C3F8BC2007F11003184605F0CBFE0346B9
S3150802D060002B01D0FFF778FF294BD3F8A030284AC6
S3150802D07043F40073C2F8A030254BD3F8A03003F46A
S3150802D080007207F59873A3F592731A6007F59873F9
S3150802D090A3F592731B681E4BD3F88C301C4A43F0D7
S3150802D0A00103C2F88C301A4BD3F88C3003F0010214
S3150802D0B007F59873A3F594731A6007F59873A3F5A1
S3150802D0C094731B684FF4C053C7F81C310223C7F880
S3150802D0D020310023C7F824310023C7F82831092351
S3150802D0E0C7F82C3107F58E7319460A4804F030FC46
S3150802D0F000220021272002F046F9272002F05DF9D6
S3150802D10000BF07F59877BD4680BD00BF00A4004062
S3150802D110000C02440000024280B586B000AF786077
S3150802D1207B681B68B3F1804F17D12A4BD3F89C3022
S3150802D130284A43F00103C2F89C30264BD3F89C30A8
S3150802D14003F001037B617B69002200212D2002F096
S3150802D1501AF92D2002F031F938E07B681B681E4A5D
S3150802D160934217D11B4BD3F89C301A4A43F0020359
S3150802D170C2F89C30174BD3F89C3003F002033B618C
S3150802D1803B69002200212E2002F0FDF82E2002F033
S3150802D19014F91BE07B681B68104A934216D10D4BA3
S3150802D1A0D3F89C300B4A43F00403C2F89C30094B6F
S3150802D1B0D3F89C3003F00403FB60FB6800220021CD
S3150802D1C02F2002F0E0F82F2002F0F7F800BF1837F8
S3150802D1D0BD4680BD000C0244000400400008004021
S3150802D1E080B5EEB000AF07F5DC73A3F5DA73186005
S3150802D1F007F5D27300221A605A609A60DA601A61D9
S3150802D20007F5DC73A3F5C47318464FF484731A46FC
S3150802D210002110F043FA07F5DC73A3F5DA731B68ED
S3150802D2201B68A54A934266D107F5DC73A3F5C47158
S3150802D2304FF008024FF00003C1E9002307F5DC733B
S3150802D240A3F5C47300229A6607F13003184605F05F
S3150802D250D1FD0346002B01D0FFF77EFE974BD3F88C
S3150802D2609C30964A43F40023C2F89C30934BD3F879
S3150802D2709C3003F4002207F5DC73A3F5C6731A6023
S3150802D28007F5DC73A3F5C6731B688C4BD3F88C3091
S3150802D2908A4A43F00803C2F88C30884BD3F88C309C
S3150802D2A003F0080207F5DC73A3F5C8731A6007F5DD
S3150802D2B0DC73A3F5C8731B684FF4C053C7F8A431CF
S3150802D2C00223C7F8A8310023C7F8AC310323C7F8ED
S3150802D2D0B0310823C7F8B43107F5D273194678482E
S3150802D2E004F036FB002200213D2002F04CF83D20D6
S3150802D2F002F063F84EE207F5DC73A3F5DA731B68EE
S3150802D3001B68704A934266D107F5DC73A3F5C471AC
S3150802D3104FF010024FF00003C1E9002307F5DC7352
S3150802D320A3F5C4730022DA6607F13003184605F03E
S3150802D33061FD0346002B01D0FFF70EFE5F4BD3F8C3
S3150802D3409C305E4A43F48013C2F89C305B4BD3F898
S3150802D3509C3003F4801207F5DC73A3F5CA731A60CE
S3150802D36007F5DC73A3F5CA731B68544BD3F88C30E4
S3150802D370524A43F00203C2F88C30504BD3F88C3031
S3150802D38003F0020207F5DC73A3F5CC731A6007F5FE
S3150802D390DC73A3F5CC731B684FF44053C7F8A4316A
S3150802D3A00223C7F8A8310023C7F8AC310323C7F80C
S3150802D3B0B0310E23C7F8B43107F5D273194642487D
S3150802D3C004F0C6FA002200213E2001F0DCFF3E20CE
S3150802D3D001F0F3FFDEE107F5DC73A3F5DA731B68E8
S3150802D3E01B683A4A934275D107F5DC73A3F5C471F3
S3150802D3F04FF001024FF00003C1E9002307F5DC7381
S3150802D400A3F5C4730022DA6507F13003184605F05E
S3150802D410F1FC0346002B01D0FFF79EFD274BD3F8FC
S3150802D420A430264A43F48043C2F8A430234BD3F8E7
S3150802D430A43003F4804207F5DC73A3F5CE731A60B1
S3150802D44007F5DC73A3F5CE731B681C4BD3F88C3037
S3150802D4501A4A43F00103C2F88C30184BD3F88C30C1
S3150802D46003F0010207F5DC73A3F5D0731A6007F51A
S3150802D470DC73A3F5D0731B684FF4C063C7F8A431F5
S3150802D4800223C7F8A8310023C7F8AC310323C7F82B
S3150802D490B0310723C7F8B43107F5D27319460C48D9
S3150802D4A004F056FA002200213A2001F06CFF3A20D5
S3150802D4B001F083FF6EE100BF004C0040000C0244FD
S3150802D4C0000C0242005000400004024200380140AB
S3150802D4D00000024207F5DC73A3F5DA731B681B68C2
S3150802D4E0AF4A934240F0E78007F5DC73A3F5C471AF
S3150802D4F04FF002024FF00003C1E9002307F5DC737F
S3150802D500A3F5C47300221A6607F13003184605F01C
S3150802D51071FC0346002B01D0FFF71EFDA14BD3F881
S3150802D5209C30A04A43F40033C2F89C309D4BD3F892
S3150802D5309C3003F4003207F5DC73A3F5D2731A6044
S3150802D54007F5DC73A3F5D2731B68964BD3F88C30B8
S3150802D550944A43F00103C2F88C30924BD3F88C30CC
S3150802D56003F0010207F5DC73A3F5D4731A6007F515
S3150802D570DC73A3F5D4731B680C23C7F8A431022302
S3150802D580C7F8A8310023C7F8AC310323C7F8B0316E
S3150802D5900723C7F8B43107F5D2731946824804F04F
S3150802D5A0D7F92123C7F838311723C7F83C310023A6
S3150802D5B0C7F840310023C7F844310023C7F8483179
S3150802D5C04FF40023C7F84C310023C7F85031002323
S3150802D5D0C7F854310123C7F85C310123C7F8603113
S3150802D5E00023C7F864310023C7F868310023C7F857
S3150802D5F06C310023C7F87C310023C7F87031002349
S3150802D600C7F8743107F59C736849184602F084FC1A
S3150802D6100346002B01D0FFF79FFC644A00216448A9
S3150802D62002F090FC0346002B01D0FFF795FC6048F8
S3150802D63002F051FD0346002B01D0FFF78DFC5D4B2E
S3150802D6405D4A1A605B4B00229A635A4B0022DA63E0
S3150802D650584B00221A64574B00225A64554B8122B2
S3150802D6609A64544802F098FA0346002B01D0FFF751
S3150802D67073FC4F494F4802F08FFD0346002B01D039
S3150802D680FFF76AFC07F5DC73A3F5DA731B68494AE8
S3150802D690C3F88020474A07F5DC73A3F5DA731B68DB
S3150802D6A0D3651021434802F016FA0346002B71D0BF
S3150802D6B0FFF752FC6EE007F5DC73A3F5DA731B6815
S3150802D6C01B683E4A934265D107F5DC73A3F5C4711C
S3150802D6D04FF004024FF00003C1E9002307F5DC739B
S3150802D6E0A3F5C47300225A6607F13003184605F0FB
S3150802D6F081FB0346002B01D0FFF72EFC294BD3F8FA
S3150802D7009C30284A43F48023C2F89C30254BD3F830
S3150802D7109C3003F4802207F5DC73A3F5D6731A60EE
S3150802D72007F5DC73A3F5D6731B681E4BD3F88C304A
S3150802D7301C4A43F00803C2F88C301A4BD3F88C30D3
S3150802D74003F0080207F5DC73A3F5D8731A6007F528
S3150802D750DC73A3F5D8731B684FF44073C7F8A4317A
S3150802D7600223C7F8A8310023C7F8AC310323C7F848
S3150802D770B0310723C7F8B43107F5D27319461048F2
S3150802D78004F0E6F8002200213C2001F0FCFD3C20D2
S3150802D79001F013FE00BF07F5DC77BD4680BD00BF6A
S3150802D7A000440040000C0244000002421418022001
S3150802D7B03818022050180220500002400048004043
S3150802D7C0000C024280B582B000AF78607B681B68A5
S3150802D7D0384A934210D1384BD3F89C30364A23F450
S3150802D7E00023C2F89C304FF4C051344804F002FAC0
S3150802D7F03D2001F0F0FD58E07B681B68304A9342F1
S3150802D80010D12D4BD3F89C302B4A23F48013C2F83F
S3150802D8109C304FF440512B4804F0ECF93E2001F0BD
S3150802D820DAFD42E07B681B68274A934210D1224BF5
S3150802D830D3F8A430204A23F48043C2F8A4304FF424
S3150802D840C061224804F0D6F93A2001F0C4FD2CE062
S3150802D8507B681B681E4A934212D1174BD3F89C3039
S3150802D860154A23F40033C2F89C300C21174804F0F9
S3150802D870C1F97B68D3F88030184601F0C7FD14E079
S3150802D8807B681B68134A93420FD10B4BD3F89C3023
S3150802D890094A23F48023C2F89C304FF440710748A2
S3150802D8A004F0A8F93C2001F096FD00BF0837BD46F2
S3150802D8B080BD00BF004C0040000C0244000C02422E
S3150802D8C000500040000402420038014000000242B3
S3150802D8D0004400400048004080B400AF00BFFDE7A6
S3150802D8E080B400AF00BFFDE780B400AF00BFFDE71C
S3150802D8F080B400AF00BFFDE780B400AF00BFFDE70C
S3150802D90080B400AF00BFBD465DF8047B704780B4A3
S3150802D91000AF00BFBD465DF8047B704780B400AF18
S3150802D92000BFBD465DF8047B704780B500AF01F0C5
S3150802D9300BFC00BF80BD000080B500AF024801F0B5
S3150802D94044FF00BF80BD00BF5018022080B500AF5B
S3150802D950024803F091FD00BF80BD00BFD413022028
S3150802D96080B500AF02480AF09DFB00BF80BD00BF2C
S3150802D9704C14022080B500AF02480AF093FB00BFA0
S3150802D98080BD00BF9814022080B500AF02480AF095
S3150802D99089FB00BF80BD00BFE414022080B500AF3A
S3150802D9A002480BF00BFC00BF80BD00BF58160220D0
S3150802D9B080B500AF02480BF001FC00BF80BD00BF76
S3150802D9C08017022080B500AF02480BF0F7FB00BFB4
S3150802D9D080BD00BF3015022080B500AF02480BF0AB
S3150802D9E0EDFB00BF80BD00BFC415022080B400AFA6
S3150802D9F001231846BD465DF8047B704780B582B0A0
S3150802DA0000AF786039600FF0ABFE034616221A6043
S3150802DA104FF0FF3318460837BD4680BD80B582B041
S3150802DA2000AF78604FF0FF317868FFF7E7FF00BF75
S3150802DA30FDE780B586B000AFF860B9607A6000236A
S3150802DA407B610AE0AFF300800146BB685A1CBA60E4
S3150802DA50CAB21A707B6901337B617A697B689A421A
S3150802DA60F0DB7B6818461837BD4680BD80B586B0A0
S3150802DA7000AFF860B9607A6000237B6109E0BB6891
S3150802DA805A1CBA601B781846AFF300807B690133CB
S3150802DA907B617A697B689A42F1DB7B68184618379C
S3150802DAA0BD4680BD80B483B000AF78604FF0FF33C7
S3150802DAB018460C37BD465DF8047B704780B483B0C0
S3150802DAC000AF786039603B684FF400525A60002311
S3150802DAD018460C37BD465DF8047B704780B483B0A0
S3150802DAE000AF7860012318460C37BD465DF8047B03
S3150802DAF0704780B485B000AFF860B9607A600023D9
S3150802DB0018461437BD465DF8047B704780B586B063
S3150802DB1000AF7860144A154BD31A7B617B693B6167
S3150802DB20134B1B68002B02D1114B124A1A60104B79
S3150802DB301A687B6813443A699A4207D20FF010FEB4
S3150802DB4003460C221A604FF0FF3309E0084B1B68A4
S3150802DB50FB60074B1A687B681344054A1360FB6827
S3150802DB6018461837BD4680BD00000A20000400008A
S3150802DB70CC180220D067022080B483B000AF354BA0
S3150802DB80D3F88830334A43F47003C2F88830324BEC
S3150802DB9001221A60304B0022DA612F4B00221A62E8
S3150802DBA02D4B1A682C492D4B13400B602A4B002229
S3150802DBB09A62294B0022DA62274B00221A63264B05
S3150802DBC0274A5A63244B00229A63234B244ADA6370
S3150802DBD0214B00221A64204B214A5A641E4B00220A
S3150802DBE09A641D4B1B681C4A23F4802313601A4B44
S3150802DBF000221A65174B4FF000629A60194B9B690F
S3150802DC0003F060437B607B68B3F1604F03D07B68A7
S3150802DC10B3F1404F17D1134BDB6903F00103002B15
S3150802DC2005D0104B104ADA600E4B104ADA600D4BDB
S3150802DC30DB690C4A43F00203D3610A4BDB69094AE2
S3150802DC4043F00103D36100BF0C37BD465DF8047B80
S3150802DC50704700BF00ED00E0000C0244E3EAE2EA86
S3150802DC6080020101002002403B2A19087F6E5D4CA2
S3150802DC7080B582B000AF7860396039687868FEF797
S3150802DC802DF903469BB218460837BD4680BD0000EB
S3150802DC9080B5A2B000AF0023A7F886303B1D8022CC
S3150802DCA0002118460FF0FAFC1048FDF77BFF0346E1
S3150802DCB083F00103DBB2002B14D03B1D19460B4837
S3150802DCC0FFF7D6FF0346A7F88630B7F88630002B4B
S3150802DCD007D0B7F886203B1D1146184600F036FCD9
S3150802DCE000E000BF8837BD4680BD00BFD0180220BD
S3150802DCF080B400AF024B1846BD465DF8047B7047F8
S3150802DD00F018022080B400AF024B1846BD465DF8F3
S3150802DD10047B7047FC18022080B400AF024B1846F9
S3150802DD20BD465DF8047B70474822022080B582B062
S3150802DD3000AF78600B467B807B881946786800F0CE
S3150802DD4005F800BF0837BD4680BD000080B584B01F
S3150802DD5000AF786039600023FB603B689BB21A46C5
S3150802DD6079680448FEF7A9F80346FB6000BF103736
S3150802DD70BD4680BDE018022090B589B000AFF860B4
S3150802DD80B9601346FB80FB68BB610123FB83BB6852
S3150802DD901A78BB691A70BB685A78BB695A70BB682D
S3150802DDA09A78BB699A70BB691B78002B1BD1BB6931
S3150802DDB05B78002B17D1BB699B78AB2B13D1032356
S3150802DDC0FB830BE0BB699868FB8BBA6813441B7824
S3150802DDD019460DF0B1FFFB8B0133FB83FA8BFB88E7
S3150802DDE09A42EFD336E0BB6801331B7818460DF02A
S3150802DDF0B1FD0346002B07D1BB6801331C78FDF73A
S3150802DE0021FB03469C4213D80323FB830BE0BB6921
S3150802DE109868FB8BBA6813441B7819460DF08CFF79
S3150802DE20FB8B0133FB83FA8BFB889A42EFD311E013
S3150802DE300DF0B6FD0346002B0CD000F05DFF7861AD
S3150802DE40BB68DA1CFB88033B9BB27969B8690DF09B
S3150802DE508DFCFFE700BF2437BD4690BD90B58FB055
S3150802DE6002AFF860B9601346FB80FB68BB62002309
S3150802DE707B62002387F823300023FB61BB6A5C7848
S3150802DE800DF08EFD03469C423AD1BB6A5B78002BA5
S3150802DE9036D0BB681B78052B06D0052B2BDC012B4D
S3150802DEA00DD0042B23D026E00DF07AFD0346052279
S3150802DEB01946B86A0DF011FDFEF7AAFB1FE0A54840
S3150802DEC000F076FBA44B9B783B76A34BDB787B76FC
S3150802DED007F11803A14918460EF0B1FAFFF708FF31
S3150802DEE09E4B1B881A469E49FFF73CF807E09D4859
S3150802DEF000F05EFB03E09C4800F05AFB00BF16E206
S3150802DF00BB6A5C780DF04CFD03469C4240F2D78012
S3150802DF10BB6A5B78013BDBB21846FDF761FA03463A
S3150802DF2087F82330BB6A5B781946904800F040FBB5
S3150802DF3097F82330013B0D2B00F2BA8001A252F862
S3150802DF4023F000BF7DDF020893DF0208A9DF02087B
S3150802DF50BFDF0208D5DF0208EBDF020801E002088C
S3150802DF6017E002082DE0020843E0020859E0020819
S3150802DF706FE0020885E002089BE002087C4800F090
S3150802DF8017FB00F07FFFFB881A46B9680DF0BCFF45
S3150802DF908EE0784800F00CFB00F0E2FFFB881A4698
S3150802DFA0B9680DF0B1FF83E0734800F001FBFDF795
S3150802DFB093FCFB881A46B9680DF0A6FF78E06F480D
S3150802DFC000F0F6FAF9F728F9FB881A46B9680DF04F
S3150802DFD09BFF6DE06A4800F0EBFAF9F767FAFB88EF
S3150802DFE01A46B9680DF090FF62E0664800F0E0FA5A
S3150802DFF0F3F71CF8FB881A46B9680DF085FF57E057
S3150802E000614800F0D5FAFDF7D5FCFB881A46B968CF
S3150802E0100DF07AFF4CE05D4800F0CAFAF9F76AF9A2
S3150802E020FB881A46B9680DF06FFF41E0584800F0C0
S3150802E030BFFAF9F7CDF9FB881A46B9680DF064FFFD
S3150802E04036E0544800F0B4FAF9F79EFAFB881A4605
S3150802E050B9680DF059FF2BE04F4800F0A9FAF9F715
S3150802E06001FBFB881A46B9680DF04EFF20E04B48C3
S3150802E07000F09EFAFDF746F9FB881A46B9680DF0D4
S3150802E08043FF15E0464800F093FAFDF749FBFB8883
S3150802E0901A46B9680DF038FF0AE0424800F088FAD5
S3150802E0A0FDF7ACFBFB881A46B9680DF02DFF00BFD9
S3150802E0B0BB681B7819463C4800F07AFA37E1BB6818
S3150802E0C01B78C13B052B00F2298101A252F823F0E5
S3150802E0D0E9E002081DE302083BE202085FE20208E1
S3150802E0E01DE30208F9E20208BB6802331B78D02B4B
S3150802E0F040F018812D4800F05BFABB6801331B78A3
S3150802E100013319462A4800F053FABB6801331B78D3
S3150802E1100133DBB218460DF031FC0023FB750DF016
S3150802E1203FFC03461C460DF059FC0346194607F107
S3150802E1301703012200920A462146B86A0DF0E7F94A
S3150802E140002387F82F30002387F82E30012387F81B
S3150802E1502F3061E030120408E0BF1F089433022012
S3150802E160963302204412040860120408781204083E
S3150802E1708412040894120408A4120408B4120408A7
S3150802E180C4120408D8120408EC120408FC12040883
S3150802E1901013040824130408381304084C1304083B
S3150802E1A06013040870130408801304088C13040807
S3150802E1B09813040897F82F301846FDF711F9034605
S3150802E1C0FF2B24D097F82F301846FDF709F9034696
S3150802E1D0FB750DF0E5FB03461A4697F82F301344F4
S3150802E1E0DCB20DF0FBFB0346194607F117030122C1
S3150802E1F000920A462146B86A0DF089F90DF0D0FB5D
S3150802E20003461A4697F82F30134487F82E3097F8A4
S3150802E2102F30013387F82F3097F82F30142BC9D9AE
S3150802E22000F06AFD7862BB6802331B7897F82E20E5
S3150802E230796AB86A0DF0C3F974E03F4800F0B8F994
S3150802E2400DF0AEFB0346002B6ED000F055FD78624A
S3150802E250FB88BA68796AB86A0DF0FDFA64E00DF0CF
S3150802E2609FFB03461C460DF0B9FB03461A460023DC
S3150802E270009300232146B86A0DF0E6F9BB6801331C
S3150802E2801B78FB61FB691B029BB2FB61BB6802330D
S3150802E2901B781A46FB691344FB61FB691B0223F0D0
S3150802E2A07F4323F0FF03FB61BB6803331B781A46DF
S3150802E2B0FB691344FB61FB691B02FB61BB68043300
S3150802E2C01B781A46FB691344FB611C4AFB691360F7
S3150802E2D000F012FD7862BB6802331B781A46796A27
S3150802E2E0B86A0DF009FABB6801330422194640F2EE
S3150802E2F0F170F5F773F91AE0114800F059F90DF0C3
S3150802E3004FFB0346002B11D000F0F6FC7862FB881F
S3150802E310BA68796AB86A0DF09EFA07E0094800F009
S3150802E32047F904E000BF02E000BF00E000BF00BFFB
S3150802E3303437BD4690BD00BFAC130408CC13022087
S3150802E340BC130408CC13040880B500AF4FF400626E
S3150802E35002490348FDF79CFB00BF80BD942B0220AF
S3150802E360E018022080B584B004AFFFF7EDFF074B33
S3150802E3700293074B0193074B0093044B064A07493E
S3150802E38007480DF037FB00BFBD4680BD2DDD0208EC
S3150802E3905DDE0208FC18022079DD02084822022006
S3150802E3A0F018022080B582B000AF7860396039680B
S3150802E3B07868FDF793FD03469BB218460837BD46B3
S3150802E3C080BD000080B5ADF6080D00AF0023A7F8A2
S3150802E3D006383B1D4FF40062002118460FF05EF91D
S3150802E3E01048FDF7DFFB034683F00103DBB2002B7F
S3150802E3F014D03B1D19460B48FFF7D4FF0346A7F86E
S3150802E4000638B7F80638002B07D0B7F806283B1D9A
S3150802E4101146184600F01AFA00E000BF07F6080788
S3150802E420BD4680BDE018022080B582B000AF034623
S3150802E430FB71FB1D012219460348FDF7CFFB00BFFE
S3150802E4400837BD4680BD00BF9834022080B582B029
S3150802E45000AF78600B467B807B681B780D2B04D156
S3150802E4600221064800F072F804E07B8819467868AB
S3150802E47000F06CF800BF0837BD4680BDEC130408EF
S3150802E48080B582B000AF00237B710023FB80802217
S3150802E490002129480FF002F92848FDF783FB0346B5
S3150802E4A083F00103DBB2002B1DD00BE0FB885A1C5C
S3150802E4B0FA801A467979204B9954FB887F2B0BD818
S3150802E4C000237B717B1D012219461C48FDF7C1FBFF
S3150802E4D00346002BEAD100E000BFFB88194616481E
S3150802E4E0FFF7B4FF23E016480BF066F90346202B24
S3150802E4F010D1134B0122A3F85C20114B0122A3F879
S3150802E5005E2001220F490E480AF05AFC0E4800F016
S3150802E5104FF80CE00A4BB3F85C20094BB3F85E30AF
S3150802E5209BB29A4203D0FEF709F8FEF70EF800BF2F
S3150802E5300837BD4680BD00BFE8380220983402205D
S3150802E54058160220E83C0220F013040880B582B06F
S3150802E55000AF78600B467B807A884FF47A737968C5
S3150802E56003480AF08EFB012318460837BD4680BDCC
S3150802E5705816022080B500AF802203490348FDF7EA
S3150802E58087FA00BF80BD00BFE83402209834022013
S3150802E59080B500AFFFF7EEFF0122034903480AF0F0
S3150802E5A00FFC00BF80BD00BFE83C022058160220BF
S3150802E5B00FB480B582B000AF4FF4807200211248C2
S3150802E5C00FF06CF807F114033B603A6839690E4894
S3150802E5D00FF04AF878600C4A0C490B480EF0CAFF4D
S3150802E5E00948F1F755FE03469BB21A460649012029
S3150802E5F000F068FB03467B607B6818460837BD4611
S3150802E600BDE8804004B07047F43C022008140408B0
S3150802E61080B582B000AF0346FB71FB1D0122194685
S3150802E6200348FDF7DBFA00BF0837BD4680BD00BFC9
S3150802E630A834022080B582B000AF78600B467B8092
S3150802E6407B881946786800F061F800BF0837BD462E
S3150802E65080BD000080B582B000AF00237B71002325
S3150802E660FB808022002124480FF018F82348FDF782
S3150802E67099FA034683F00103DBB2002B1DD00BE0A7
S3150802E680FB885A1CFA801A4679791B4B9954FB88DF
S3150802E6907F2B0BD800237B717B1D01221946174855
S3150802E6A0FDF7D7FA0346002BEAD100E000BFFB8844
S3150802E6B019461148FFF7BEFF19E011480BF07CF81E
S3150802E6C00346202B10D10E4B0122A3F85C200C4BDB
S3150802E6D00122A3F85E2001220A4909480AF070FBC2
S3150802E6E00948FFF765FF02E0054BB3F85E3000BF45
S3150802E6F00837BD4680BD00BF683B0220A834022009
S3150802E70080170220E93C02201414040880B582B05E
S3150802E71000AF78600B467B807A884FF47A73796803
S3150802E72003480AF0AEFA012318460837BD4680BDEB
S3150802E7308017022080B500AF802203490348FDF7FF
S3150802E740A7F900BF80BD00BF68350220A8340220A1
S3150802E75080B500AFFFF7EEFF0122034903480AF02E
S3150802E7602FFB00BF80BD00BFE93C022080170220B4
S3150802E77080B582B000AF0346FB71FB1D0122194624
S3150802E7800348FDF72BFA00BF0837BD4680BD00BF18
S3150802E790B834022080B584B000AF78600B467B801F
S3150802E7A00023FB810023FB810BE0FFF7B5FAFB8907
S3150802E7B07A6813441B7819460DF0BEFAFB890133B1
S3150802E7C0FB81FA897B889A42EFD300BF00BF1037D4
S3150802E7D0BD4680BD80B582B000AF00237B710023A1
S3150802E7E0FB804FF40072002116480EF057FF1648B8
S3150802E7F0FDF7D8F9034683F00103DBB2002B1DD0DF
S3150802E8000CE0FB885A1CFA801A4679790D4B995402
S3150802E810FB88B3F5007F0BD200237B717B1D012297
S3150802E82019460948FDF715FA0346002BE9D100E017
S3150802E83000BFFB8819460348FFF7ACFF00BF08373D
S3150802E840BD4680BD68390220B834022080B582B040
S3150802E85000AF78600B467B807A884FF47A737968C2
S3150802E86003480AF00EFA012318460837BD4680BD4A
S3150802E870EC16022080B500AF4FF400720249034835
S3150802E880FDF706F900BF80BDE8350220B83402203C
S3150802E89080B500AFFFF7EEFF04480AF0DBFB012262
S3150802E8A0034902480AF0EEFA00BF80BDEC160220C0
S3150802E8B0EA3C022080B582B000AF0346FB71FB1D1D
S3150802E8C0012219460348FDF789F900BF0837BD46F4
S3150802E8D080BD00BFC834022080B582B000AF786020
S3150802E8E00B467B807B881946786800F03FF800BFA4
S3150802E8F00837BD4680BD000080B582B000AF002350
S3150802E9007B710023FB808022002116480EF0C6FE8A
S3150802E9101548FDF747F9034683F00103DBB2002BDE
S3150802E9201CD00BE0FB885A1CFA801A4679790D4BE3
S3150802E9309954FB887F2B0BD800237B717B1D012200
S3150802E94019460948FDF785F90346002BEAD100E086
S3150802E95000BFFB8819460348FFF7BEFF00BF08370A
S3150802E960BD4680BDE83B0220C834022080B582B08D
S3150802E97000AF78600B467B807A884FF47A737968A1
S3150802E98003480AF07EF9012318460837BD4680BDBA
S3150802E9903015022080B500AF802203490348FDF7EF
S3150802E9A077F800BF80BD00BFE8370220C8340220CE
S3150802E9B080B500AFFFF7EEFF0122034903480AF0CC
S3150802E9C0FFF900BF80BD00BFEB3C022030150220D4
S3150802E9D080B582B000AF0346FB71FB1D01221946C2
S3150802E9E00348FDF7FBF800BF0837BD4680BD00BFE8
S3150802E9F0D834022080B582B000AF78600B467B809F
S3150802EA007B881946786800F061F800BF0837BD466A
S3150802EA1080BD000080B582B000AF00237B71002361
S3150802EA20FB808022002124480EF038FE2348FDF799
S3150802EA30B9F8034683F00103DBB2002B1DD00BE0C5
S3150802EA40FB885A1CFA801A4679791B4B9954FB881B
S3150802EA507F2B0BD800237B717B1D01221946174891
S3150802EA60FDF7F7F80346002BEAD100E000BFFB8862
S3150802EA7019461148FFF7BEFF19E011480AF09CFE35
S3150802EA800346202B10D10E4B0122A3F85C200C4B17
S3150802EA900122A3F85E2001220A4909480AF090F9E0
S3150802EAA00948FFF785FD02E0054BB3F85E3000BF63
S3150802EAB00837BD4680BD00BF683C0220D834022014
S3150802EAC0C4150220EC3C02202C14040880B582B03E
S3150802EAD000AF78600B467B807A884FF47A73796840
S3150802EAE003480AF0CEF8012318460837BD4680BD0A
S3150802EAF0C415022080B500AF802203490348FCF7FB
S3150802EB00C7FF00BF80BD00BF68380220D834022084
S3150802EB1080B500AFFFF7EEFF0122034903480AF06A
S3150802EB204FF900BF80BD00BFEC3C0220C41502208D
S3150802EB3080B582B000AF78607B681B682D4A934225
S3150802EB400DD12D4B1B781846FFF76EFC2A4B002277
S3150802EB501A700122284929480AF032F945E07B68E9
S3150802EB601B68274A934208D1264B1B781846FFF79B
S3150802EB70FFFD244B00221A7037E07B681B68224A85
S3150802EB8093420DD1214B1B781846FFF741FD1F4BC7
S3150802EB9000221A7001221D491D480AF011F924E0C3
S3150802EBA07B681B681B4A93420DD11B4B1B78184680
S3150802EBB0FFF780FE184B00221A70012216491748E1
S3150802EBC00AF0FEF811E07B681B68154A93420CD1DD
S3150802EBD0144B1B781846FFF7FBFE124B00221A70DD
S3150802EBE00122104910480AF0EBF800BF0837BD4663
S3150802EBF080BD00BF00380140E83C022058160220BA
S3150802EC0000440040EA3C022000480040E93C022059
S3150802EC1080170220004C0040EB3C022030150220EF
S3150802EC2000500040EC3C0220C415022080B582B098
S3150802EC3000AF786078680AF0D4FD03461B4A136071
S3150802EC407B681B681A4A934204D1FDF777FCFDF7E5
S3150802EC507CFC26E07B681B68164A934204D1FDF7C2
S3150802EC607BFCFDF78DFC1CE07B681B68124A93420D
S3150802EC7004D1FDF78DFCFDF795FC12E07B681B6855
S3150802EC800E4A934204D1FDF795FCFDF79DFC08E078
S3150802EC907B681B680A4A934203D1FDF79DFCFDF780
S3150802ECA0A5FC00BF0837BD4680BD00BFF03C022068
S3150802ECB0003801400044004000480040004C004033
S3150802ECC00050004080B582B000AF03463960FB7140
S3150802ECD01346BB80FB79012B06D1BA884FF47A73A7
S3150802ECE03968044809F0CDFF012318460837BD469E
S3150802ECF080BD00BF5816022080B400AF024B1846EA
S3150802ED00BD465DF8047B7047043E022080B582B09A
S3150802ED1000AF78600B467B807B881946786800F0DE
S3150802ED2005F800BF0837BD4680BD000080B584B02F
S3150802ED3000AF786039600023FB603B689BB21A46D5
S3150802ED4079680448FDF7B9F80346FB6000BF103737
S3150802ED50BD4680BDF43D022080B586B000AFF8609E
S3150802ED60B9601346FB80FB683B610123FB82BB68E3
S3150802ED701A783B691A70BB685A783B695A70BB683D
S3150802ED809A783B699A703B691B78002B1BD13B69C1
S3150802ED905B78002B17D13B699B78AB2B13D10323E6
S3150802EDA0FB820BE03B699868FB8ABA6813441B78B6
S3150802EDB019460CF0C1FFFB8A0133FB82FA8AFB88EB
S3150802EDC09A42EFD31FE0BB6801331B7818460CF052
S3150802EDD0C1FD0346002B13D00323FB820BE03B69DC
S3150802EDE09868FB8ABA6813441B7819460CF0A4FF84
S3150802EDF0FB8A0133FB82FA8AFB889A42EFD302E046
S3150802EE000CF0CEFDFFE700BF1837BD4680BD80B4C3
S3150802EE1085B000AFF860B9601346FB8000BF1437AF
S3150802EE20BD465DF8047B704780B500AF4FF480722B
S3150802EE3002490348FCF72CFE00BF80BDA8500220F9
S3150802EE40F43D022080B584B004AFFFF7EDFF074B0F
S3150802EE500293074B0193074B0093044B064A074953
S3150802EE6007480CF0C7FD00BFBD4680BD0DED020880
S3150802EE700FEE0208103E022059ED02085C470220F6
S3150802EE80043E022080B400AF024B1846BD465DF828
S3150802EE90047B7047C451022080B582B000AF786007
S3150802EEA00B467B807B881A4679684FF40070FAF71E
S3150802EEB0A5F900BF0837BD4680BD000090B589B0E8
S3150802EEC002AFF860B9601346FB800120FCF798FA96
S3150802EED003460133DBB23B75CE237B75D623BB755E
S3150802EEE03B7D1946BB681B781A460B48FFF760FB41
S3150802EEF0FEF712FF0446FEF705FF014607F1140264
S3150802EF00FB880093BB6820460CF0A1FE00BF00BF39
S3150802EF101C37BD4690BD00BF4414040880B500AF37
S3150802EF204FF4807202490348FCF7B2FD00BF80BD68
S3150802EF30105B0220A851022080B500AFFFF7EEFF52
S3150802EF40034B044A044905480CF0CDFA00BF80BDBC
S3150802EF5099EE0208BDEE0208C4510220B8510220F9
S3150802EF6080B400AF024B1846BD465DF8047B704775
S3150802EF702C5C022080B582B000AF78600B467B809D
S3150802EF807B881A4679684FF48060FAF737F900BF2A
S3150802EF900837BD4680BD000090B589B002AFF8605B
S3150802EFA0B9601346FB800220FCF72AFA03460133AE
S3150802EFB0DBB23B75CE237B75D623BB753B7D1946E3
S3150802EFC0BB681B781A46FB880A48FFF7F1FAFEF770
S3150802EFD0A3FE0446FEF796FE014607F11402FB88D5
S3150802EFE00093BB6820460CF032FE00BF00BF1C37F8
S3150802EFF0BD4690BD6C14040880B500AF4FF480720C
S3150802F00002490348FCF744FD00BF80BD786502202B
S3150802F010105C022080B500AFFFF7EEFF034B044AEF
S3150802F020044905480CF05FFA00BF80BD75EF020877
S3150802F03099EF02082C5C0220205C02200D488546C6
S3150802F040FEF79AFD0C480D490D4A002302E0D458F2
S3150802F050C4500433C4188C42F9D30A4A0A4C002312
S3150802F06001E013600432A242FBD30EF07FFBFDF7E8
S3150802F070E7FAFEE700000A20000000200802002046
S3150802F0805019040808020020CC670220FEE7000097
S3150802F09080B500AF032000F06BF903F021FD0246AC
S3150802F0A00B4B1B6A03F00F030A49CB5C22FA03F3E4
S3150802F0B0094A13600F2000F011F80346002B01D00D
S3150802F0C0012302E0FDF789FF0023184680BD00BF31
S3150802F0D0000C0244981404083400002080B582B05B
S3150802F0E000AF7860154B1B78002B01D1012321E074
S3150802F0F0134B1A68114B1B7819464FF47A73B3FBF4
S3150802F100F1F3B2FBF3F3184600F073F90346002B4A
S3150802F11001D001230EE07B680F2B0AD800227968FA
S3150802F1204FF0FF3000F02FF9064A7B681360002380
S3150802F13000E0012318460837BD4680BD3C00002082
S3150802F140340000203800002080B400AF064B1B783C
S3150802F1501A46064B1B681344044A136000BFBD4691
S3150802F1605DF8047B704700BF3C00002078660220E9
S3150802F17080B400AF034B1B681846BD465DF8047B96
S3150802F180704700BF7866022080B485B000AF786009
S3150802F1907B6803F00703FB600C4BDB68BB60BA684D
S3150802F1A04FF6FF031340BB60FB681A02BB681343A2
S3150802F1B043F0BF6343F40033BB60044ABB68D360C1
S3150802F1C000BF1437BD465DF8047B704700ED00E0CA
S3150802F1D080B400AF044BDB681B0A03F0070318462A
S3150802F1E0BD465DF8047B704700ED00E080B483B04D
S3150802F1F000AF0346FB80B7F90630002B0BDBFB8812
S3150802F20003F01F020749B7F906305B09012000FA25
S3150802F21002F241F8232000BF0C37BD465DF8047B95
S3150802F220704700BF00E100E080B483B000AF034638
S3150802F230FB80B7F90630002B12DBFB8803F01F02AE
S3150802F2400A49B7F906305B09012000FA02F22033AF
S3150802F25041F82320BFF34F8F00BFBFF36F8F00BF64
S3150802F26000BF0C37BD465DF8047B704700E100E03D
S3150802F27080B483B000AF03463960FB80B7F9063025
S3150802F280002B0ADB3B68DAB20C49B7F906301201E1
S3150802F290D2B20B4483F800230AE03B68DAB2084983
S3150802F2A0FB8803F00F03043B1201D2B20B441A7611
S3150802F2B000BF0C37BD465DF8047B704700E100E0ED
S3150802F2C000ED00E080B489B000AFF860B9607A60FA
S3150802F2D0FB6803F00703FB61FB69C3F10703042B11
S3150802F2E028BF0423BB61FB690433062B02D9FB69D9
S3150802F2F0033B00E000237B614FF0FF32BB6902FA51
S3150802F30003F3DA43BB681A407B699A404FF0FF3130
S3150802F3107B6901FA03F3D9437B680B40134318460A
S3150802F3202437BD465DF8047B7047000080B582B07D
S3150802F33000AF78607B68013BB3F1807F01D301237C
S3150802F3400FE00A4A7B68013B53600F214FF0FF30FA
S3150802F350FFF78EFF054B00229A60044B07221A60BC
S3150802F360002318460837BD4680BD00BF10E000E0FE
S3150802F37080B582B000AF78607868FFF705FF00BFF6
S3150802F3800837BD4680BD80B586B000AF0346B96072
S3150802F3907A60FB81FFF71CFF78617A68B968786939
S3150802F3A0FFF790FF0246B7F90E3011461846FFF7E7
S3150802F3B05FFF00BF1837BD4680BD80B582B000AF7B
S3150802F3C00346FB80B7F906301846FFF70FFF00BF62
S3150802F3D00837BD4680BD80B582B000AF0346FB80C4
S3150802F3E0B7F906301846FFF71FFF00BF0837BD46B4
S3150802F3F080BD80B582B000AF78607868FFF796FF67
S3150802F400034618460837BD4680BD000080B584B05D
S3150802F41000AF7860FFF7ACFEF8607B68002B01D17D
S3150802F4200123B9E07B681B6823F47F6323F00F038B
S3150802F430BB607B681B685A697B681B6842F00602D8
S3150802F4405A610FE0FFF794FE0246FB68D31A052BB2
S3150802F45008D97B6810229A657B68032283F85420B0
S3150802F460012399E07B681B685B6903F00103002BA3
S3150802F470E8D17B681B6800221A607B681B68002239
S3150802F4805A617B681B6800221A647B681B68002223
S3150802F4905A647B681B6800229A647B681B68002290
S3150802F4A0DA647B681B6800221A657B681B6800227F
S3150802F4B0DA677B681B683A4A934222D07B681B68E4
S3150802F4C0384A93421DD07B681B68374A934218D044
S3150802F4D07B681B68354A934213D07B681B68344A9B
S3150802F4E093420ED07B681B68324A934209D07B68E6
S3150802F4F01B68314A934204D07B681B682F4A9342A1
S3150802F50001D1012300E00023002B07D07B681B688A
S3150802F51000225A657B681B6800229A65BB685A688E
S3150802F5207B681B68C3F30B03503BDB0903F01F031D
S3150802F530012101FA03F3DB431A40BB685A607B6870
S3150802F5401B684FF4FE42DA607B6800221A667B6803
S3150802F55000225A667B6800229A667B680022DA666F
S3150802F5607B6800221A677B6800225A677B68DB6D14
S3150802F570002B02D07B680022DA657B6800221A65B6
S3150802F5807B6800229A657B68002283F854207B6890
S3150802F590002283F84C20002318461037BD4680BD4A
S3150802F5A05003024050030250D0030240D0030250D7
S3150802F5B05013024050130250D0130240D013025087
S3150802F5C080B584B000AFF860B9607A603B60FB68CA
S3150802F5D0002B01D101234FE0FB6893F84C30012B35
S3150802F5E001D1022348E0FB68012283F84C20FB681C
S3150802F5F093F85430DBB2012B36D1FB68022283F82A
S3150802F6005420FB6800229A653B687A68B968F868EC
S3150802F61000F09DFAFB681B685A69FB681B6842F48E
S3150802F620BA425A61FB685B6E002B07D0FB681B68FF
S3150802F6305A69FB681B6842F400725A61FB681B6FC1
S3150802F640002B07D0FB681B685A69FB681B6842F4E3
S3150802F65000525A61FB681B685A69FB681B6842F0CC
S3150802F66001025A61002307E0FB6840229A65FB689B
S3150802F670002283F84C20012318461037BD4680BD68
S3150802F68080B584B000AF7860FFF772FDF8607B68DA
S3150802F690002B01D101236BE07B6893F85430DBB26F
S3150802F6A0022B08D07B6820229A657B68002283F8A1
S3150802F6B04C2001235CE07B681B685A697B681B68DF
S3150802F6C042F004025A617B68052283F8542020E03E
S3150802F6D0FFF74EFD0246FB68D31A052B19D97B683C
S3150802F6E09B6D43F010027B689A657B68032283F858
S3150802F6F054207B681B6D03F08003002B03D07B68C4
S3150802F7005B6F01221A737B68002283F84C2001235F
S3150802F7102EE07B681B681B6903F40053002BD7D0C5
S3150802F7207B681B685A697B681B6842F002025A6149
S3150802F7307B68042283F854207B681B684FF4FE42D8
S3150802F740DA607B68012283F854207B681B6D03F01C
S3150802F7508003002B07D07B685B6F01221A737B68D4
S3150802F7601B6800229A647B68002283F84C200023D7
S3150802F77018461037BD4680BD80B483B000AF7860A6
S3150802F7807B68002B01D1012319E07B6893F854307A
S3150802F790DBB2022B04D07B6820229A6501230EE095
S3150802F7A07B68042283F854207B681B685B697A6845
S3150802F7B0126843F4005343F00403536100231846C6
S3150802F7C00C37BD465DF8047B704780B586B000AF3E
S3150802F7D078607B681B6823F47F6323F00F037B61E1
S3150802F7E07B681B68C3F30B03503BDB0903F01F035B
S3150802F7F0012202FA03F33B617B69DB683A6913402B
S3150802F800FB60FB68002B00F054817B681B681B6950
S3150802F81003F48063002B11D07B681B685B6903F4D1
S3150802F8208063002B0AD07B681B684FF48062DA601B
S3150802F8307B689B6D43F001027B689A657B681B684F
S3150802F8401B6903F40063002B11D07B681B685B6994
S3150802F85003F40063002B0AD07B681B684FF400622E
S3150802F860DA607B689B6D43F002027B689A657B6867
S3150802F8701B681B6903F48053002B11D07B681B6835
S3150802F8805B6903F48053002B0AD07B681B684FF42C
S3150802F8908052DA607B689B6D43F004027B689A6546
S3150802F8A07B681B681B6903F48043002B11D07B68B5
S3150802F8B01B685B6903F48043002B0AD07B681B68CC
S3150802F8C04FF48042DA607B689B6D43F008027B68DE
S3150802F8D09A657B681B681B6903F40073002B13D0B7
S3150802F8E07B681B685B6903F40073002B0CD07B688A
S3150802F8F01B684FF40072DA607B685B6E002B03D0DC
S3150802F9007B685B6E786898477B681B681B6903F49B
S3150802F9100053002B59D07B681B685B6903F40053BC
S3150802F920002B52D07B681B684FF40052DA607B6862
S3150802F93093F85430DBB2042B3BD17B681B685A69B7
S3150802F9407B681B6822F400525A617B681B685A69F5
S3150802F9507B681B6842F002025A617B681B685B6916
S3150802F96003F00103002B04D07B68032283F854209A
S3150802F97003E07B68012283F854207B681B6D03F041
S3150802F9808003002B07D07B685B6F01221A737B68A2
S3150802F9901B6800229A647B68002283F84C207B68E5
S3150802F9A0DB6E002B00F087807B68DB6E78689847F1
S3150802F9B081E07B68052283F854207B681B6F002B45
S3150802F9C003D07B681B6F786898477B681B681B693E
S3150802F9D003F48073002B39D07B681B685B6903F4D8
S3150802F9E08073002B32D07B681B6D03F08003002BDB
S3150802F9F012D07B681B68DB6F002B16D17B681B68ED
S3150802FA009B6C002B11D17B68012283F854207B68FA
S3150802FA105B6F01221A7308E07B681B689B6C002BDC
S3150802FA2003D17B68012283F854207B681B684FF454
S3150802FA304072DA607B68002283F84C207B681B6E72
S3150802FA40002B03D07B681B6E786898477B689B6D92
S3150802FA50002B31D07B681B685A697B681B6842F0A9
S3150802FA6002025A617B681B685B6903F00103002B7B
S3150802FA7004D07B68032283F8542003E07B680122C2
S3150802FA8083F854207B681B6D03F08003002B03D098
S3150802FA907B685B6F01221A737B68002283F84C200D
S3150802FAA07B689B6E002B07D07B689B6E78689847AD
S3150802FAB002E000BF00E000BF1837BD4680BD80B433
S3150802FAC083B000AF78607B689B6D18460C37BD46DD
S3150802FAD05DF8047B704780B485B000AF7860396002
S3150802FAE07B68002B01D101232BE07B681B6823F47A
S3150802FAF07F6323F00F03FB607B681B68C3F30B036A
S3150802FB00503BDB0903F01F03012202FA03F3BB6031
S3150802FB103B6803F01003002B12D03B6803F0110375
S3150802FB20112B06D1FB685A68BB681A43FB685A60F0
S3150802FB3006E0FB685A68BB68DB431A40FB685A60F2
S3150802FB40002318461437BD465DF8047B704780B417
S3150802FB5085B000AFF860B9607A603B60FB681B68E5
S3150802FB609B6C1B0C1B043A6891B2FA6812680B4329
S3150802FB709364FB681B684FF4FE42DA60FB681B68F5
S3150802FB80BA68DA64FB681B687A681A6500BF1437B4
S3150802FB90BD465DF8047B704780B584B000AF7860D7
S3150802FBA0FFF7E6FAF8607B68002B01D10123DBE058
S3150802FBB07B681B686E4A934200F09F807B681B68CD
S3150802FBC06C4A934200F099807B681B686A4A9342A2
S3150802FBD000F093807B681B68684A934200F08D8028
S3150802FBE07B681B68664A934200F087807B681B68BD
S3150802FBF0644A934200F081807B681B68624A93429A
S3150802FC007BD07B681B68614A934276D07B681B6807
S3150802FC105F4A934271D07B681B685E4A93426CD0F6
S3150802FC207B681B685C4A934267D07B681B685B4AA1
S3150802FC30934262D07B681B68594A93425DD07B68BF
S3150802FC401B68584A934258D07B681B68564A9342A7
S3150802FC5053D07B681B68554A93424ED07B681B6813
S3150802FC60534A934249D07B681B68524A934244D00E
S3150802FC707B681B68504A93423FD07B681B684F4A91
S3150802FC8093423AD07B681B684D4A934235D07B68CB
S3150802FC901B684C4A934230D07B681B684A4A934297
S3150802FCA02BD07B681B68494A934226D07B681B681F
S3150802FCB0474A934221D07B681B68464A93421CD026
S3150802FCC07B681B68444A934217D07B681B68434A81
S3150802FCD0934212D07B681B68414A93420DD07B68D7
S3150802FCE01B68404A934208D07B681B683E4A934287
S3150802FCF003D07B681B683D4A93427B68002283F8DF
S3150802FD004C207B68022283F854207B681B685A6958
S3150802FD107B681B6842F006025A610FE0FFF728FA71
S3150802FD200246FB68D31A052B08D97B6810229A6506
S3150802FD307B68032283F85420012315E07B681B683D
S3150802FD405B6903F00103002BE8D1786800F0BAFA80
S3150802FD507B689A6C7B681A657B6800229A657B6861
S3150802FD60012283F85420002318461037BD4680BD69
S3150802FD705000024050000250D0000240D00002500B
S3150802FD805001024050010250D0010240D0010250F7
S3150802FD905002024050020250D0020240D0020250E3
S3150802FDA05003024050030250D0030240D0030250CF
S3150802FDB05010024050100250D0100240D01002508B
S3150802FDC05011024050110250D0110240D011025077
S3150802FDD05012024050120250D0120240D012025063
S3150802FDE05013024050130250D0130240D01302504F
S3150802FDF080B586B000AF78607B68002B03D07B683D
S3150802FE005B6F002B01D1012382E07B6893F85430A3
S3150802FE10FB757B681B685B6903F480333B61FB7D7A
S3150802FE20012B05D0FB7D022B6AD13B69002B67D0DB
S3150802FE307B6893F85430DBB2012B57D17B6893F871
S3150802FE404C30012B01D1022362E07B68012283F840
S3150802FE504C207B68022283F854207B685B6F02225F
S3150802FE601A737B6800229A657B685B6F00221A61A7
S3150802FE707B681B685A697B681B6842F4BA425A61F6
S3150802FE807B685B6E002B07D07B681B685A697B68A8
S3150802FE901B6842F400725A617B681B6F002B07D0FD
S3150802FEA07B681B685A697B681B6842F400525A6170
S3150802FEB07B685B6F1B6807F10C010022184600F08D
S3150802FEC01DFD7B685B6F1B6819467B681A680B0CFD
S3150802FED01B0413607B685B6F1B681A464FF6FC733C
S3150802FEE01340F9687A6812680B43D3677B681B6804
S3150802FEF05A697B681B6842F001025A61002307E0CF
S3150802FF007B6840229A657B68002283F84C2001238D
S3150802FF1018461837BD4680BD80B582B000AF7860F6
S3150802FF2039607B68002B02D03B68002B01D1012384
S3150802FF3004E03968786800F01DFB00231846083784
S3150802FF40BD4680BD80B58CB000AFF860B9607A60F6
S3150802FF50FB68002B02D07B68002B01D10123B6E097
S3150802FF60FB685B69012B04D1FB6804221A61012331
S3150802FF70ADE0FB681B687A68B968184600F052FC5F
S3150802FF800346002B04D0FB6805221A6101239EE072
S3150802FF90FB681B687A68B968184600F073FC034662
S3150802FFA0002B04D0FB6804221A6101238FE0FB6848
S3150802FFB002221A73FB6800221A6107F1280207F166
S3150802FFC02C031946786800F099FCFB681B68002B1D
S3150802FFD01AD1BB68002B06D1FB687A681A60FB68DF
S3150802FFE001229A606CE0FB68BA681A607A684FF672
S3150802FFF0FC731340F96ABA6A1943BB6843F82210BC
S31508030000FB6802229A605BE0BB68002B0FD1FB6892
S315080300101B681A464FF6FC731340F96ABA6A194302
S315080300207B6843F82210FB687A681A6043E0BB6A68
S315080300307B6107F114031A46B968F86800F08EFC69
S315080300400346002B32D1FA69FB689B689A421AD198
S31508030050FB685B68002B0BD0FB685B681A464FF698
S31508030060FC731340F96ABA6A19437B6843F822108A
S315080300707A684FF6FC731340F96ABA6A1943BB6880
S3150803008043F8221017E0B96ABA6ABB6853F8211015
S315080300907B6843F822107A684FF6FC731340F96AB3
S315080300A0BA6A1943BB6843F8221004E0FB680622C0
S315080300B01A6101230BE0FB689B685A1CFB689A606C
S315080300C0FB6800221A61FB6801221A73002318468B
S315080300D03037BD4680BD80B58AB000AF78607B688F
S315080300E0002B01D1012352E07B681B68002B04D146
S315080300F07B6802221A61012349E07B685B68002B4F
S315080301000CD07B685A687B681B689A4201D1002326
S315080301103DE07B6804221A61012338E07B685B694A
S31508030120012B04D17B6804221A6101232FE07B6823
S3150803013002221A737B6800221A617B681B6807F11F
S31508030140200207F12401184600F0D8FB3B6AFB603E
S3150803015007F10C031A460021786800F0FFFB7B6859
S315080301601B681A464FF6FC731340796ABA69104638
S315080301703A6A0B4340F822307B681A687B685A60F0
S315080301807B6800221A617B6801221A7300231846CA
S315080301902837BD4680BD000080B485B000AF7860BF
S315080301A039607B68002B02D03B68002B01D1012301
S315080301B072E07B6893F85430FB737B6893F854308A
S315080301C0DBB2022B02D0FB7B052B08D17B684022CE
S315080301D09A657B68002283F84C2001235CE03B6820
S315080301E01B7BDBB2022B04D13B6801221A61012374
S315080301F052E07B681B682B4A934222D07B681B68B4
S31508030200294A93421DD07B681B68284A934218D013
S315080302107B681B68264A934213D07B681B68254A6A
S3150803022093420ED07B681B68234A934209D07B68A6
S315080302301B68224A934204D07B681B68204A934270
S3150803024001D1012300E00023002B0BD13B681B6877
S315080302501B6A03F00203002B04D03B6803221A61CE
S31508030260012319E07B681B6D812B08D13B685B680A
S31508030270002B0DD13B6804221A6101230CE03B686D
S315080302805B68002B04D03B6804221A61012303E050
S315080302907B683A685A67002318461437BD465DF8E3
S315080302A0047B70475003024050030250D0030240B8
S315080302B0D00302505013024050130250D013024089
S315080302C0D013025080B485B000AF78607B689A6B10
S315080302D07B68DB6B1343FB607B681B68854A934229
S315080302E000F0A0807B681B68834A934200F09A80DB
S315080302F07B681B68814A934200F094807B681B687D
S315080303007F4A934200F08E807B681B687D4A93423E
S3150803031000F088807B681B687B4A934200F08280E2
S315080303207B681B68794A93427CD07B681B68784A4A
S31508030330934277D07B681B68764A934272D07B6870
S315080303401B68754A93426DD07B681B68734A934250
S3150803035068D07B681B68724A934263D07B681B68C4
S31508030360704A93425ED07B681B686F4A934259D0A2
S315080303707B681B686D4A934254D07B681B686C4A3A
S3150803038093424FD07B681B686A4A93424AD07B687C
S315080303901B68694A934245D07B681B68674A934240
S315080303A040D07B681B68664A93423BD07B681B68D0
S315080303B0644A934236D07B681B68634A934231D0BA
S315080303C07B681B68614A93422CD07B681B68604A2A
S315080303D0934227D07B681B685E4A934222D07B6888
S315080303E01B685D4A93421DD07B681B685B4A934230
S315080303F018D07B681B685A4A934213D07B681B68DC
S31508030400584A93420ED07B681B68574A934209D0D1
S315080304107B681B68554A934204D07B681B68544A19
S31508030420934201D1012300E00023002B04D07B680B
S315080304301B6CFA681343FB607B681B685B6923F4D0
S3150803044043017B681B68FA680A435A617B681B6821
S3150803045000221A647B681B687A68526C5A647B6844
S315080304601B6800229A647B681B680022DA647B682F
S315080304701B6800221A657B681B682A4A934222D0A6
S315080304807B681B68284A93421DD07B681B68274AEA
S31508030490934218D07B681B68254A934213D07B681E
S315080304A01B68304A93420ED07B681B682E4A9342D8
S315080304B009D07B681B682D4A934204D07B681B6866
S315080304C02B4A934201D1012300E00023002B07D0D6
S315080304D07B681B6800225A657B681B6800229A653D
S315080304E07B681B680022DA6700BF1437BD465DF8D0
S315080304F0047B70475000024050000250D00002406F
S31508030500D00002505001024050010250D00102406F
S31508030510D00102505002024050020250D00202405B
S31508030520D00202505003024050030250D003024047
S31508030530D00302505010024050100250D01002400F
S31508030540D01002505011024050110250D0110240EF
S31508030550D01102505012024050120250D0120240DB
S31508030560D01202505013024050130250D0130240C7
S31508030570D013025080B485B000AF786039607B68C9
S315080305805A697B68DB691A437B68DB6B1A437B68AA
S315080305901B691A437B689B691A433B681A607B6825
S315080305A01B6803F02003002B17D03B681A687B6887
S315080305B0D96A7B689B6B19437B689B6A013B1B055E
S315080305C003F07C7319437B685B6A013B1B0103F4E5
S315080305D07C730B431A433B681A607B681A6B7B6808
S315080305E0596840F2FF230B401A433B685A607B68FD
S315080305F0DB68B3F5806F0CD17B681B6803F02003B7
S31508030600002B11D03B685B6843F480623B685A60F1
S315080306100AE07B68DB68B3F5007F05D13B685B6856
S3150803062043F400723B685A603B685A687B685B6BA5
S315080306301A433B685A607B685B6C002B0FD03B6898
S315080306405A687B68196C7B685B6C19437B689B6C7F
S315080306501B0403F47C130B431A433B685A607B68F9
S315080306609B6E9AB23B689A607B681B6803F0020329
S31508030670002B4ED03B689A687B68DB6C013B1904F8
S31508030680664B0B401A433B689A607B681B6D002BCD
S3150803069006DA3B689B6843F080523B689A6005E03C
S315080306A03B689B6823F080523B689A607B685B6D66
S315080306B0002B06DA3B689B6843F000523B689A6056
S315080306C005E03B689B6823F000523B689A607B68A9
S315080306D09B6D002B06DA3B689B6843F080423B68B8
S315080306E09A6005E03B689B6823F080423B689A6002
S315080306F07B68DB6D002B06DA3B689B6843F0004298
S315080307003B689A6005E03B689B6823F000423B68B8
S315080307109A607B681A6E3B68DA607B685A6E3B6838
S315080307201A617B681B6803F00203002B59D07B68A8
S315080307301B6D002B09DA7B681B6D5B42FB60FB684C
S31508030740C3F30C023B685A6105E07B681B6DC3F370
S315080307500C023B685A617B685B6D002B0DDA7B687C
S315080307605B6D5B42FB603B685A69FB6819042C4B5B
S315080307700B401A433B685A6109E03B685A697B6830
S315080307805B6D1904264B0B401A433B685A617B6819
S315080307909B6D002B08DA7B689B6D5B42FB60FB68ED
S315080307A09AB23B689A6104E07B689B6D9AB23B6890
S315080307B09A617B68DB6D002B0BDA7B68DB6D5B422A
S315080307C0FB603B689A69FB681B041A433B689A619A
S315080307D007E03B689A697B68DB6D1B041A433B6831
S315080307E09A617B681A683B681A627B681B6803F020
S315080307F00203002B06D03B681B6A43F4E0623B689E
S315080308001A6205E03B681B6A43F4A0623B681A62F6
S3150803081000BF1437BD465DF8047B70470000FF0729
S315080308200000FF1F80B487B000AFF860B9607A6034
S31508030830FA68BB681A437B6813431B0C1B043B61AA
S3150803084000237B61FB68002B02D0FB687B610AE00F
S31508030850BB68002B02D0BB687B6104E07B68002B76
S3150803086001D07B687B617B691B0C1B043A699A423E
S3150803087001D0012300E0002318461C37BD465DF866
S31508030880047B704780B487B000AFF860B9607A60BC
S3150803089000237B61FB68002B04D0FB681B6ADBB271
S315080308A07B610EE0BB68002B04D0BB681B6ADBB216
S315080308B07B6106E07B68002B03D07B681B6ADBB28F
S315080308C07B61BB68002B07D0BB681B6ADBB27A69FE
S315080308D09A4201D002230BE07B68002B07D07B6882
S315080308E01B6ADBB27A699A4201D0032300E000232C
S315080308F018461C37BD465DF8047B704780B485B03F
S3150803090000AFF860B9607A60FB681B6A03F00203FC
S31508030910002B0CD0BB68002B02D0BB680D4A1A60AB
S315080309207B68002B0FD07B6807221A600BE0BB6835
S31508030930002B02D0BB68084A1A607B68002B02D0DA
S315080309407B6805221A6000BF1437BD465DF8047B31
S31508030950704700BF000001FE000001F880B489B0AB
S3150803096000AFF860B9607A600023FB610023BB61BE
S3150803097000237B617B681B683B61BB68002B42D104
S315080309801DE0FB69002B07D1FB681B681A464FF667
S31508030990FC731340BB610FE0BB697B61FB681B6893
S315080309A01B0C1B04BA6913441A463B6952F82320E5
S315080309B04FF6FC731340BB61FB690133FB61FB68AC
S315080309C09B68FA699A42DCD329E0FB69002B07D1B5
S315080309D0FB681B681A464FF6FC731340BB610FE0AE
